:020000040000FA
:100000000002040000000000D87E0000D87E00003E
:10001000D87E0000D87E0000D87E0000D87E000088
:10002000D87E0000D87E0000D87E0000D87E000078
:10003000D87E0000D87E0000D87E0000D87E000068
:10004000D87E0000D87E0000D87E0000D87E000058
:10005000D87E00000E2F0000342F0000D87E000054
:10006000D87E0000D87E0000D87E0000D87E000038
:10007000D87E0000D87E0000D87E0000D87E000028
:10008000D87E0000D87E0000D87E0000D87E000018
:10009000D87E0000D87E0000D87E0000D87E000008
:1000A000D87E0000D87E0000D87E0000D87E0000F8
:1000B000D87E0000D87E0000D87E0000D87E0000E8
:1000C000D87E0000D87E0000D87E0000D87E0000D8
:1000D000D87E0000D87E0000D87E0000D87E0000C8
:1000E000D87E0000D87E0000D87E0000D87E0000B8
:1000F000D87E0000D87E0000D87E0000D87E0000A8
:10010000D87E0000D87E0000D87E0000D87E000097
:10011000D87E0000D87E0000D87E0000D87E000087
:10012000D87E0000D87E0000D87E0000D87E000077
:10013000D87E0000D87E0000D87E0000D87E000067
:10014000D87E0000D87E0000D87E0000D87E000057
:10015000D87E0000D87E0000D87E0000D87E000047
:10016000D87E0000D87E0000D87E0000D87E000037
:10017000D87E0000D87E0000D87E0000D87E000027
:10018000D87E0000D87E0000D87E0000D87E000017
:10019000D87E0000D87E0000D87E0000D87E000007
:1001A000D87E0000D87E0000D87E0000D87E0000F7
:1001B000D87E0000D87E0000D87E0000D87E0000E7
:1001C000D87E0000D87E0000D87E0000D87E0000D7
:1001D000D87E0000D87E0000D87E0000D87E0000C7
:1001E000D87E0000D87E0000D87E0000D87E0000B7
:1001F000D87E0000D87E0000D87E0000D87E0000A7
:10020000FFFFFF00FFFFFF00D87E0000D87E000048
:10021000D87E0000D87E0000D87E0000D87E000086
:10022000D87E0000D87E0000D87E0000D87E000076
:10023000D87E0000D87E0000D87E0000D87E000066
:10024000D87E0000D87E0000D87E0000D87E000056
:10025000D87E00000E2F0000342F0000D87E000052
:10026000D87E0000D87E0000D87E0000D87E000036
:10027000D87E0000D87E0000D87E0000D87E000026
:10028000D87E0000D87E0000D87E0000D87E000016
:10029000D87E0000D87E0000D87E0000D87E000006
:1002A000D87E0000D87E0000D87E0000D87E0000F6
:1002B000D87E0000D87E0000D87E0000D87E0000E6
:1002C000D87E0000D87E0000D87E0000D87E0000D6
:1002D000D87E0000D87E0000D87E0000D87E0000C6
:1002E000D87E0000D87E0000D87E0000D87E0000B6
:1002F000D87E0000D87E0000D87E0000D87E0000A6
:10030000D87E0000D87E0000D87E0000D87E000095
:10031000D87E0000D87E0000D87E0000D87E000085
:10032000D87E0000D87E0000D87E0000D87E000075
:10033000D87E0000D87E0000D87E0000D87E000065
:10034000D87E0000D87E0000D87E0000D87E000055
:10035000D87E0000D87E0000D87E0000D87E000045
:10036000D87E0000D87E0000D87E0000D87E000035
:10037000D87E0000D87E0000D87E0000D87E000025
:10038000D87E0000D87E0000D87E0000D87E000015
:10039000D87E0000D87E0000D87E0000D87E000005
:1003A000D87E0000D87E0000D87E0000D87E0000F5
:1003B000D87E0000D87E0000D87E0000D87E0000E5
:1003C000D87E0000D87E0000D87E0000D87E0000D5
:1003D000D87E0000D87E0000D87E0000D87E0000C5
:1003E000D87E0000D87E0000D87E0000D87E0000B5
:1003F000D87E0000D87E0000D87E0000D87E0000A5
:10040000CFCC2100007F2200000188000000000006
:100410000C00070080642600010020001100070086
:10042000000020000000E000020032000000020096
:1004300000000000B47B0200000000000040DA0071
:100440000000FE004440A900C0AB21000000E00015
:100450000300320000002000A00188004440A800F2
:100460000000060091018800800078000000EB0089
:1004700015003700E280400032A0B4009101BA00BC
:10048000E280400032A0B4009102BA00E280400055
:1004900032A0B4000002EB00472BDE00F507B200EB
:1004A000602CE10004003A000059EB008301E900F0
:1004B000FDFF3E00040037006128E100010032002A
:1004C0000082EB00040007001101BA000200E00006
:1004D000E8FF3A00000006003159BA008301E90044
:1004E0000C0032002159BA008301E90008003200F3
:1004F0000400E00003003A00E280400032A0B400B3
:10050000F5FF370011D9BA008301E900FAFF3A007C
:100510008100E800E180400032A0B4000000060045
:10052000889FBE008A9FBE00010578000100E000A0
:100530000400350008003C000000E000200032000C
:100540000500370060001000E080180002003B004A
:1005500001F02C001A0037000004BE006011B80042
:100560006B0920000982CF00020039000882CF0009
:100570000441B000694252000E00320008003B0006
:1005800082817100610164008904D1000884D30074
:100590008B05E8000442E800F9FF3A000500370047
:1005A0000804440089844C008B05E9000442E900FA
:1005B000FBFF3A00250107000AF0A70001F0A000A8
:1005C0004F05BE004F04BE000000060003F0A2006D
:1005D000889FBE008A9FBE008C1F780041010700E3
:1005E000480133006450E1004F0032006420E10014
:1005F0005200320003826C0007003B000905D00066
:100600000306D000820F54000C065D000200390082
:1006100002003200890178000306780085825500C7
:1006200004003D000003FD008103FD008502EA0097
:100630008B854200840F720002003B0060001000B6
:10064000E08018006011B8000005EB007A28E10096
:100650000A00390006007800C75DDD00F707B20028
:10066000878075002D003700828171000A017800B3
:10067000610560008180D1000080D3008502E9001F
:10068000F9FF3B00060440008784480002003B005D
:1006900060041400E0841C000988A30007003200F5
:1006A0008A81710082817100610164008904D10036
:1006B0000884D3008B05E800170037000978A300F1
:1006C00013003A000B00E000130034008B05E90032
:1006D0000804440089844C000A4474000978A3008B
:1006E0000D003A000B00E000070034008B05E90024
:1006F0000804440089844C0001003A000B002000EB
:100700000978A300F7FF32000001EB000200370078
:10071000828171000A017800CC0007000CF0A7006C
:1007200001F0A000000137006420E10002003A005F
:10073000838F6C00000133000801BE000200BE0080
:10074000F9003700889FBE008A9FBE008C1F78008A
:10075000E4000700EB00330003866C006450E10006
:100760002E0032006420E100330032006150E100CD
:100770002F0032006120E1003100320085855500F4
:10078000EB07B00009002000080420000500370036
:100790000804440089844C000A0031000603430029
:1007A00087834B000001530081815B00F8FF330019
:1007B0000203BE000800A0000804440089844C0025
:1007C000F6FF3900C639DD008301730001003200F5
:1007D000130020008904D1000884D3000998A300E5
:1007E000050032000800A7000300A0008904D10022
:1007F0000884D3008B05E8008904D1000884D30065
:100800000001EB000281D2009000070001F0A1007E
:100810000CF0A70001F0A000C30037006420E10045
:10082000C50032000801BE000200BE00F7FF37001D
:100830006120E100C00032006000B800F3FF370023
:100840000000200001F82700F0FF3700889FBE005D
:100850008A9FBE008C1F7800A2000700A900330009
:1008600003866C006450E100240032006420E10043
:10087000270032006150E100220032006120E100D7
:10088000210032008B854200EB07B1000134B80033
:10089000003AB8000804420089844A00013AB800CE
:1008A0000030B8008880400009014A00040033008D
:1008B0000000400081804800020149008B05E900EA
:1008C000C909DD008301700001003200130020001F
:1008D000C814DE004814DD004709DE001200B20033
:1008E000C808DE00088470005800070001F0A1006D
:1008F0000CF0A70001F0A0008B0037006120E100A0
:100900008D0032000801BE000200BE00F7FF370074
:100910006150E100FCFF3A00870037000001BE0093
:10092000880007000470A70003F0A10003F8A300EB
:1009300013003A006509B1001000320009003500CB
:100940006928E100020035000100280000000500D0
:1009500000004000818048008502E900FCFF3A0069
:1009600000000600F88F4200050035008100D1002C
:100970000080D3008502E800FCFF3A00000006007A
:100980008000EB00000005006022B8000602200095
:100990000000D0008180D2000482D2008582D20083
:1009A0000000A0000202520083825A0003003100BE
:1009B0000202420083824A000000A1000603E9000F
:1009C000F3FF3A00000006000001BE005D000700D2
:1009D0000470A70003F0A1006509B1001600320001
:1009E0000D0035006828E10006003500F0FF2F00FB
:1009F000F1FF27000300E00013003B000100280086
:100A00000000050000004000818048008502E900E8
:100A1000FCFF3A0008003700F88F420002003C005B
:100A20008000EB00000005008100D1000080D300B1
:100A30008502E800FCFF3A000300E00002003B00F2
:100A400060001000E0801800000006008100200017
:100A5000618055000B003D000B00200061FE2F005F
:100A60000100E1001D003400828171006101640019
:100A70008904D1000884D3000000E800FAFF3A009E
:100A8000710020006100640003007000020060003B
:100A90000900320061044400E0844C000988A5008C
:100AA000050032008B05E8006808E10002003A000A
:100AB0008904D1000884D300F20F20000258E1001D
:100AC00005003D00C75DDD00F907B20089807500B3
:100AD00008007800000006000BF827008B00780063
:100AE000000005000004BE00160007000003BE0061
:100AF0000405BE000200BE0012000700844F75000E
:100B0000000006000200BE006450E100050036004F
:100B10006420E100020036000968A30001003A00E9
:100B20000800BE000160A0004F0678004F05BE001F
:100B30004F04BE0000000600F0FF2F00F1FF270069
:100B4000F9FF3700C70ADE00F107B200F50FB20067
:100B500008003200E1CF4200020032000170A00024
:100B600024000500810F7000010032000408050018
:100B700044000500810F700002003A0014000500D7
:100B80008502E9000000400081C04800FCFF3B00F6
:100B90000170A000240005005245000041440000FF
:100BA000590D00000A0000005245000041440000B9
:100BB0003A2000000052000045410000442000009F
:100BC000002000004259000054450000533A000044
:100BD0000D0A000000570000524900005445000073
:100BE0003A20000000200000544900004D4500005C
:100BF00053000000414300004B0000004E41000044
:100C0000434B000000490000324300002053000025
:100C1000544100005254000020420000495400009A
:100C20000D0A00000049000032430000205300007C
:100C3000544F00005020000042490000540D0000B5
:100C40000A00000043530000204500004E41000010
:100C5000424C0000454400000D0A00000043000023
:100C6000532000004449000053410000424C000062
:100C7000454400000D0A00000054000068690000AF
:100C8000732000006D6F000064650000207200009A
:100C90006571000075690000726500007320000036
:100CA000616E00002061000064610000707400004B
:100CB000657200000D0A000000520000454100006E
:100CC0004420000042490000543A00002000000087
:100CD0004441000054410000204900004E500000F3
:100CE000555400002C2000005354000041540000D3
:100CF000453A000020000000202A00007069000032
:100D00006E20000069730000206E00006F77000005
:100D100020480000695A00000D0A00000020000071
:100D2000434C00004F4300004B200000544900009A
:100D3000434B0000530D00000A000000434C00002C
:100D40004F4300004B2C0000203100000D0A000032
:100D5000004300004C4F0000434B00002C200000DB
:100D6000300D00000A000000444100005441000022
:100D7000204F00005554000050550000542C000036
:100D8000203100000D0A0000004400004154000022
:100D9000412000004F550000545000005554000001
:100DA0002C200000300D00000A000000504F000011
:100DB00057450000522000005355000050500000DD
:100DC0004C49000045530000204F00004E0D00002C
:100DD0000A000000504F000057450000522000005C
:100DE00053550000505000004C490000455300008E
:100DF000204F0000464600000D0A0000005500008C
:100E00006E6B00006E6F0000776E0000206D0000BA
:100E100061630000726F00002C20000074720000FB
:100E2000792000003F2000006F72000020280000A1
:100E300030290000206600006F720000206800006A
:100E4000656C0000700D00000A000000436F000098
:100E50006D6D0000616E0000642000006E6F000088
:100E600074200000757300006564000020690000B4
:100E70006E2000007468000069730000206D00009F
:100E80006F640000650D00000A0000002A200000C9
:100E9000537900006E740000617800002065000046
:100EA000727200006F7200002C2000007479000044
:100EB00070650000203F0000206600006F72000097
:100EC00020680000656C0000700D00000A00000042
:100ED0002A20000054450000524D0000494E0000F9
:100EE000414C0000204200005546000046450000ED
:100EF000522000004F56000045520000464C0000B2
:100F00004F5700002C2000005452000059200000D0
:100F1000534D0000414C00004C45000052200000A1
:100F200053450000474D0000454E0000545300005B
:100F30000D0A0000004E00006F2000006D6F0000E1
:100F40006465000020730000657400002C20000020
:100F50004D200000666F0000722000006D6F0000E1
:100F6000646500000D0A00000057000041520000B7
:100F70004E4900004E4700003A2000007069000012
:100F80006E730000206E00006F740000206F000080
:100F9000706500006E20000064720000616900004E
:100FA0006E20000028480000695A0000290D00004A
:100FB0000A00000045720000726F0000722C0000F1
:100FC0002074000072790000206100006761000059
:100FD000696E0000203E000000530000656C0000B8
:100FE00065630000742000006F75000074700000DD
:100FF000757400002074000079700000653A0000EC
:101000000D0A0000203100002E2000004F7000006B
:10101000656E00002064000072610000696E0000CF
:1010200020280000483D0000486900002D5A0000BB
:101030002C2000004C3D0000474E000044290000D9
:101040000D0A0000203200002E2000004E6F00002C
:10105000726D0000616C000020280000483D000017
:10106000332E0000335600002C2000004C3D0000C1
:10107000474E0000442900000D0A0000004D00000A
:101080006F64000065200000736500006C6500005F
:1010900063740000656400000D0A00000020000079
:1010A000312E000020480000455800000D0A0000C5
:1010B000203200002E20000044450000430D0000B7
:1010C0000A200000332E000020420000494E00009C
:1010D0000D0A0000203400002E20000052410000C4
:1010E000570D00000A000000446900007370000002
:1010F0006C61000079200000666F0000726D0000D6
:101100006174000020730000657400000D0A000087
:1011100000200000312E000020500000756C0000FF
:101120006C2D000075700000732000006F660000D9
:10113000660D00000A200000322E00002050000042
:10114000756C00006C2D00007570000073200000AD
:101150006F6E00000D0A000000500000756C00006A
:101160006C2D000075700000207200006573000097
:1011700069730000746F000072730000204F00005C
:10118000464600000D0A000000500000756C00008B
:101190006C2D000075700000207200006573000067
:1011A00069730000746F000072730000204F00002C
:1011B0004E0D00000A000000566F00006C74000025
:1011C00061670000652000006D6F00006E6900001F
:1011D000746F0000727300003A20000000200000CD
:1011E000312E0000204D0000534200002066000018
:1011F00069720000737400000D0A000020320000C4
:101200002E2000004C5300004220000066690000C0
:1012100072730000740D00000A0000004D530000BE
:101220004220000073650000743A0000204D000069
:101230004F53000054200000736900006720000035
:10124000626900007420000066690000727300008B
:10125000740D00000A0000004C5300004220000002
:1012600073650000743A0000204C00004541000006
:1012700053540000207300006967000020620000E2
:101280006974000020660000697200007374000039
:101290000D0A0000004100005558000020630000C6
:1012A0006F6D00006D6100006E640000732000002F
:1012B000636F00006E740000726F00006C0D000020
:1012C0000A200000312E0000204100005558000087
:1012D000202800006465000066610000756C000055
:1012E000742900000D0A0000203200002E200000AA
:1012F000435300002F5400004D5300000D0A00001E
:10130000006100002F4100002F400000206300001A
:101310006F6E0000747200006F6C0000732000009C
:101320004155000058200000706900006E0D00005B
:101330000A000000612F0000412F00004020000043
:10134000636F00006E740000726F00006C73000029
:1013500020430000532F0000544D00005320000094
:10136000706900006E0D00000A000000416400007A
:101370006A75000073740000207900006F7500002A
:101380007220000074650000726D0000696E00003C
:10139000616C0000206100006E640000207000009D
:1013A000726500007373000020730000706100001C
:1013B00063650000207400006F200000636F000070
:1013C0006E740000696E0000756500000D0A000073
:1013D0000053000065740000207300006572000077
:1013E000696100006C200000706F000072740000E2
:1013F0002073000070650000656400003A20000062
:101400002862000070730000290D00000A2000000F
:10141000312E000020330000303000000D0A0000A3
:10142000203200002E200000313200003030000059
:101430000D0A0000203300002E200000323400008E
:10144000303000000D0A0000203400002E20000083
:1014500034380000303000000D0A00002035000054
:101460002E20000039360000303000000D0A000048
:10147000203600002E2000003139000032300000FC
:10148000300D00000A200000372E0000203300003D
:1014900038340000303000000D0A00002038000011
:1014A0002E2000003537000036300000300D0000DF
:1014B0000A200000392E00002031000031350000E4
:1014C00032300000300D00000A000000436C0000C4
:1014D0006F6300006B200000706F00006C61000003
:1014E00072690000747900003A0D00000A200000C3
:1014F000312E000020490000646C000065200000CF
:101500006C6F0000772000002A6400006566000010
:10151000617500006C7400000D0A000020320000AC
:101520002E200000496400006C6500002068000067
:1015300069670000680D00000A0000004F75000098
:101540007470000075740000206300006C6F000070
:10155000636B00002065000064670000653A0000CE
:101560000D0A0000203100002E2000004964000018
:101570006C650000207400006F20000061630000B3
:1015800074690000766500000D0A0000203200003A
:101590002E200000416300007469000076650000A1
:1015A000207400006F200000696400006C6500007A
:1015B000202A00006465000066610000756C000070
:1015C000740D00000A000000496E000070750000F4
:1015D00074200000736100006D7000006C650000F5
:1015E0002070000068610000736500003A0D000083
:1015F0000A200000312E0000204D00006964000028
:10160000646C0000652000002A640000656600002C
:10161000617500006C7400000D0A000020320000AB
:101620002E200000456E0000640D00000A0000003E
:1016300053650000742000007370000065650000B1
:10164000643A00000D0A0000203100002E20000046
:101650007E3500004B4800007A0D00000A20000093
:10166000322E0000207E0000353000004B48000084
:101670007A0D00000A200000332E0000207E0000BA
:1016800031300000304B0000487A00000D0A0000A5
:10169000203400002E2000007E3400003030000096
:1016A0004B4800007A0D00000A0000004F70000057
:1016B000656E00002064000072610000696E000029
:1016C000206F0000757400007075000074730000D6
:1016D00020280000483D0000486900002D5A000005
:1016E0002C2000004C3D0000474E00004429000023
:1016F0000D0A0000004E00006F7200006D610000D6
:101700006C2000006F75000074700000757400009C
:1017100073200000284800003D5600002B2C0000DC
:10172000204C00003D4700004E440000290D000001
:101730000A000000507500006C6C00002D75000060
:10174000702000007265000073690000737400006F
:101750006F720000732000006E6F000074200000A4
:10176000616C00006C6F000077650000640D000084
:101770000A00000042690000746F000072640000FB
:1017800065720000206300006F6E00006669000053
:101790006775000072610000746900006F6E0000E0
:1017A000206E00006F740000206100006C6C00006F
:1017B0006F770000656400000D0A0000004D000016
:1017C000454E000055530000003F00002048000037
:1017D000656C000070000000492000005374000098
:1017E0006174000075730000206900006E660000DF
:1017F0006F0000004D2000004275000073200000C3
:101800006D6F00006465000000420000205400007D
:10181000657200006D6900006E6100006C200000C0
:101820007370000065650000640000004F20000038
:1018300044610000746100002064000069730000CE
:10184000706C000061790000206600006F7200007B
:101850006D61000074000000562000004368000025
:10186000656300006B20000073750000707000005D
:101870006C790000207600006F6C0000746100003D
:1018800067650000730000004620000046720000FB
:1018900065710000756500006E630000792000002E
:1018A000636F0000756E0000742000006F6E000012
:1018B000204100005558000000470000204600006D
:1018C0007265000071750000656E000063790000AC
:1018D00020670000656E0000657200006174000002
:1018E0006F7200002F500000574D0000206F000065
:1018F0006E20000041550000580000004320000009
:101900004155000058200000706900006E20000062
:101910006173000073690000676E00006D65000070
:101920006E740000004C000020420000697400004A
:10193000206F00007264000065720000005000001B
:1019400020500000756C00006C75000070200000D5
:101950007265000073690000737400006F7200000C
:10196000730000003D20000048450000582F000093
:1019700044450000432F0000424900004E20000073
:10198000636F00006E7600006572000074650000F1
:10199000720000007E200000536500006C660000AD
:1019A0002074000065730000740000002320000014
:1019B00052650000736500007400000024200000E0
:1019C000426F00006F7400006C6F000061640000E3
:1019D0006572000000530000594E000054410000A1
:1019E00058000000412F0000612F0000402000003F
:1019F00041550000582000006F7500007470000011
:101A000075740000207400006F670000676C0000B0
:101A100065200000482F00004C2F00007265000078
:101A200061640000005700002F7700002050000084
:101A30006F77000065720000207300007570000071
:101A4000706C000079200000746F00006767000070
:101A50006C650000206F00006E2F00006F660000B4
:101A600066000000642000002844000029200000D7
:101A70004D65000061730000757200006520000074
:101A8000766F00006C740000616700006520000044
:101A90006F6E0000204100004443000020700000F1
:101AA000726F00006265000020280000636F000074
:101AB0006E740000696E0000756F000075730000A1
:101AC000290000005B200000287B00002920000086
:101AD0005374000061720000742000002877000039
:101AE00069740000682000007265000061640000F5
:101AF000290000005D2000006F720000207D0000C2
:101B000020530000746F000070000000522000009D
:101B10006F7200002072000020520000656100001A
:101B2000642000006279000074650000003000004D
:101B300062200000577200006974000065200000F8
:101B4000424900004E2000006279000074650000E8
:101B500000300000682000006F720000203000009C
:101B600078200000577200006974000065200000B2
:101B700048450000582000006279000074650000AC
:101B8000003000002D3200003535000020570000E5
:101B900072690000746500002044000045430000A5
:101BA0002062000079740000650000002C20000015
:101BB000446500006C6900006D69000074650000F8
:101BC00072200000286100006C7300006F2000008C
:101BD00073700000616300006529000000260000AA
:101BE000203100007553000020640000656C000087
:101BF00061790000003A000020520000657000008A
:101C00006561000074200000287200003A32000074
:101C10002C20000030780000306100003A340000D1
:101C20002C200000263A0000323000002C2000005A
:101C30005E3A0000322C0000206500007463000052
:101C40002E29000000280000232900002052000057
:101C5000756E0000206D000061630000726F00006F
:101C60002C2000002830000029200000666F0000B2
:101C7000722000006D610000637200006F200000A0
:101C80006C690000737400000052000041570000AE
:101C90002042000055530000204F00005045000036
:101CA00052410000544900004F4E00005300000014
:101CB0002F5C0000204300006C6F0000636B00008D
:101CC000204800002F4C0000002D00002F5F000076
:101CD000204400006174000061200000482F0000D3
:101CE0004C0000002E2000005265000061640000DE
:101CF000206400006174000061200000696E000033
:101D00007075000074200000706900006E200000F3
:101D10007374000061740000650000005E20000024
:101D2000436C00006F6300006B20000074690000CA
:101D3000636B00000021000020520000656100007C
:101D400064200000626900007400000000000000D0
:101D5000002000002C20000000200000575200004E
:101D6000495400004520000042490000542800006A
:101D7000532900002028000000290000005700001F
:101D80005249000054450000204200004954000020
:101D90003A200000002000002A6E00006578000054
:101DA00074200000636C00006F6300006B20000073
:101DB000285E000029200000776900006C6C00009C
:101DC000206100006C7300006F200000686100005B
:101DD0007665000020740000686900007320000030
:101DE000766100006C75000065000000315700004E
:101DF0004952000045200000726F00007574000019
:101E0000696E000065730000204300006F700000E1
:101E100079720000696700006874000020280000E3
:101E20004329000020320000303000003020000044
:101E30004D69000063680000616500006C200000CF
:101E400050650000617200006365000000520000F0
:101E5000656C00006561000073650000642000008F
:101E6000756E00006465000072200000474E00009F
:101E700055200000476500006E650000726100009B
:101E80006C20000050750000626C00006963000067
:101E9000204C000069630000656E0000736500005F
:101EA000004E00006F2000006465000076690000AD
:101EB000636500002C20000074720000792000008F
:101EC000284100004C410000524D00002920000034
:101ED000534500004152000043480000206D0000BF
:101EE00061630000726F00002066000069720000EC
:101EF000737400000041000044440000524500009B
:101F000053530000204D000041430000524F000099
:101F1000200000003A200000002000000020000007
:101F2000302E00004D610000637200006F20000041
:101F30006D6500006E750000004D000061630000DB
:101F4000726F0000202000002020000020310000DF
:101F50005749000052450000206100006464000001
:101F60007265000073730000002E0000000D000079
:101F70000A200000202000002A0000003157000045
:101F80004952000045200000524F00004D20000043
:101F9000434F00004D4D0000414E00004420000022
:101FA0004D410000435200004F7300003A0D000005
:101FB0000A200000353100002E520000454100008B
:101FC00044200000524F00004D2000002830000047
:101FD0007833000033290000202A0000666F0000DB
:101FE00072200000736900006E6700006C650000DD
:101FF0002064000065760000696300006520000031
:1020000062750000730D00000A20000038350000E2
:102010002E4D0000415400004348000020520000B3
:102020004F4D0000202800003078000035350000BA
:10203000292000002A6600006F6C00006C6F000011
:1020400077650000642000006279000020360000FF
:1020500034620000697400002061000064640000C4
:1020600072650000737300000D0A0000203200004A
:10207000303400002E5300004B4900005020000077
:10208000524F00004D20000028300000784300002F
:1020900043290000202A0000666F00006C6C0000DD
:1020A0006F77000065640000206200007920000066
:1020B000636F00006D6D0000616E0000640D000034
:1020C0000A20000032330000362E0000414C000090
:1020D000415200004D2000005345000041520000D5
:1020E00043480000202800003078000045430000ED
:1020F000290D00000A20000032340000302E0000BC
:1021000053450000415200004348000020520000A7
:102110004F4D0000202800003078000046300000BD
:1021200029000000414C0000415200004D200000F9
:1021300053450000415200004348000020280000A1
:10214000307800004543000029000000534500009E
:102150004152000043480000202800003078000071
:102160004630000029000000446500007669000048
:1021700063650000204900004473000020610000F6
:10218000726500002061000076610000696C00004B
:10219000616200006C650000206200007920000090
:1021A0004D410000435200004F2C000020730000FE
:1021B0006565000020280000302900002E00000086
:1021C0005245000041440000205200004F4D0000E5
:1021D000202800003078000033330000293A000046
:1021E000200000004D410000544300004820000042
:1021F000524F00004D2000002830000078350000CC
:1022000035290000005300004B4900005020000019
:10221000524F00004D20000028300000784300009D
:1022200043290000004200005553000020520000E6
:102230004553000045540000200000004F4B0000B3
:1022400000450000525200004F5200003A200000AA
:10225000002A0000536800006F7200007420000024
:102260006F720000206E00006F200000707500008B
:102270006C6C00002D75000070200000002A00002A
:102280004E6F000020640000657600006963000066
:102290006520000064650000746500006374000040
:1022A0006564000020000000280000004453000086
:1022B000313800005332000030200000486900002F
:1022C0006768000020500000726500007320000065
:1022D0004469000067200000546800006572000037
:1022E0006D0000004453000031380000423200000D
:1022F00030200000507200006F6700002052000084
:10230000657300002044000069670000205400004D
:1023100068650000726D0000004400005331000049
:102320003832000032200000456300006F6E00006C
:102330002044000069670000205400006865000028
:10234000726D000000440000533200003430000081
:1023500034200000456300006F6E000072610000D1
:102360006D200000746900006D65000020430000CE
:10237000686900007000000044530000323400001F
:1023800033310000203100004B20000045450000A3
:10239000505200004F4D0000005500006E6B0000D1
:1023A0006E6F0000776E000020640000657600000C
:1023B0006963000065000000315700003031000003
:1023C000000000004A54000041470000534D000047
:1023D0003A2000005244000059200000544F0000F1
:1023E00020570000524900005445000020490000D9
:1023F0004E53000054520000554300005449000061
:102400004F4E000020520000454700004953000095
:1024100054450000520000004A54000041470000AB
:10242000534D00003A2000005244000059200000A3
:10243000544F00002052000045410000442F00008E
:10244000575200004954000045200000444100005C
:10245000544100002052000045470000495300004D
:1024600054450000520000004A540000414700005B
:10247000534D00003A200000494400004C45000044
:1024800000000000202C0000200000002030000090
:102490002E4D000061630000726F0000206D00008F
:1024A000656E0000750D00000A200000312E00004E
:1024B000526500007365000074200000636800002E
:1024C000616900006E0D00000A200000322E00003D
:1024D000507200006F620000652000006368000019
:1024E000616900006E0D00000A200000332E00001C
:1024F0005853000046560000207000006C61000038
:1025000079650000722000002864000065700000FA
:1025100072650000636100007465000064290000BA
:102520000D0A0000004A000054410000475300001B
:102530004D3A000020520000455300004554000071
:10254000004A00005441000047200000494E0000AE
:10255000495400002043000048410000494E00005B
:10256000002000004445000056490000434500009B
:102570002853000029200000494E0000204A000096
:10258000544100004720000043480000414900003A
:102590004E000000203A00002000000058530000C8
:1025A00046560000207000006C6100007965000054
:1025B0007220000077610000732000007265000047
:1025C0006D6F00007665000064200000696E0000F9
:1025D00020760000322E0000312C0000206900001F
:1025E00066200000796F0000752000006E65000015
:1025F000656400002069000074200000646F000022
:10260000776E0000677200006164000065200000C2
:10261000746F000020760000322E0000302E000083
:102620000049000074270000732000006875000056
:10263000676500002C200000756700006C790000C1
:102640002C200000616E000064200000746800000F
:102650006520000058530000465600002066000028
:102660006F7200006D61000074200000697300004B
:10267000207300007065000063690000616C000059
:10268000697A0000656400002E00000057650000B4
:10269000276C00006C2000006164000064200000D2
:1026A0006120000072650000616C00002053000092
:1026B00046560000207000006C6100007965000043
:1026C00072200000696E0000207400006865000040
:1026D000206600007574000075720000652E000011
:1026E000004A000054410000475300004D3A0000EA
:1026F00020000000414C0000524500004144000011
:1027000059200000494400004C45000000520000E0
:1027100045530000455400002D3E00004944000090
:102720004C45000000280000575200004F540000A4
:1027300045200000444500004C4100005945000080
:1027400044200000424900005429000020000000FD
:10275000495200002D3E0000494400004C45000055
:1027600000440000522D00003E490000444C00008F
:1027700045000000554E00004B4E00004F57000032
:102780004E2000005354000041540000450000005A
:102790004A54000041470000534D00003A20000019
:1027A00057410000524E0000494E000047200000F3
:1027B0004F550000542000004F46000020530000F9
:1027C000594E0000430000005245000053450000F0
:1027D00054000000494400004C4500002D3E00001C
:1027E0004461000074610000205200006567000031
:1027F0006973000074650000720000004944000025
:102800004C4500002D3E0000496E0000737400002E
:102810007275000063740000696F00006E20000094
:102820005265000067690000737400006572000063
:1028300020280000444500004C410000594500009C
:10284000442000004F4E0000452000004249000097
:1028500054200000464F000052200000544D00005C
:1028600053290000005500004E4B00004E20000090
:102870005354000041540000452C00002054000037
:1028800052590000205200004553000045540000FA
:102890002028000031290000004E00004F540000A5
:1028A000453A000020570000524F000054450000F8
:1028B00020440000454C0000415900004544000000
:1028C000204200004954000000000000002D0000DC
:1028D00070200000002D000066200000002A00008B
:1028E00042790000746500007320000064720000EB
:1028F0006F70000070650000642A00000046000050
:10290000414900004C450000442C0000204E0000CE
:102910004F2000004441000054410000002000000E
:102920002C200000005500004152000054200000FF
:102930004C49000056450000204400004953000067
:10294000504C0000415900002C2000007D20000068
:10295000544F000020530000544F0000500000006E
:102960004C49000056450000204400004953000037
:10297000504C00004159000020530000544F00000B
:10298000505000004544000000200000313000009D
:102990002E200000333100003235000030200000CE
:1029A000284D00004944000049290000004400006F
:1029B000617400006120000062690000747300000F
:1029C000206100006E640000207000006172000051
:1029D00069740000793A00000D0A000020310000FF
:1029E0002E200000382C0000204E00004F4E00002A
:1029F000452000002A640000656600006175000043
:102A00006C740000200D00000A200000322E00002F
:102A1000203800002C20000045560000454E0000E4
:102A2000200D00000A200000332E00002038000096
:102A30002C2000004F440000442000000D0A00003C
:102A4000203400002E200000392C0000204E000011
:102A50004F4E000045000000537400006F700000EE
:102A60002062000069740000733A00000D0A000043
:102A7000203100002E200000312000002A640000D8
:102A800065660000617500006C7400000D0A0000AE
:102A9000203200002E2000003200000052650000AD
:102AA000636500006976000065200000706F00001B
:102AB0006C61000072690000747900003A0D00003A
:102AC0000A200000312E000020490000646C000044
:102AD00065200000312000002A64000065660000C7
:102AE000617500006C7400000D0A000020320000C7
:102AF0002E200000496400006C65000020300000BA
:102B000000200000302E00004D61000063720000C4
:102B10006F2000006D6500006E7500000D0A00005A
:102B2000203100002E540000726100006E7300001E
:102B300070610000726500006E7400002055000096
:102B400041520000542000006272000069640000DD
:102B5000676500000D0A0000203200002E200000F2
:102B60004C690000766500002055000041520000CD
:102B7000542000006D6F00006E690000746F00004B
:102B8000720D00000A200000332E000055410000A5
:102B90005254000020620000726900006467000067
:102BA000652000007769000074680000206600005E
:102BB0006C6F000077200000636F00006E740000EF
:102BC000726F00006C00000055410000525400007C
:102BD000206200007269000064670000652E00003A
:102BE0002053000070610000636500002063000056
:102BF0006F6E0000746900006E7500006573000060
:102C00002C200000616E00007974000068690000EB
:102C10006E670000206500006C73000065200000F6
:102C20006578000069740000732E000000520000F7
:102C30006573000065740000207400006F200000C0
:102C400065780000697400002E00000052610000E9
:102C50007720000055410000525400002069000018
:102C60006E700000757400002E200000537000008C
:102C70006163000065200000746F000020650000A3
:102C800078690000742E00000041000052540000DA
:102C900031000000004300004D440000200000000F
:102CA0004441000054200000002000002C200000BF
:102CB00000520000532000004C4F0000572C000031
:102CC000204300004F4D00004D4100004E440000E5
:102CD000204D00004F44000045000000525300000A
:102CE0002048000049470000482C00002044000014
:102CF00041540000412000004D4F000044450000B9
:102D0000004C000043440000207400007970000073
:102D1000653A00000D0A0000203100002E2000005E
:102D200048440000343400003738000030200000F0
:102D300028750000736900006E67000020500000D5
:102D400043460000383500003734000020490000B9
:102D50004F20000065780000706100006E64000084
:102D60006572000029000000203000002E4D000098
:102D700061630000726F0000206D0000656E00004E
:102D8000750D00000A200000312E00004C430000A9
:102D9000442000005265000073650000740D0000BF
:102DA0000A200000322E0000496E00006974000005
:102DB000204C0000434400000D0A000020330000B6
:102DC0002E4300006C65000061720000204C000082
:102DD000434400000D0A0000203400002E43000090
:102DE00075720000736F000072200000706F0000A9
:102DF00073690000746900006F6E000020650000B8
:102E0000783A0000283400003A300000290D000014
:102E10000A200000352E00002864000065700000C4
:102E200072650000636100007465000064290000A1
:102E30000D0A0000203600002E57000072690000C5
:102E400074650000203A00006E7500006D6200009D
:102E5000657200002074000065730000742000009B
:102E60006E7500006D620000657200007320000046
:102E7000657800003A280000363A0000383000003B
:102E8000290D00000A200000372E000057720000B4
:102E900069740000652000003A6E0000756D000046
:102EA0006265000072200000746500007374000009
:102EB000206300006861000072610000637400001C
:102EC0006572000073200000657800003A28000059
:102ED000373A000038300000290D00000A200000B9
:102EE000382E0000496E0000736500007274000007
:102EF00020740000657800007420000061740000F8
:102F00002063000075720000736F00007200000003
:102F10005245000053450000540000004469000081
:102F2000737000006C610000792000006C69000083
:102F30006E650000733A00000D0A000020310000A9
:102F40002E200000312000000D0A00002032000079
:102F50002E2000004D7500006C74000069700000A8
:102F60006C650000004900004E490000540000005C
:102F7000434C000045410000524500004400000061
:102F800043550000525300004F52000020530000F0
:102F900045540000004900006E7300006572000097
:102FA0007420000074650000787400003A0000008E
:102FB0004E6F000020410000434B00002C20000019
:102FC00063680000656300006B200000616400001E
:102FD00061700000746500007200000000200000B5
:102FE0002C200000002800005C2D00002F5F000056
:102FF0005C290000002800005F2F00002D5C00000D
:1030000029000000203000002E4D00006163000008
:10301000726F0000206D0000656E0000750D0000ED
:103020000A200000312E0000495300004F370000F5
:1030300038310000362D00003320000041540000DC
:10304000520D00000A200000322E000049530000FB
:103050004F37000038310000362D000033200000CB
:103060007061000072730000652000006F6E000048
:103070006C7900000D0A000000490000534F000069
:103080002037000038310000362D000033200000CA
:103090004154000052200000285200004553000017
:1030A00045540000206F00006E20000043530000D4
:1030B0002900000052450000534500005420000044
:1030C00048490000474800002C200000434C000005
:1030D0004F4300004B20000054490000434B0000C8
:1030E0002C200000524500005345000054200000F1
:1030F0004C4F000057000000495300004F200000D3
:1031000037380000313600002D33000020720000F7
:10311000657000006C7900002028000075730000C5
:103120006573000020630000757200007265000086
:103130006E740000204C0000534200002073000019
:1031400065740000746900006E670000293A000091
:1031500020000000507200006F7400006F630000D8
:103160006F6C00003A2000000073000065720000E0
:10317000696100006C0000003320000077690000E6
:1031800072650000003200002077000069720000C4
:10319000650000005246000055000000756E0000FA
:1031A0006B6E00006F7700006E000000526500003B
:1031B000616400002074000079700000653A00002E
:1031C00020000000746F0000206500006E640000A5
:1031D000007600006172000069610000626C00000E
:1031E000652000006C6500006E67000074680000D8
:1031F000004400006174000061200000756E000052
:1032000069740000733A0000200000006E6F000037
:10321000206900006E6400006963000061740000B2
:10322000696F00006E0000004461000074610000DE
:10323000207500006E690000742000006C650000BD
:103240006E670000746800002028000062690000BA
:1032500074730000293A000020000000002A0000DA
:10326000284E000029410000434B00002050000080
:10327000454E0000444900004E4700000020000079
:103280002C20000000570000415200004E49000071
:103290004E4700003A200000484100005244000020
:1032A0005741000052450000204900003243000011
:1032B0002069000073200000627200006F6B000044
:1032C000656E0000206F00006E2000007468000032
:1032D00069730000205000004943000021200000D5
:1032E000285200004556000020410000332900000C
:1032F000005300006574000020730000706500003A
:10330000656400003A0D00000A200000312E000024
:1033100020310000303000004B4800007A0D0000E2
:103320000A200000322E000020340000303000005F
:103330004B4800007A0D00000A200000332E0000E8
:10334000203100004D4800007A00000020300000CD
:103350002E4D000061630000726F0000206D0000C0
:10336000656E0000750D00000A200000312E00007F
:10337000376200006974000020610000646400008E
:103380007265000073730000207300006561000027
:1033900072630000680D00000A200000322E000059
:1033A0004932000043200000736E0000696600008F
:1033B0006665000072000000536500006172000045
:1033C00063680000696E000067200000376200003B
:1033D00069740000204900003243000020610000B1
:1033E00064640000726500007373000020730000C5
:1033F00070610000636500002E2000000D0A0000CF
:1034000020200000204600006F7500006E64000060
:1034100020640000657600006963000065730000A9
:1034200020610000743A00000020000057000000F6
:103430002052000000290000004900003243000033
:103440002062000075730000207300006E690000A8
:1034500066660000657200002C200000707200009B
:103460006573000073200000616E00007920000089
:103470006B65000079200000746F0000206500007B
:1034800078690000740000004932000043310000F8
:1034900000000000524500005345000054000000A9
:1034A000424F00004F5400004C4F000041440000C8
:1034B0004552000000530000656C0000662D0000BE
:1034C0007465000073740000206900006E20000025
:1034D000486900005A2000006D6F0000646500001C
:1034E000206F00006E6C0000792E00000043000089
:1034F0004F4E0000564500005254000020000000CE
:103500000042000075730000205000006972000046
:103510006174000065200000763300000046000062
:10352000697200006D770000617200006520000084
:10353000763400002E35000000200000426F0000AD
:103540006F7400006C6F0000616400006572000021
:103550002076000000440000455600004944000069
:103560003A00000020520000455600004944000087
:103570003A00000020280000004100003300000055
:10358000423400000042000035000000554E0000AB
:103590004B000000290000006874000074700000F7
:1035A0003A2F00002F640000616E00006765000084
:1035B000726F000075730000707200006F7400007D
:1035C0006F74000079700000657300002E630000C6
:1035D0006F6D0000002A00002D2D00002D2D000031
:1035E0002D2D00002D2D00002D2D00002A000000A3
:1035F000506900006E3A0000534F00007C43000009
:103600004B7C0000534900007C430000537C0000C9
:10361000415500005800000044690000723A000063
:10362000004900006E7000003A000000696E000062
:103630007C0000006F7400007C00000068690000DE
:103640007C0000006C6F00007C0000002E20000059
:1036500000350000563A000020000000207C0000E9
:10366000203300002E330000563A000020000000F6
:10367000207C000020560000505500004C4C0000FB
:10368000555000003A200000002000007C0000009F
:1036900043460000473100003A000000204300008C
:1036A00046470000323A0000000000004469000074
:1036B000736300006F6E00006E65000063740000AD
:1036C000206100006E790000206400006576000033
:1036D0006963000065730000004300006F6E000026
:1036E0006E65000063740000202800005670000022
:1036F00075200000746F0000202B0000355600007C
:1037000029200000616E00006420000028410000B4
:1037100044430000207400006F2000002B330000A1
:103720002E33000056290000005000007265000092
:103730007373000020610000206B000065790000B9
:10374000207400006F20000073740000617200009C
:103750007400000043740000726C0000004100001F
:1037600055580000004D00004F4400004520000067
:103770004C45000044000000505500004C4C000037
:10378000555000002048000000500000554C00003B
:103790004C550000502000004C0000005652000024
:1037A0004547000000410000444300002061000044
:1037B0006E6400002073000075700000706C0000E3
:1037C00079000000355600000056000050550000FA
:1037D000003300002E33000056000000414400007A
:1037E000430000004275000073200000686900007B
:1037F0006768000000420000757300002048000068
:10380000692D00005A2000003000000042750000C1
:1038100073200000486900002D5A0000203100008C
:10382000004D00004F44000045200000616E000084
:10383000642000005652000045470000204C000064
:103840004544000073200000736800006F7500009D
:103850006C64000020620000652000006F6E0000B4
:1038600021200000416E0000792000006B650000FF
:10387000792000006578000069740000732E000054
:103880000028000000290000004D00004F530000F8
:1038900049000000434C00004B0000004D4900006F
:1038A000534F00000043000053000000204F000071
:1038B0004B00000020460000414900004C00000081
:1038C000505700004D200000646900007361000043
:1038D000626C000065640000003100004B4800008D
:1038E0007A2D0000342C000030300000304B0000F6
:1038F000487A0000206600007265000071750000C3
:10390000656E00006379000020670000656E0000AE
:1039100065720000617400006F7200002F5000009B
:10392000574D00002028000062650000746100000F
:1039300029000000467200006571000075650000F6
:103940006E63000079200000696E0000204B0000CB
:10395000487A0000200000005072000065730000EB
:10396000636100006C6500003A0000003235000021
:10397000360000003634000000380000003100003E
:1039800000500000523200003A00000000440000E5
:10399000757400007920000063790000636C0000FA
:1039A00065200000696E0000202500002000000056
:1039B000505700004D200000616300007469000052
:1039C0007665000000500000574D000020610000A7
:1039D0006374000069760000653A000020740000FE
:1039E0007279000020470000207400006F20000062
:1039F0006469000073610000626C000065200000D3
:103A0000505700004D000000467200006571000034
:103A1000756500006E630000792000006F6E000085
:103A2000204100005558000020700000696E000021
:103A30003A200000004800007A0000002028000022
:103A4000006B0000487A0000290000004D4800008B
:103A50007A2900000041000055580000204900006C
:103A60004E500000555400002F480000492D000022
:103A70005A0000004155000058200000484900004D
:103A8000474800000041000055580000204C00004D
:103A90004F57000000410000555800002049000029
:103AA0004E500000555400002F480000492D0000E2
:103AB0005A2C00002052000045410000443A00000A
:103AC00020000000005E0000BCE20000613F00003A
:103AD000DD830000C29C00007E200000A3FD0000EA
:103AE0001F4100009DC30000217F0000FCA20000D8
:103AF000401E00005F010000E3BD00003E600000CA
:103B000082DC0000237D00009FC10000421C0000F9
:103B1000FEA00000E1BF00005D03000080DE0000A9
:103B20003C620000BEE00000025C0000DF8100009B
:103B3000633D00007C220000C09E00001D43000089
:103B4000A1FF000046180000FAA400002779000039
:103B50009BC5000084DA000038660000E5BB000069
:103B600059070000DB85000067390000BAE4000057
:103B70000658000019470000A5FB00007826000049
:103B8000C49A0000653B0000D9870000045A000079
:103B9000B8E60000A7F900001B450000C698000029
:103BA0007A240000F8A60000441A000099C700001B
:103BB000257B00003A64000086D800005B05000009
:103BC000E7B900008CD20000306E0000EDB30000B9
:103BD000510F00004E100000F2AC00002F710000E9
:103BE00093CD0000114F0000ADF30000702E0000D7
:103BF000CC920000D38D00006F310000B2EC0000C9
:103C00000E500000AFF10000134D0000CE900000F8
:103C1000722C00006D330000D18F00000C520000A8
:103C2000B0EE0000326C00008ED00000530D00009A
:103C3000EFB10000F0AE00004C12000091CF000088
:103C40002D730000CA94000076280000ABF5000038
:103C50001749000008560000B4EA00006937000068
:103C6000D58B000057090000EBB500003668000056
:103C70008AD4000095CB000029770000F4AA000048
:103C800048160000E9B70000550B000088D6000078
:103C9000346A00002B75000097C900004A14000028
:103CA000F6A80000742A0000C8960000154B00001A
:103CB000A9F70000B6E800000A540000D789000008
:103CC0006B350000002000002C2000000053000095
:103CD00065740000207300007065000065640000DA
:103CE0003A0D00000A200000312E000020330000B1
:103CF000304B0000487A00000D0A0000203200001E
:103D00002E20000031320000354B0000487A0000C0
:103D10000D0A0000203300002E2000003235000084
:103D2000304B0000487A00000D0A000020340000EB
:103D30002E200000314D0000487A000000200000D5
:103D4000302E00004D610000637200006F20000003
:103D50006D6500006E7500000D0A00002031000046
:103D60002E530000504900002062000075730000CF
:103D7000207300006E690000666600006572000036
:103D8000005300006E6900006666000020770000A6
:103D9000686500006E3A00000D0A00002031000046
:103DA0002E20000043530000206C00006F770000BD
:103DB0000D0A0000203200002E20000043530000B6
:103DC0002068000069670000680D00000A200000FC
:103DD000332E0000204100006C6C000020740000B5
:103DE0007261000066660000696300000053000015
:103DF000504900002062000075730000207300002D
:103E00006E69000066660000657200002C200000EC
:103E1000616E0000792000006B65000079200000D1
:103E2000657800006973000074730000005300009F
:103E3000504900003100000000200000424900000D
:103E400054200000544900004D4500004F5500002B
:103E500054000000203000002E2000004D610000C2
:103E6000637200006F2000006D6500006E75000039
:103E70000D0A0000203100002E2000004C690000D7
:103E800076650000206900006E7000007574000007
:103E9000206D00006F6E0000697400006F720000FA
:103EA000004900006E70000075740000206D000075
:103EB0006F6E0000697400006F7200002C2000001B
:103EC000616E0000792000006B6500007920000021
:103ED000657800006974000073000000202A00006B
:103EE0007374000061720000746200006974000065
:103EF00020650000727200006F7200000020000058
:103F00002A700000617200006974000079200000CE
:103F100065720000726F000072000000202A00002D
:103F2000737400006F70000062690000742000006C
:103F300065720000726F000072000000204E0000E9
:103F40004F4E000045000000205500004E4B000081
:103F50004E4F0000574E0000204500005252000016
:103F60004F52000000000000486900005A000000A5
:103F7000312D000057490000524500000055000057
:103F8000415200005400000049320000430000008C
:103F900053500000490000004A540000414700000F
:103FA0000052000041570000325700004952000003
:103FB00045000000524100005733000057490000FF
:103FC0005245000000500000432000004B45000017
:103FD000594200004F41000052440000004C0000D4
:103FE0004344000000000000564F00004C54000005
:103FF0004D45000054450000522000004D4F000088
:10400000444500000050000072650000737300001A
:10401000206100006E790000206B000065790000CF
:10402000207400006F2000006578000069740000B3
:10403000005600004F4C000054410000474500006E
:1040400020500000524F0000424500003A2000007E
:1040500000560000000800000808000008080000E2
:1040600000000000444500004C41000059200000C1
:104070000075000053000000564F00004C54000033
:104080004147000045200000505200004F42000010
:10409000453A0000200000005600000029200000E2
:1040A00000000000306200000030000031320000EB
:1040B0003334000035360000373800003941000045
:1040C00042430000444500004630000078000000F4
:1040D000002000002C2000000000000042420000F0
:1040E000494F0000310000005241000057310000EC
:1040F00000000000314100004C53000000000000AF
:104100004F430000443100000000000000000000A8
:104110000600FA00881F78000CD8BF000080FB0062
:104120006101B9001207980023079800D001200010
:10413000010020001E019000AE019000800F510090
:10414000818F5900BE013E001E009000AE0090001D
:10415000006001001D0037003F0037005D003700A0
:104160005C003700B60137009C0037005B00370069
:10417000B301370062003700B1013700B0013700EA
:104180007400370073003700AD013700AC01370011
:10419000AB013700AA013700A9013700A801370099
:1041A000A7013700A6013700A5013700A401370099
:1041B000A3013700A2013700790037007C003700E7
:1041C000A10137009E0137009F01370080C08000A9
:1041D000E10F500007003A0010C0B300D82E0700CE
:1041E0003D2C070065FBB70065DBBF00092D07000C
:1041F0001600370020C0B300D12E070080C0800019
:10420000042D070030C0B300CD2E07000000EB00E6
:1042100010DB8800090037002F2C070065FBB70072
:1042200065DBBF00FB2C070000C2B300D40607000B
:1042300010DB80000000E80010DB880081C08000F7
:1042400010DB8000808F5000F3FF3E0080EA2800E2
:104250004C0507007C01370040C0B300B82E0700B2
:1042600070C08000EB2C070080C08000E10F500080
:1042700003003A0070C08000D62B07001200370000
:1042800090EA28002905070080C08000E12C070083
:1042900050C0B300AA2E07000000EB0010DB88001E
:1042A0000500370070C08000CA2B070010DB8000BB
:1042B0000000E80010DB880081C0800010DB800077
:1042C000808F5000F7FF3E0080EA28002D05070090
:1042D0005D0137005F0107005B013700292C0700F3
:1042E00065FBB700D0C0B300952E070065DBBF00AB
:1042F00007050700F0C0B300912E070052013700F8
:1043000080C08000C32C0700D0EA28000705070002
:104310000000EB0010DB88000500370058DBBF0011
:10432000D42B070010DB80000000E80010DB8800C1
:1043300081C0800010DB8000808F5000F7FF3E00BE
:1043400058DBBF00F2040700D0EB28000D05070082
:104350003D013700F0EB2800F40407000CD8BF0043
:10436000EC4F500005003A000040EB0058FBB7004E
:104370000040EB00E60407000400370010C0B30063
:1043800058FBB70010C0B300E1040700B0EC2800F0
:10439000FC04070058DBBF00B62B07002A013700DA
:1043A0000B58A9000B98A8000BD8A80026013700CD
:1043B0000040EB006AFBB700C922A800CB22A9008D
:1043C00060EF2800EF04070070F22800ED040700FA
:1043D0000040EB005A2E07001B01370070C0800020
:1043E0000000E0003600320071C080002003200091
:1043F000808F500032003E0070C080000000E90055
:1044000070C0880071C080006ADBBF000080FB00C4
:10441000808F50000300390010F52800D9040700F0
:1044200009013700B0F72800C004070070C0800001
:104430000040E8007D050700A0F82800BB04070045
:104440000040EB0064FBB7001700370072C080002B
:1044500064DBBF008080FB004310DD008100400072
:10446000B0B621000080400010407800692C0700A1
:1044700000C2B3004206070072C0800064DBBF00C8
:104480008080FB004310DD0081004000B0B62100B9
:1044900000804000104078004E2B070064DBBF0016
:1044A0000040E80064FBB70064DBBF00E74F50004A
:1044B000E6FF3600D0F82800B2040700E20037001B
:1044C00071C08000010F7800500520001E017800A7
:1044D000800F5100CB003200500520009E01780073
:1044E000808F510008003E001E0078000000E000B0
:1044F00012003200300320009E007800808F5000B0
:10450000A0003200CB003700C00E20001E01780052
:10451000800F510046003200000F20009E017800FD
:10452000808F510042003200C00C20009E007800B5
:10453000808F5000B9003200BE003700F0F828002C
:1045400090040700D0F928008E0407006ADBBF0042
:104550000004E00003003A0010F528008904070079
:10456000300037000040EB0065FBB7002800370043
:1045700000C2B3000206070065DBBF000040E80090
:104580002A05070050FB2800680407000040EB00E4
:1045900064FBB7000F00370065DBBF000081FB0044
:1045A00064DBBF008080FB004310DD008100400021
:1045B000B0B621000080400010407800152C0700A4
:1045C00000C2B300EE05070064DBBF000040E80056
:1045D00064FBB70064DBBF00E74F5000EEFF36001E
:1045E00070FB28005104070065DBBF000080FB0062
:1045F000C300DD00B0B6210000804000104078000C
:10460000B500070065DBBF000040E80065FBB700B0
:10461000A1B621009140780065DBBF0080CF50003B
:10462000D3FF3E00E0FB2800560407008600370059
:1046300070C08000A2F9B70071C08000C00E2000D9
:10464000808F500003003A00200929004D04070024
:1046500002003700600A29004A040700D0F9280048
:10466000480407000040EB0064FBB700C9000700E6
:1046700065FBB7000040EB006AFBB7003B0037006A
:1046800000C2B300BE05070064DBBF000040E800C5
:10469000E604070050FB2800240407000000EB009C
:1046A00010DB88000A00370011DB8000B0BB21005E
:1046B0000080400010407800D62B070000C2B300F5
:1046C000AF05070010DB80000000E80010DB880069
:1046D00010DB8000E70F5000F3FF360070FB28006E
:1046E00012040700BBDBBF007B00070064DBBF00D8
:1046F000E94F500018003E000000EB0010DB88007E
:104700000F0037006ADBBF008081FB0014DB8000F4
:1047100011DB8000B0BB2100008040001041780018
:104720004318DD0084004000B0B621000080400046
:104730000248780010DB80000000E80010DB8800F1
:1047400010DB8000E70F5000EEFF36006ADBBF0091
:104750000040E8006AFBB70064DBBF000040E800EF
:1047600064FBB7009600070065FBB70065DBBF0080
:104770000004E000C2FF3A00400B290001040700DA
:104780003100370033000700000E2900E70307005F
:1047900030C3B3008F2A07000000EB0010DB880055
:1047A0001000370018DB8000CB2A0700804078001B
:1047B00090B52100000044000148780011DB800022
:1047C00090B521000080400010407800912B070038
:1047D00000C2B3006A05070010DB80000000E8009B
:1047E00010DB880010DB8000E70F5000EDFF360083
:1047F00080EA2800E303070059DBBF00360007000A
:104800001100370013000700200F2900DD03070007
:1048100050C5B3006F2A07000B0037000D000700DA
:1048200030102900D7030700C0CCB300692A070065
:104830000500370070C1B300412D070002003700AA
:1048400080C1B3003E2D07004F0478000080FA00BD
:10485000000006000200FA00252A0700004F780039
:1048600030112900B10307001E04E00003003A00E4
:10487000E0112900C30307001500370010122900BA
:10488000AA0307001E80FB00610060000004E00036
:104890000200320090122900A40307001E80FB00D2
:1048A0000000D100610060000004E000020032005E
:1048B000F01329009D030700401529009B03070002
:1048C0001E407800532B0700D0EB2800AD030700F3
:1048D0000080FA00000006000400FA00004F780093
:1048E0001E80FB0010079800200220009E00900010
:1048F000808F50001A003200200220009E0090009D
:10490000808F500007003C001E009000E40F500014
:10491000160032009E009000F08F50000A00320016
:1049200018003700800220009E009000808F500009
:1049300008003200D00220009E009000808F5000BE
:104940000D0032000F003700601529008D030700AD
:104950000E003700201729008A0307000B003700DC
:10496000D01829008703070008003700301A2900F3
:104970008403070005003700C01B290081030700DE
:1049800002003700D01C29007E0307000080FA00D7
:10499000000006000000FA000040EB00C3FBB70077
:1049A0000040EB00C5FBB7000040EB00C4FBB700C4
:1049B000080007000080FB000080FA0000000600ED
:1049C0000000FA00030007000080FB000080FA00EE
:1049D000000006000A00FA0010C0B30070479800FB
:1049E0000040EB00604798000040EB005047980003
:1049F00010C0B300104798000040EB0040479800FB
:104A00000040EB00C6FBB700C5DBBF000004E000C0
:104A10008D003A00B62907000004E00009003200CA
:104A20000040EB00C3FBB7000040EB00C5FBB70044
:104A30000040EB00C4FBB7000000EB00400798000B
:104A400092003700A2D9BF00E22907004D2A0700D3
:104A5000304798004B2A0700204798003E409000BE
:104A6000E14F500003003A002E409000E14F50000B
:104A700065003200BE4090002E40900080CF500074
:104A8000030032003E409000004F780024003700C1
:104A900031BC2100914078007E409000814F500051
:104AA0000E0031005E4090008080FB00B0BB210012
:104AB00000804000904078001E40900080C0600060
:104AC0000040EB00004F78000104E0000B003200D2
:104AD00010C0B300004F780008003700C3DBBF00F0
:104AE0008040EB00014F7800FE40900080CF5000E6
:104AF00002003A0010C0B300004F78001E04E0002E
:104B000007003A007E409000604798006E40900099
:104B1000E84F500002003E006E409000C4FBB7001A
:104B200010C0B3009E4F10000D003A005E40900090
:104B30000081FB005E4090008080FB00B0BB210044
:104B400000804000904078001E40900080C07000BF
:104B5000B0BB21000000410001487800110037007F
:104B60005E4090000082FB005E4090008080FB0071
:104B7000B0BB2100008040001040780080417800E8
:104B80001E419000024078000080EA008180EA0027
:104B900000C0610080407800B0BB210000004200EE
:104BA000014878001E407800B22907007E4090003E
:104BB0000040E800704798001E4090000040400010
:104BC000104798001E4090000004E0000B003A00DF
:104BD0005E4090008080FB00B0BB21000080400060
:104BE00010407800840007005E4090000040E8001C
:104BF0005047980010C0B300104798005E409000E6
:104C0000E74F500091FF3600FE40900000C4B30013
:104C100080CF50000C003600C6DBBF000004E0006F
:104C200009003A006E409000C3FBB700C3DBBF0031
:104C30000004E00002003A0010C0B300C5FBB7005A
:104C400010C0B300404798004E4090000004E000C0
:104C500003003200BBDBBF000004E00008003A00A4
:104C60000040EB00C3FBB7000040EB00C5FBB70002
:104C70000040EB00C4FBB7000040EB004047980049
:104C80004E4090000080FB00400798004E009000CE
:104C90000080FA00000006000E00FA000040EB0061
:104CA000404798000C0037004E4090000081FB0008
:104CB0004E4090008080FB00B0BB2100008040008F
:104CC0009040780065004700017178004E409000E8
:104CD0000040E800404798004E409000E74F5000E9
:104CE000F1FF3600C3DBBF0020479800C5DBBF00E3
:104CF00010479800C4DBBF00004F780000C4B30029
:104D0000C3FBB7000040EB00C5FBB70031FF070055
:104D10000004E0001A00320010C0B30030479800D1
:104D20000040EB0040479800110037004E409000D3
:104D30008080FB0065004700614178004E40900094
:104D40008080FB00B0BB2100008040001040780054
:104D5000804F5100030032000040EB0030479800C4
:104D6000090037004E4090000040E800404798009E
:104D70004E409000E74F5000ECFF36000200370035
:104D80000040EB00304798000040EB00404798009F
:104D90000C0037004E4090000081FB004E40900018
:104DA0008080FB0065004700E1407800B0BB210037
:104DB00000004100014878004E4090000040E800AB
:104DC000404798004E409000E74F5000F1FF3600FA
:104DD0002E409000C3FBB7001E409000C5FBB700FB
:104DE0001E407800C4FBB7003E4090000080FB00EE
:104DF0000080FA00000006000200FA00004F780070
:104E0000C6DBBF001E4068008080FB00309A210096
:104E10000080400010407800C6FBB700C6DBBF0032
:104E20000080FB000080FA00000006000000FA008D
:104E3000C01D29003D0207000080FA0000000600A6
:104E40000400FA00C922A800CB22A900C8C2A90008
:104E50000BD8A8000B78A900F4FF0700000037006A
:104E600022C2BF00614060000004E000FCFF32008D
:104E70003011800069FBB70069DBBF000080FB00D8
:104E80004400DE0068FBB70068DBBF000080FB0069
:104E9000100798001E009000E10F50005C003200E7
:104EA0009E009000E48F5000770032001E009000BA
:104EB0000000E000010032007800370069DBBF002D
:104EC0000080FB00000F78009E007800E28F500009
:104ED000170032001E007800E20F500007003C006F
:104EE0009E0078000100E0006F0032001E00780094
:104EF000E10F50000C003200420037009E007800A5
:104F0000E48F50000F0032001E007800E40F5000C4
:104F10003C0035009E00780068805000E10F500092
:104F200038003E000A003700C0FF0700CCFF370002
:104F30006F28070066FBB70010C0B300900307009E
:104F4000C7FF3700E42807008D030700C4FF3700C0
:104F500010C0B3008A03070069DBBF00E94F5000AF
:104F600003003A00C0CEB300A2F9B7000200370038
:104F700000CFB300A2F9B70086FE070066FBB700BA
:104F8000110037000040EB0067FBB7000900370055
:104F900067DBBF008080FB00B0BB210000804000C9
:104FA000104078007603070067DBBF000040E80090
:104FB00067FBB70067DBBF00E74F5000F4FF360028
:104FC0007FFE070066FBB70066DBBF000004E00061
:104FD000ECFF3A000040EB0067FBB700050037002C
:104FE00000C0EB006603070067DBBF000040E8007D
:104FF00067FBB70067DBBF00E74F5000F8FF3600E4
:1050000097FF37000040EB005D03070094FF370077
:1050100091B6210091407800F0C0B30000C060005C
:1050200069FBB70069DBBF000040E80069FBB7001F
:1050300010C0B300520307000040EB0067FBB7004D
:105040000B00370022C2BF00614060000004E00096
:10505000FCFF3200301180005E28070010C0B30052
:105060004703070067DBBF000040E80067FBB700AD
:1050700071B621009140780069DBBF0080CF5000FD
:10508000F0FF390076FF370069DBBF00EC2A07002C
:1050900010C0B3003A03070071FF37000040EB0077
:1050A000370307006EFF37000080FA00000006009B
:1050B0000E00FA0030079800410798005207980048
:1050C0000000EB00100798000000EB00200798009C
:1050D0005E0090000000E0000600320080C2B300D5
:1050E000270307005E00900021020700E0042A0069
:1050F0008E010700E0C3B300210307000000EB00AE
:10510000100798000E80E80002BF2100BE0090004A
:10511000200007000000E000FAFF32001E009000AF
:105120000000E00006003A005E0090000000E00091
:10513000030032005E009000600798001200370004
:105140000000EB00200798001E009000E4004700DC
:1051500002BF210063000700000F78001E00E0007E
:10516000060032004E0090009E0F100003003E002B
:105170001E0078006007980003003700D0C1B3001C
:10518000EF2A0700DDFF37006E0090000080FA0074
:10519000000006000C00FA00100798002107980094
:1051A0003207980047003700EC020700004F7800F4
:1051B0001E80FB00500798005E009000E80F500032
:1051C0001C0032005E009000E80F500007003C0019
:1051D0005E0090000000E0000B0032005E009000D6
:1051E000E20F50000B0032001E0037005E009000FE
:1051F000EA0F50000A0032005E009000ED0F5000F0
:105200000700320017003700F00F20004007980019
:1052100031003700E00F2000400798002E003700D3
:1052200010052A00570107001000200040079800D1
:10523000290037001E009000100078000000E000F8
:10524000200032001E009000100078008000E9006D
:105250001E009000010878001E407800C802070078
:10526000180037001E009000900078002E0090007B
:10527000808F500013003100F0C1B3009E4F10002A
:1052800010003600E0C7B3009E4F10000D003E0036
:105290001E00900010007800800078003E00900012
:1052A000008040001E4878001E407800B4020700CD
:1052B0001E009000100078008000E8001E009000A2
:1052C000010878009F0207000004E000B6FF3A00E2
:1052D0000000EB00400798004E0090000080FA00AC
:1052E000000006001400FA0070079800010F9800F3
:1052F000120F98000040EB00004F78008E00E8008D
:105300000040EB00904098000E089000900078005C
:105310007E009000808F500006003A000E0890003A
:10532000100078008000E9000E0890000108780065
:105330006F0037000E0890001000780080007800A1
:105340001E0890000080400090407800F0C2B3003A
:1053500080CF5000090036000E0890001000780041
:10536000800078001E089000008040009040780087
:1053700090C3B30080CF5000480036000E08900064
:1053800010007800800078001E0890000080400027
:105390009040780000C4B30080CF50000900360070
:1053A0000E08900010007800800078001E08900021
:1053B000008040009040780060C4B30080CF50006F
:1053C000360036000E08900010007800800078004B
:1053D0001E089000008040009040780000C6B30096
:1053E00080CF5000090036000E08900010007800B1
:1053F000800078001E0890000080400090407800F7
:1054000060C6B30080CF5000240036000E08900024
:1054100010007800800078001E0890000080400096
:105420009040780080C7B30080CF50001B0032004E
:105430000E08900010007800800078001E08900090
:10544000008040009040780080C6B30080CF5000BC
:10545000120032000E0890001000780080007800E2
:105460001E089000008040009040780080C5B30086
:1054700080CF5000090032000E0890001000780024
:10548000800078001E089000008040009040780066
:1054900080C4B30080CF500010003A001E81FB0092
:1054A0000E08900010007800800078001E08900020
:1054B00000804000904078000E00E8000171780004
:1054C0001E4FE8000E089000100078008000E800F1
:1054D0000E089000010878008BFF37000E0890003E
:1054E000100078008000E9000E08900001087800A4
:1054F0008E00E8001E407800020007000080FA00DD
:10550000000006000A00FA004047980031079800A2
:105510000000EB00100798003E0090000000E8003B
:10552000104078000080FB004007980080062000B3
:10553000CE009000808F50000900320080072000CC
:10554000CE009000808F5000050032002006200021
:10555000CE009000808F50003F0032005400370092
:1055600020C0B300004F7800370037001E009000C5
:105570004400DD00100798001E80FB0080007800CA
:105580003E0090000080400090407800F0C3B300DF
:1055900080CF50000C003E001E80FB008000780091
:1055A0003E00900000804000104078008080FB00AA
:1055B0001E0090008080400000FD2F000080400011
:1055C000100798001F0037001E80FB008000780045
:1055D0003E009000008040009040780060C4B3001E
:1055E00080CF50000C003E001E80FB008000780041
:1055F0003E00900000804000104078008080FB005A
:105600001E0090008080400090FC2F000080400031
:10561000100798000B0037001E80FB008000780008
:105620003E00900000804000104078008080FB0029
:105630001E0090008080400090FA2F000080400003
:10564000100798001E4FE8004E4090009E4F10003B
:10565000C6FF39002B00370020C0B300004F780090
:105660000F0037001E009000000040001007980057
:105670001E80FB00800078003E009000008040000B
:105680009040780010C3B30080CF500003003A0070
:105690001E0090000000A000100798001E4FE800B8
:1056A0004E4090009E4F1000EEFF3900150037006D
:1056B0000040EB00004F78000F0037001E00900004
:1056C0006A00B900100798001E80FB008000780077
:1056D0003E00900000804000104078008080FB0079
:1056E0001E0090008080400000FD2F0000804000E0
:1056F000100798001E4FE8004E4090009E4F10008B
:10570000EEFF39001E0090000080FA000000060045
:105710000200FA00004F78001E4078000043B000FD
:10572000970107000080FA00000006000600FA005A
:1057300010079800020037001E4078009001070013
:105740001E009000104F78001E40780040479800DF
:105750004E4090000004E0000200320010C0B30090
:10576000404798004E4090009E0090008100E80065
:10577000110798000004E000EFFF3A000080FA00F3
:10578000000006000600FA0010079800020037002B
:105790001E4078007A0107001E009000104F78002C
:1057A0001E407800404798004E4090000004E00002
:1057B0000200320010C0B300404798004E409000F5
:1057C0009E0090008100E800110798000004E000AE
:1057D000EFFF3A00D0C0B30069010700A0C0B300DA
:1057E000670107000080FA00000006000400FA00CC
:1057F0002047980000C8B300004F780020052A0019
:10580000CAFF07000040EB00104798000F00370068
:105810002E4090001E4060000004E00003003200B3
:1058200010C3B300560107000200370000C3B300E5
:10583000530107001E80FB000000D100004F7800DC
:105840001E4090000040E800104798001E40900065
:10585000E74F5000EEFF36000080FA00000006001F
:105860000E00FA0050079800610798000040EB0016
:10587000004F780000102E00515F20003007980084
:10588000410798000040EB001047980030003700B7
:105890003E019000CE0190005E009000EE0090006E
:1058A00039EC070010079800210798001E04E0005B
:1058B00005003A001E009000AE009000E00F50007E
:1058C000E08F5800180032001E0090000043B00026
:1058D0002B0107009E0090003E009000000AB800D7
:1058E0009E0090004E0090000088B90005017800ED
:1058F00000014100BE0090002E0090000088B90019
:1059000000014100820278005E009000EE009000ED
:1059100004005000858058005007980061079800E7
:1059200010C0B300004F78003E009000CE00900001
:10593000A20020000300200013EC070030079800AD
:10594000410798001E4090000040E8001047980072
:105950001E409000E74F5000CDFF36005E009000E3
:105960000043B000060107000080FA0000000600B6
:105970000800FA00300798000040EB00004F780064
:1059800000712200200798000040EB0010479800AB
:105990001E0037003E0090002E019000110009000B
:1059A0000280D800100798001E04E00003003A00AF
:1059B0001E0090000000E0000C0032001E0090006D
:1059C0000043B000EE0007009E0090002E00900003
:1059D0000088B900800078003E009000010050006F
:1059E0003007980010C0B300004F78002E009000E0
:1059F000A2002000110009000280D80020079800B2
:105A00001E4090000040E800104798001E409000A3
:105A1000E34F5000DFFF36003E0090000043B0002F
:105A2000D70007000080FA00000006000600FA0018
:105A3000404798000040EB00004F780040C6B3009C
:105A4000304798000040EB002047980020003700C6
:105A50004E4090008080FB003E4090000081FB00A3
:105A6000110009008280D800104798001E04E00051
:105A700003003A001E4090000004E0000B003200DA
:105A80001E4090000043B000BD0007004E41900052
:105A90009E4090003E4090000088B90000405100B8
:105AA0004047980010C0B300004F78003E4090007F
:105AB0000080FB00A2002000110009000280D80035
:105AC000304798002E4090000040E80020479800A2
:105AD0002E409000E14F5000DDFF36004E40900018
:105AE0000043B000A60007000080FA000000060096
:105AF0000400FA001007980050062A000BFF070068
:105B00001E0090004400DE006F0F60009E007800D1
:105B100050052A00008040001040780098000700DF
:105B20001E0090006F0F60009E00780050052A0054
:105B30000080400010407800910007000080FA00CB
:105B4000000006000400FA001007980000C3B3002C
:105B5000E100070080C7B300DF0007001E009000CF
:105B60004400DE006F0F60009E00780050052A00A0
:105B70000080400010407800D70007001E00900011
:105B80006F0F60009E00780050052A0000804000E2
:105B900010407800D00007000080FA0000000600E6
:105BA0000400FA001007980050062A00DFFE0700E4
:105BB0001E0090004C00DE006F0F60009E00780019
:105BC00050052A0000804000104078006C0007005B
:105BD0001E0090004800DE006F0F60009E007800FD
:105BE00050052A0000804000104078006400070043
:105BF0001E0090004400DE006F0F60009E007800E1
:105C000050052A0000804000104078005C0007002A
:105C10001E0090006F0F60009E00780050052A0063
:105C20000080400010407800550007000080FA0016
:105C3000000006000800FA00300798003E009000BF
:105C4000CF80DE0036EA0700926C2200B3312400D8
:105C5000BCEA070010079800210798001E0090007A
:105C6000AE00900058EB0700004F78001E4078000F
:105C70006EFF0700E0C2B300410007001E00900065
:105C8000AE00900050EB0700CF80DE0024EA070052
:105C90000001BE001E009000AE0090004BEA07001D
:105CA000100798002107980002002000031224002A
:105CB0001E009000AE009000E4EA07001007980074
:105CC000210798001E009000AE0090003EEB0700F8
:105CD000004F78001E40780054FF07001E0090001F
:105CE000AE00900038EB0700CF80DE000CEA070022
:105CF0000001BE001E009000AE00900033EA0700D5
:105D000010079800210798000200200003122400C9
:105D10001E009000AE009000CCEA0700100798002B
:105D2000210798001E009000AE00900026EB0700AF
:105D3000004F78001E4078003CFF07000080FA000A
:105D4000000006000000FA0022C2BF0061406000AF
:105D50000080FB000080FA00000006000000FA004E
:105D600022C2BF00614060000004E000FCFF32007E
:105D7000301180000080FB000080FA000000060067
:105D80000200FA00004F780023C2BF0062406000AA
:105D90000004E000FCFF3A001E00FB002011880018
:105DA0000080FA00000006000200FA00004F7800B0
:105DB0001E80FB00401188000080FA0000000600F1
:105DC0000000FA0095C0BF00704060000004E000D1
:105DD00010003A0051E0800040E08000808F5000C9
:105DE0000C00320023C2BF00624060000004E000EB
:105DF000FCFF3A008580A9009580A80031E0800072
:105E000040E0800000804000104078000080FB00EF
:105E1000201188000080FA0000000600809FBE006C
:105E20000000FA0001E0800020E080008080400057
:105E3000301180008048780020E080000000E800F9
:105E400020E0880021E0800010E08000808F50007A
:105E500001003A009560A9008560A9000080FA0061
:105E60004F00BE0000400600809FBE000000FA0008
:105E700040E080000000E80040E0880041E0800051
:105E800050E08000808F500002003A009580A90009
:105E90000600370031E0800040E0800000804000D4
:105EA000104078000080FB00201188008580A90048
:105EB0000080FA004F00BE00004006000000FA001B
:105EC0000000EB00F0DF880010002000E0DF880019
:105ED0000080FA00000006000200FA00004F78007F
:105EE000E1DF8000F0DF8000808F500002003A0088
:105EF000C222A9000E003700E1DF80001E417800B9
:105F0000008020000080400002487800E0DF800030
:105F10000000E800E0DF8800E1DF800000002100F1
:105F2000808F500002003A000000EB00E0DF8800A4
:105F30000080FA00000006000200FA00F0DF800096
:105F4000000FE800000021009E0F100002003A0040
:105F50000000EB00000F7800E0DF80009E0F500093
:105F60000C00320023C2BF00624060000004E00069
:105F700008003A001E007800F0DF8800F1DF8000A2
:105F80000080200000804000104078000080FB006E
:105F9000201188000080FA00000006000400FA00CA
:105FA000000F7800110798001E007800900188000B
:105FB0001E0090001080BA00C800DD001E00900096
:105FC0001000BA00008070000080FA000000060097
:105FD0000600FA000CD8BF000080FB006101B90088
:105FE0001207980023079800D0012000010020002C
:105FF0001E019000AE019000800F5100818F59006A
:10600000F0003E001E009000AE0090000060010015
:106010002B0037004D0037001B0037001A003700F7
:1060200023003700CA003700E6003700E5003700DC
:10603000E4003700E3003700E2003700E1003700FA
:10604000E0003700DF003700DE003700DD003700FA
:10605000DC003700DB003700DA003700D9003700FA
:10606000D8003700D7003700D6003700D5003700FA
:10607000D400370060003700A9003700B2003700B5
:10608000D0003700D10037000CD8BF00E34F5000DC
:1060900002003A00767CA80001003700767CA90057
:1060A000CAC2A900A0C0B30025270700C700370057
:1060B000CAC2A800B0C0B30021270700C300370040
:1060C00080C08000E10F500008003A0010C0B3000B
:1060D0001B27070000C0EB002201070070FCB7007F
:1060E00070DCBF004B2507001500370020C0B3004F
:1060F0001327070080C080004625070030C0B3008A
:106100000F2707000000EB0070E38800080037004D
:1061100000C0EB00130107003E25070000C2B300DA
:1061200017FF070070E380000000E80070E38800BC
:1061300081C0800070E38000808F5000F4FF3E003B
:1061400020E629008FFD0700A000370040C0B30003
:10615000FB26070070C080002E25070080C080004D
:10616000E10F50000E003A0070C08000FD000700F3
:1061700070FCB70076DCBF00684060000004E000FF
:106180001A00320000C2B300FDFE070010C0B300C9
:10619000EB26070070DCBF001E2507001300370048
:1061A00030E6290061FD070080C080001925070046
:1061B00050C0B300E22607000000EB0070E3880047
:1061C0000600370070C08000E600070070FCB700D2
:1061D00070E380000000E80070E3880081C0800068
:1061E00070E38000808F5000F6FF3E0020E629001B
:1061F00064FD07007500370070E6290061FD0700A7
:10620000120020004100200010002000A8FB070021
:106210000040E9000AF8B700E0C2B300C826070052
:10622000120020002100200010002000A0FB070029
:106230000040E900614060006141600061C72100E9
:1062400091407800E0CFB30000C0600002407000D1
:1062500076FCB700F0C2B300B92607002200200088
:10626000210020001000200091FB07000040E90001
:1062700061406000614060000041400061C7210052
:1062800091407800D0CFB30000C0600002407000A1
:1062900076FCB70000C3B300A92607001200200057
:1062A000210020001000200081FB07000040E900D1
:1062B00061406000614060004201DD0061C7210073
:1062C00091407800B0CFB30000C060000240700081
:1062D00076FCB700E0C1B300992607001200200049
:1062E000210020001000200071FB07000040EA00A0
:1062F00061406000614060004601DD00B180210026
:1063000091407800F0CBB30000C060000240700004
:106310000BF8B7000B58A9000B98A8002B0037000A
:10632000767CA9000AD8BF008080FB0060C52100F0
:106330000080400010407800260007000040EB007D
:106340007F26070021003700720007001F0037007A
:1063500071C08000010F78001E0178000200E0008B
:10636000040032009E017800E18F510004003200E9
:1063700011003700F0E9290002FD07001300370083
:1063800010EC2900FFFC0700120020003100200063
:106390001000200046FB07000040E90070FCB70039
:1063A00070EF2900F7FC070070DCBF0011C0B300DC
:1063B0007A0007000500370070C1B30060260700AF
:1063C0000200370080C1B3005D2607000080FA009C
:1063D000000006000200FA00004F780041E2A90028
:1063E0000BD8BF000044B2000004E00004003200FB
:1063F000CEE2A800CF02A800CEC2A800030037005A
:10640000CEE2A900CF02A900CEC2A900816A200075
:106410009140780000CEB30000C060007040B3002F
:10642000A8E6B700916C20009140780000CEB30040
:1064300000C060007040B300C9E6B700816C200066
:106440009140780000CEB30000C060000034A0008E
:10645000C8E6B700CAC2A800C8C2A900C902A900FC
:10646000C8E2A800C922A9001E80FB001012880003
:1064700042A2A80076DCBF0061406000614060007D
:106480004601DD002124200091407800F0CBB300CC
:1064900000C060000240700042E2B70076DCBF003E
:1064A0000080FB000000D10061406000614160009D
:1064B0003124200091407800E0CFB30000C060009C
:1064C0000240700043E2B70076DCBF000080FB00B2
:1064D0004200DE0061406000614060000041400019
:1064E0003124200091407800D0CFB30000C060007C
:1064F0000240700043E2B7000000EB002012880069
:106500000000EB000012880041E2A8000080FA00C1
:10651000000006000000FA0041E2A900A8C6BF0082
:10652000F041B300A8E6B700916C200091407800DC
:1065300000CEB30000C06000C9E6B700816C200047
:106540009140780000CEB30000C06000C8E6B700FC
:10655000CEE2A900CF02A900CEC2A9000080FA00B5
:10656000000006000200FA00004F78001E80FB00C9
:106570004012880085C0BF00644060000004E00055
:10658000FCFF320040128000004F78008540A900D7
:106590001E80FB000080FA00000006000400FA00E4
:1065A000204798003147980044FE0700D9FF0700B4
:1065B0005F0007002E409000E14F500009003E00B0
:1065C000CAC2BF000080FB004600DE0061406000E0
:1065D0008080FB002E4090000080FB00808F5000E8
:1065E0000A003A0041C2BF0001C8B3000140600088
:1065F0000004E0000E003A0041E2A80061E2A800B9
:10660000B0C5B30034FE07000900370041C2BF0027
:1066100001C8B300014060000004E0000400320043
:1066200041E2A90061E2A900D0C5B3002AFE07003B
:1066300040C2BF000042B2000004E00020003A0067
:1066400060C2BF000042B2000004E0001C003A003B
:1066500040128000004F78003E4090000004E000AF
:10666000030032001E80FB0036FD070004003700E7
:10667000C0C5B30018FE07001E40780016FE0700D4
:1066800040138000004F780080C2B30012FE070064
:106690003E4090000004E000030032001E80FB003A
:1066A00028FD070004003700C0C5B3000AFE07003C
:1066B0001E40780008FE070090C2B30006FE0700E7
:1066C00040C2BF000044B2000004E00004003A00F1
:1066D00060C2BF000044B2000004E00002003200CB
:1066E00040C2A90060C2A90013FE070022C2BF0079
:1066F000614060000004E000AEFF32003011800015
:10670000004F780020E629001EFC070075000700F6
:106710000AD8BF008080FB0060C5210000804000D7
:10672000104078002BFF07000080FA0000000600F0
:106730000000FA00C8C2A800C902A800C8E2A80068
:10674000C922A800816A20009140780000CEB300E1
:1067500000C060009040B300A8E6B700916A200036
:106760009140780000CEB30000C060000034A0006B
:10677000A9E6B700C16A20009140780000CEB300BE
:1067800000C060007040B300ACE6B700D16A2000E2
:106790009140780000CEB30000C060000034A0003B
:1067A000ADE6B7000AD8BF008080FB0060C52100BD
:1067B00000804000104078000080FB00101288002C
:1067C00076DCBF0061406000614060004601DD0092
:1067D0002124200091407800F0CBB30000C060007D
:1067E0000240700042E2B70076DCBF000080FB0090
:1067F0000000D10061406000614160003124200050
:1068000091407800E0CFB30000C06000024070000B
:1068100043E2B7000000EB00201288000000EB000C
:10682000001288000AD8BF008080FB0060C52100EC
:1068300000804000104078000080FB0010138800AA
:1068400076DCBF0061406000614060004601DD0011
:106850002126200091407800F0CBB30000C06000FA
:106860000240700062E2B70076DCBF000080FB00EF
:106870000000D100614060006141600031262000CD
:1068800091407800E0CFB30000C06000024070008B
:1068900063E2B7000000EB00201388000000EB006B
:1068A000001388000000EB00401288000000EB009D
:1068B000401388004322A9006322A9004362A80074
:1068C00042A2A9006362A80062A2A90040C2A90076
:1068D00060C2A9004402A8006402A8000080FA0077
:1068E000000006000000FA0041E2A9004362A9008E
:1068F00061E2A9006362A900A8C6BF00F041B3002D
:10690000A8E6B700A9C6BF00F041B300A9E6B700EA
:10691000ACC6BF00F041B300ACE6B700ADC6BF00E7
:10692000F041B300ADE6B7000080FA0000000600B9
:106930000000FA0070F129007CFB07000080FA00DB
:10694000000006000400FA0010C0B3000AF8B70007
:10695000761CA900763CA800765CA9000BD8A8009C
:106960000AD8BF008080FB00A0C521000080400045
:106970001040780097FE0700EDFF07000000370089
:1069800022C2BF00614060000004E000FCFF320052
:106990003011800073FCB70073DCBF000080FB0087
:1069A0004400DE0072FCB70072DCBF000080FB0018
:1069B000100798001E009000E30F50008600320080
:1069C0001E009000E30F50000A003C001E009000E3
:1069D000E10F5000550032001E009000E10F500002
:1069E0006F003C001E0090000000E0000B00320031
:1069F000C60037001E009000E60F50008A003200EB
:106A00001E009000E80F5000970032001E0090001A
:106A1000E40F50007F003200BC00370073DCBF0081
:106A20000080FB00000F78001E007800E30F50008C
:106A3000220032001E007800E30F50000A003C00E4
:106A40001E007800E10F5000130032001E00780095
:106A5000E10F500012003C001E0078000000E00032
:106A60000B0032002E0037001E007800EE0F5000A1
:106A70001F0032001E007800EF0F5000220032008D
:106A80001E007800ED0F5000130032002400370084
:106A9000A0FE0700A0003700A5FF0700B8FF3700E1
:106AA00060168000F1FB2F00010060006016880076
:106AB00010C0B300B2FC0700B1FF370060168000C1
:106AC00001042000010070006016880010C0B300AF
:106AD000ABFC0700AAFF37008040EB0020C0B300EA
:106AE000AEFE070010C0B300A5FC0700A4FF3700EE
:106AF0008040EB000040EB00A8FE070010C0B30090
:106B00009FFC07009EFF37008040EB0010C0B300E1
:106B1000A2FE070010C0B30099FC070098FF3700E1
:106B20000040EB0096FC070095FF370031C72100BD
:106B300091407800F0C0B30000C0600073FCB70063
:106B400073DCBF000040E80073FCB70010C0B30066
:106B50008BFC07000040EB0071FCB7000A00370017
:106B600022C2BF00614060000004E000FCFF320070
:106B7000301180007BFE070081FC070071DCBF0044
:106B80000040E80071FCB70011C721009140780077
:106B900073DCBF0080CF5000F1FF390078FF370071
:106BA00031C7210091407800F0C0B30000C0600000
:106BB00073FCB70041C721009140780073DCBF002F
:106BC00000C0700074FCB70074DCBF0065FE0700F5
:106BD0006BFC07006AFF370041C721009140780035
:106BE000F0C0B30000C0600074FCB70073DCBF00ED
:106BF0000080FB004400DD008040780074DCBF00B2
:106C000000C0700074FCB70010C0B3005CFC07004B
:106C10005BFF370073DCBF000924070010C0B3001E
:106C200057FC070056FF370031C72100914078001C
:106C300070C0B30000C0600073FCB70073DCBF001D
:106C40000AF8B7000AD8BF008080FB00A0C5210069
:106C50000080400010407800DEFD070010C0B30047
:106C600047FC070046FF3700761CA900763CA900C8
:106C7000765CA9000BD8A90073DCBF000080FB0084
:106C80004200DE00610060000004E000010032000C
:106C9000761CA80073DCBF000080FB000000D10060
:106CA000610060000004E00001003200763CA800B2
:106CB00073DCBF000080FB00610060000004E000A6
:106CC00001003200765CA80073DCBF000080FB008E
:106CD0004300DE000000A200610060000004E0004C
:106CE000010032000BD8A8000AD8BF008080FB004A
:106CF000A0C521000080400010407800B5FD0700CD
:106D000010C0B3001EFC07001DFF37000040EB0061
:106D10001BFC07001AFF37000080FA000000060085
:106D20000600FA0048DCBF00E14F50002C003A009A
:106D300000C2B30012FC07000CD8BF00E34F5000A4
:106D4000060032000CD8BF00E24F500003003200B2
:106D50000CD8BF00E44F50000D003A0070C0B300E3
:106D6000F7230700E092290086FA070049DCBF00FC
:106D70000004E00003003A0010C0B3005D150700F6
:106D80001500370010C0B30077010700120037006C
:106D90000CD8BF00FD4F500003003A00F0922900CC
:106DA00078FA07005701370060C0B300E4230700FA
:106DB000E092290073FA070049DCBF000004E000FC
:106DC00003003A000040EB004A15070002003700BC
:106DD0000040EB00640107000040EB0048FCB700F6
:106DE0000CD8BF000080FB006101B90012079800B9
:106DF00023079800D0012000010020001E01900010
:106E0000AE019000800F5100818F59003B013E0080
:106E10001E009000AE009000006001001D003700D1
:106E20005A0037008900370088003700900037008B
:106E3000CE00370031013700300137002F01370015
:106E40002E0137002D0137002C0137002B013700B0
:106E50002A013700290137002801370027013700B0
:106E600026013700250137002401370023013700B0
:106E70002201370021013700200137001F013700B0
:106E800084003700A2003700B10037001B01370033
:106E90001C01370080C08000E10F50000D003A0057
:106EA00010C0B300A623070049DCBF000004E000C7
:106EB00003003A00CE1407004AFCB7000200370076
:106EC000460107004AFCB7004ADCBF00D121070099
:106ED0002B00370020C0B3009923070080C080003A
:106EE000CC21070030C0B300952307000000EB0061
:106EF00060E288001E00370060E280000000E000D1
:106F00000E00320000C2B3009DFB070060C0B3005A
:106F10008B23070000C2B30099FB070049DCBF00C8
:106F20000004E00003003A000040EB00F114070009
:106F3000020037000040EB000B01070049DCBF00F6
:106F40000004E00003003A00A91407004AFCB7005F
:106F500002003700210107004AFCB7004ADCBF00ED
:106F6000AC21070060E280000000E80060E28800D9
:106F700081C0800060E28000808F5000DEFF3E0014
:106F800010C0B30048FCB700DE00370040C0B300BB
:106F90006B23070070C080009E21070080C0800026
:106FA000E10F500006003600F0932900DFF90700DA
:106FB00080C080009721070050C0B3006023070005
:106FC0000000EB0060E288000F00370049DCBF00E2
:106FD0000004E00005003A0070C080005314070070
:106FE000B31407004AFCB7000400370070C08000EB
:106FF000F0000700D50007004AFCB70060E28000FF
:107000000000E80060E2880081C0800060E280004B
:10701000808F5000EDFF3E0000C2B30058FB070018
:107020004ADCBF000004E00003003A0060C0B30087
:10703000432307000200370070C0B300402307005D
:10704000E0922900CFF90700AE00370049DCBF000D
:107050000004E00002003A00C913070001003700F5
:10706000AA00070080C0B30035230700A500370041
:1070700049DCBF000004E00002003A00D31307001F
:1070800001003700A900070090C0B3002C230700BF
:107090009C0037000BD8A8000B98A8000040EB001C
:1070A00049FCB70049DCBF000004E00009003A00D9
:1070B00010C3B3002223070012002000410020006B
:1070C00010002000FAF707000040E9000AF8B700B6
:1070D0008C00370041C0800030002300808F5000BA
:1070E00002003E0030942900A6F90700909729007D
:1070F000A4F9070012002000310020001000200039
:10710000EBF707000040E9000AF8B7007D00370000
:1071100049DCBF000004E00009003A00C922A800D1
:10712000C902A800CB02A900CB22A900A18021009E
:107130009140780020C0B3005613070001003700CB
:10714000B10007000040EB00FD2207006D00370092
:107150000040EB0048FCB70049DCBF00E14F5000A5
:1071600068003A0007E2A9006600370071C080009D
:10717000010F78001E017800E10F51000A00320073
:107180009E017800E18F5100040039001E00780054
:10719000E20F50004900320055003700609A290084
:1071A00078F9070057003700C09D290075F90700DE
:1071B0000000EB0060E288003900370049DCBF00C6
:1071C0000004E00006003A006D13070060E2800052
:1071D000D6130700361407004AFCB7000500370035
:1071E0004A00070060E280007200070057000700B5
:1071F0004AFCB7004ADCBF000004E0001F003A0070
:1072000060E280000321070080C2B300DCFA0700BF
:1072100060E280000000D100FE20070060E28000F4
:107220000000A200610060000004E00003003200E2
:1072300050A129003DF907000C00370049DCBF00D0
:107240000004E00004003A00E913070010C0B30096
:1072500028140700030037006000070010C0B300C7
:107260004100070080A1290030F90700B0A12900E2
:107270002EF9070000C2B300C1FA070049DCBF00C5
:107280000004E00002003A0050130700010037003C
:107290002600070060E280000000E80060E288004D
:1072A00061E28000F00F2000808F5000C3FF3600A5
:1072B000E092290033F907001200370049DCBF00D3
:1072C000E14F500001003A0007E2A900D0A12900D7
:1072D0002CF9070010C0B3008E00070049DCBF0086
:1072E000E14F500007003A00470007000500370053
:1072F00070C1B300922207000200370080C1B300C2
:107300008F2207000080FA00000006000000FA004B
:107310000602A80006C2BF00614060000004E00051
:10732000FCFF3A000080FA00000006000000FA00AE
:107330000642A80006C2BF00644060000004E000EE
:10734000FCFF3A000080FA00000006000000FA008E
:1073500009C2BF000080FB004700DE000080FB0088
:107360000080FA00000006000200FA00004F7800DA
:107370009E40780061C06000614060004501DD0012
:107380006120200091407800F0CDB30000C0600083
:107390000240700006E2B7000682A80006C2BF00E5
:1073A000704060000004E000FCFF3A000080FA003A
:1073B000000006000200FA00004F78001E4078002E
:1073C00002E2B70009C2BF000044B2000004E000BE
:1073D000FCFF3A000080FA00000006000200FA00FC
:1073E0000662A80006C2BF00684060000004E0001A
:1073F000FCFF3A0000C2BF00004F78001E80FB0077
:107400000080FA00000006000000FA000742A90010
:107410000782A9000000EB00501088000000EB007C
:10742000601088000702A9000AD8BF008080FB0016
:1074300060CB210000804000104078000080FB00FD
:107440002010880007E2A8000080FA000000060073
:107450000000FA00C922A800C902A800CB02A900B6
:10746000CB22A90062A0A80062C0A8008660A90083
:10747000543CA9000040EB0052FCB70054DCBF00B4
:107480000080FB004200DE00634060008040780026
:10749000CBC2BF000080FB000000D1006140600053
:1074A00000C0700063406000634060004201DD0086
:1074B00041C521009140780030CFB30000C060008A
:1074C0000240700054FCB70054DCBF000080FB0099
:1074D0004400DE006340600080407800CBC2BF0003
:1074E0006140600000C07000634060006340600065
:1074F0004401DD0041C5210091407800F0CCB3008B
:1075000000C060000240700054FCB7000080FA0028
:10751000000006000400FA002047980067FA070000
:10752000CBFF07000000370083FA070022C2BF002C
:10753000614060000004E00005003200301180006E
:10754000004F7800E09229008EF807009E00370077
:1075500086C0BF00684060000004E000F2FF320017
:107560008660A90054DCBF000080FB004200DE0002
:107570006340600080407800CBC2BF000080FB0009
:107580000000D1006140600000C0700063406000F6
:10759000634060004201DD0041C521009140780058
:1075A00030CFB30000C060000240700054FCB70050
:1075B00054DCBF000080FB004400DE00634060003C
:1075C00080407800CBC2BF006140600000C0700006
:1075D00063406000634060004401DD0041C521005C
:1075E00091407800F0CCB30000C060000240700011
:1075F00054FCB70054DCBF00624060000004E000AF
:107600003B00320054DCBF000043B200F04F50009A
:1076100037003A0052DCBF00E74F500012003E0036
:1076200053DCBF000040400053FCB70053DCBF00F8
:107630000041780054DCBF000080FB004200DE0007
:107640006340600080407800D0CFB30000C060008D
:107650000040710053FCB70052DCBF000040E8005E
:1076600052FCB7003B003700CBC2BF000080FB00DC
:107670000000D100614060006141600041C521000F
:1076800091407800E0CFB30000C06000024070007D
:1076900054FCB7002E4090000004E00004003200CB
:1076A00053DCBF000080FB0026F907000400370010
:1076B000C0C5B30008FA070053DCBF0006FA070094
:1076C00054DCBF00614060000004E00003003200B1
:1076D000D0C2B30000FA070002003700B0C2B30006
:1076E000FDF907000040EB0052FCB700190037001D
:1076F00054DCBF0002C3B3008240600000C3B3008B
:1077000080CF500013003A0054DCBF006C40600092
:10771000E84F500006003A00543CA8000040EB003F
:1077200052FCB700B0C5B300EBF907000900370001
:1077300054DCBF006C406000E44F500005003A008C
:10774000543CA9000040EB0052FCB700D0C5B30088
:10775000E1F9070054DCBF000080FB004200DE00BE
:107760006340600000404000634060006340600090
:107770004201DD0041C521009140780030CFB300C7
:1077800000C060000240700054FCB70054DCBF0031
:107790000080FB004400DE006340600000404000C9
:1077A00063406000634060004401DD0041C521008A
:1077B00091407800F0CCB30000C06000024070003F
:1077C00054FCB70058FF37000080FA0000000600A4
:1077D0000000FA0040A42900D4F707000080FA0056
:1077E000000006000400FA00C922A800C902A8008F
:1077F000CB02A900CB22A900C8C2A9000BD8A800BF
:107800000B78A90080C0EB0020C0B300A1110700D5
:10781000EFFF07000000370022C2BF006140600098
:107820000004E000FCFF32003011800050FCB70083
:1078300050DCBF000080FB004400DE004FFCB700BE
:107840004FDCBF000080FB00100798001E00900076
:10785000E10F5000510032001E009000E10F500077
:1078600004003C001E0090000000E0000800320010
:10787000790037001E009000E40F500071003200C4
:107880001E009000E60F50006200320072003700C8
:1078900050DCBF000080FB00000F78001E00780065
:1078A000E30F5000240032001E007800E30F500068
:1078B0000A003C001E007800E10F50001800320062
:1078C0001E007800E10F500017003C001E007800F9
:1078D0000000E000630032002D0037001E00780039
:1078E000E60F50001B0032001E007800E60F50002B
:1078F00004003C001E007800E40F5000120032002B
:10790000230037001E007800E70F500016003200F9
:107910001E007800EF0F5000180032001C003700E6
:10792000ABFF0700BCFF37009511070010C0B30084
:1079300013F90700B8FF3700A411070010C0B30007
:107940000FF90700B4FF3700291207000CF90700F0
:10795000B1FF37000040EB006612070010C0B30013
:1079600007F90700ACFF370010C0B3006112070031
:1079700010C0B30002F90700A7FF37000040EB007A
:10798000E4FE070010C0B300FDF80700A2FF3700B7
:107990000040EB00FAF807009FFF370001C5210007
:1079A00091407800F0C0B30000C0600050FCB70008
:1079B00050DCBF000040E80050FCB70010C0B3002E
:1079C000EFF807000040EB004EFCB7000B0037005B
:1079D00022C2BF00614060000004E000FCFF3200F2
:1079E00030118000D111070031120700E4F80700C0
:1079F0004EDCBF000040E8004EFCB700E1C42100AF
:107A00009140780050DCBF0080CF5000F0FF39007B
:107A100081FF370001C521009140780030C0B300DC
:107A200000C0600050FCB70001C521009140780003
:107A300020C0B3001711070010C0B300D0F8070032
:107A400075FF370050DCBF007D20070010C0B30079
:107A5000CBF8070070FF37000040EB00C8F80700C4
:107A60006DFF37000080FA00000006000600FA00F3
:107A70000CD8BF000080FB006101B900120798001C
:107A800023079800D0012000010020001E01900073
:107A9000AE019000800F5100818F59008B013E0094
:107AA0001E009000AE00900000600100470037000B
:107AB0006B003700890037008800370090003700DE
:107AC0000101370081013700800137007F01370055
:107AD0007E0137007D0137007C0137007B013700D4
:107AE0007A013700790137007801370077013700D4
:107AF00076013700750137007401370073013700D4
:107B00007201370071013700060037006F0137003E
:107B100080003700CA003700E90037006B013700EA
:107B20006C013700ED1F07000004E000690132001E
:107B30006CDCBF00704060000004E00021003200F7
:107B4000604629000FF7070010C0B3007C20070033
:107B500032C2BF00684060000004E0000200320052
:107B600070462900F1F6070032C2BF006440600091
:107B70000004E00002003200B0462900EBF60700E6
:107B8000CD1F070064FCB70064DCBF00A11E070026
:107B900032C2BF00624060000004E0000600320014
:107BA000F0462900E1F6070090118000D1FF2F0078
:107BB000010060009011880060462900F1F607007E
:107BC00044013700BC1F07004201370010C0B3005A
:107BD0005B200700C11F07000004E0001D00320009
:107BE00032C2BF00684060000004E00002003200C2
:107BF00070462900CDF6070032C2BF006440600025
:107C00000004E00002003200B0462900C7F6070079
:107C1000A91F070064FCB70064DCBF007D1E0700DD
:107C200032C2BF00624060000004E0000600320083
:107C3000F0462900BDF6070090118000D1FF2F000B
:107C4000010060009011880060462900CDF6070011
:107C500020013700F0472900CAF607001D01370050
:107C600040C0B3003620070070C08000691E0700C6
:107C700080C08000E10F500003003A0070C0800017
:107C8000831F070012003700F0482900A7F60700FD
:107C900080C080005F1E070050C0B300282007008E
:107CA0000000EB0010E388000500370070C0800082
:107CB000771F070010E380000000E80010E3880051
:107CC00081C0800010E38000808F5000F7FF3E00ED
:107CD00060462900ABF60700FE00370090118000D7
:107CE000D1FF2F0001006000901188006C9CA8005B
:107CF0000B38A80030492900A2F60700F50037002C
:107D00006C9CA9000B38A900004B29009DF60700C8
:107D1000F0003700D0C2B30009200700504C290002
:107D200098F6070012002000A1002000200020008B
:107D3000DFF407000040E9000AF8B700704D2900A1
:107D400090F60700120020004100200010002000E3
:107D5000D7F407000040E900634060006341600021
:107D6000C1C6210091407800C0CFB30000C06000C0
:107D7000024070006CFCB700C052290081F6070079
:107D8000120020002100200010002000C8F407008D
:107D90000040E90061406000614060004201DD0098
:107DA000C1C6210091407800B0CFB30000C0600090
:107DB000024070006CFCB700E054290071F6070027
:107DC000120020002100200010002000B8F407005D
:107DD0000040E90061406000614060004301DD0057
:107DE000C1C621009140780070CFB30000C0600090
:107DF000024070006CFCB700E0C1B300D01F070068
:107E0000120020002100200010002000A8F407002C
:107E10000040EA0061406000614060004601DD0012
:107E2000B180210091407800F0CBB30000C0600029
:107E3000024070000BF8B7000B98A800A5003700AF
:107E40006CDCBF000080FB004200DE00614060008F
:107E5000004178006CDCBF00634060008041780026
:107E60006CDCBF000080FB004300DE00614060006E
:107E7000004378000BD8BF000080FB004600DE0006
:107E800061406000804278000AD8BF000080FB009B
:107E90008000400080BC210000804000100078007D
:107EA000024278000641780085407800A21E070053
:107EB0000040EB00A21F0700E11E0700850037000D
:107EC000E51E07008300370071C08000010F7800B5
:107ED0001E017800E10F5100110032009E01780070
:107EE000E18F5100070039001E007800E20F5000BA
:107EF000590032009E007800E38F500004003200E9
:107F00006F003700105829001EF607007100370077
:107F1000C062A900C082A800C8C2A800C902A90006
:107F2000405E290017F607008CF7070080407800B4
:107F300000C2B30080CF500066003A007061290093
:107F400010F6070090118000D1FF2F0001006000A3
:107F5000901188000000370032C2BF00614060000D
:107F60000004E0000600320023C2BF00624060004F
:107F70000004E00002003A00B011800020118800E7
:107F800022C2BF00614060000004E0000600320031
:107F900033C2BF00624060000004E00002003A000B
:107FA00030118000A011880032C2BF006240600022
:107FB0000004E00004003A0022C2BF0062406000FA
:107FC0000004E0000900320091118000D0FF2F0072
:107FD000008060009011880011118000D0FF2F00F8
:107FE0000080600010118800C222A90070C08000CB
:107FF000E30F5000D8FF3A00C2C2BF000080FB0070
:108000004400DE006140600061416000B12C20004E
:1080100091407800E0CFB30000C0600002407000E3
:10802000CBE2B700CAC2BF000080FB004600DE0002
:1080300061406000614060004301DD00212C2000B0
:108040009140780070CFB30000C060000240700023
:10805000C2E2B700C0FF370060622900C9F507001F
:1080600090118000D1FF2F00010060009011880066
:108070000000370032C2BF00614060000004E00031
:108080000600320023C2BF00624060000004E0002E
:1080900002003A00B01180002011880022C2BF0007
:1080A000614060000004E000F2FF32003111800006
:1080B00000022000808F500006003200EDFF3700E4
:1080C00070C1B3001E1F07000200370080C1B3005B
:1080D0001B1F07000080FA00000006000000FA00E5
:1080E0005064290091F507000080FA0000000600A6
:1080F0000400FA006C1CA9006C3CA9006C5CA9008F
:108100006C7CA9000BD8A800E0DE800030E388007A
:108110006C9CA9006CDCBF000080FB004200DE000C
:1081200061406000804178006CDCBF00634060000B
:10813000804278006CDCBF000080FB004300DE0062
:1081400061406000004178000BD8BF000080FB0058
:108150004600DE00614060008040780030E380002F
:108160000342780085417800F31D0700341E0700A4
:10817000DAFF070000003700581E07000004E00087
:10818000080032006CDCBF00704060000004E000BA
:1081900003003200481E0700F9F60700010037000F
:1081A000451E070032C2BF00624060000004E000CC
:1081B0000400320090118000D1FF2F000100600008
:1081C0009011880022C2BF00614060000004E000FE
:1081D000E9FF3200301180006AFCB7006ADCBF00A2
:1081E0000080FB004400DE0069FCB70069DCBF00D2
:1081F0000080FB00100798001E009000E40F500064
:10820000AE0032009E009000E48F500007003C005A
:108210001E0090000000E0000F0032009E00900061
:10822000E18F5000870032002C0137001E009000C3
:10823000E60F5000A60032009E009000E68F50002E
:10824000260135009E00900068805000E10F50002C
:1082500022013E00CA0037006ADCBF000080FB003C
:10826000000F78001E007800E20F50001800320066
:108270009E007800E28F500007003C001E0078004E
:108280000000E0000E0032009E007800E18F5000F8
:108290000D003200680037001E007800E70F500024
:1082A0001B0032009E007800EF8F50004600320025
:1082B0001E007800E30F5000110032005E0037000E
:1082C000E51D07000801370084FF0700AAFF3700FB
:1082D00010C0B300AAF6070032C2BF0062406000BF
:1082E0000004E0000400320090118000D1FF2F0054
:1082F00001006000901188006C9CA8009EFF370070
:108300006C9CA90010C0B3009DF607009AFF3700CF
:1083100010C0B3009AF60700CF1D070022C2BF00AD
:10832000614060000004E000FCFF3200301180007A
:108330004800DD0030E3880010C0B30090F607006D
:1083400022C2BF00614060000004E000FCFF320078
:1083500031E38000301180000080700030E388003D
:108360006CDCBF000080FB004200DE00614060006A
:10837000804178006CDCBF00634060008042780080
:108380006CDCBF000080FB004300DE006140600049
:10839000004178000BD8BF000080FB004600DE00E3
:1083A000614060008040780030E380000342780044
:1083B00085417800601D0700A11D070010C0B300B3
:1083C0006FF607006CFF370010C0B3006CF60700B3
:1083D00090118000D1FF2F000100600090118800F3
:1083E0000000370032C2BF00614060000004E000BE
:1083F0000600320023C2BF00624060000004E000BB
:1084000002003A00B01180002011880022C2BF0093
:10841000614060000004E000F2FF320033C2BF00A0
:10842000624060000004E000EEFF3A00301180007E
:10843000A0118800EBFF37000040EB0050F607006A
:108440004DFF3700A1C6210091407800F0C0B30075
:1084500000C060006AFCB7006ADCBF000040E800B2
:108460006AFCB70010C0B30045F607000040EB00FF
:1084700068FCB7000B00370022C2BF0061406000FB
:108480000004E000FCFF320030118000801D070076
:1084900010C0B3003AF6070068DCBF000040E800F7
:1084A00068FCB70081C62100914078006ADCBF00FB
:1084B00080CF5000F0FF39002FFF37006ADCBF008B
:1084C000DF1D070010C0B3002DF607002AFF37009C
:1084D000A1C6210091407800F0C0B30000C0600048
:1084E0006AFCB7006ADCBF00EA4F500002003600A9
:1084F000A0C0B3006AFCB7006ADCBF000080FB00CC
:1085000080004000C0BD21000080400010007800C5
:1085100030E38800501D07006CDCBF000080FB00CA
:108520004200DE0061406000804178006CDCBF00EA
:1085300063406000804278006CDCBF000080FB007C
:108540004300DE0061406000004178000BD8BF00AE
:108550000080FB004600DE00614060008040780043
:1085600030E380000342780085417800F21C070068
:10857000331D070010C0B30001F60700FEFE3700F0
:108580006C1CA9006C3CA9006C5CA9006C7CA90067
:108590000BD8A9006ADCBF000080FB004300DE00AE
:1085A000610060000004E0000B0032006CDCBF00E2
:1085B000634060000014A0006340600063416000FD
:1085C000C1C6210091407800C0CFB30000C0600058
:1085D000024070006CFCB7006ADCBF000080FB004A
:1085E0004200DE00610060000004E0000B00320089
:1085F0006CDCBF00634060000004A00063406000CA
:1086000063416000C1C6210091407800C0CFB30033
:1086100000C06000024070006CFCB7006ADCBF0064
:108620000080FB000000D100610060000004E00059
:10863000010032006C5CA8006ADCBF000080FB0017
:10864000610060000004E000010032006C7CA800C2
:108650006ADCBF000080FB004400DE000000A200D6
:10866000610060000004E000010032000BD8A800A7
:10867000F91C07006CDCBF000080FB004200DE003C
:1086800061406000804178006CDCBF0063406000A6
:10869000804278006CDCBF000080FB004300DE00FD
:1086A00061406000004178000BD8BF000080FB00F3
:1086B0004600DE00614060008040780030E38000CA
:1086C00003427800854178009B1C0700DC1C0700F2
:1086D00010C0B300AAF50700A7FE37000040EB006A
:1086E000A7F50700A4FE37000080FA00000006008E
:1086F0000600FA000CD8BF000080FB006101B90041
:108700001207980023079800D001200001002000E4
:108710001E019000AE019000800F5100818F590022
:108720002C013E001E009000AE0090000060010091
:108730005200370072003700400037004500370014
:108740004A003700B80037008E0037009600370027
:108750009E003700A4003700A7003700AA003700AA
:10876000AD0037001B0137001A013700190137002F
:1087700018013700170137001601370015013700BF
:1087800014013700130137001201370011013700BF
:108790001001370004003700240037000F013700B4
:1087A0000C0137000D013700E0C1B300641D070064
:1087B0001200200021002000100020003CF20700E1
:1087C0000040E900614060006141600001C8210093
:1087D00091407800E0CFB30000C06000024070001C
:1087E00080FCB70080DCBF00614060000041780081
:1087F000024078000080EA008180EA006140600069
:10880000614060004601DD00B180210091407800A8
:10881000F0CBB30000C06000024070000BF8B7005E
:108820000B58A8000B98A800EC0037007C0107004B
:108830000040EB00421D0700E8003700E900070098
:1088400020C0B30039010700201E2900CDF3070026
:10885000E2003700E300070030C0B3003301070037
:10886000C0202900C7F30700DC003700DD00070047
:1088700040232900C3F30700D800370080C08000E0
:10888000E10F500007003A00D60107007EFCB70058
:1088900010C0B3002A1D07007EDCBF005D1B07006F
:1088A0001400370020C0B300251D070080C08000E1
:1088B000581B070030C0B300211D07000000EB006B
:1088C000E0E3880007003700C6010700511B0700DE
:1088D00000C2B3002AF50700E0E380000000E800D2
:1088E000E0E3880081C08000E0E38000808F5000DA
:1088F000F5FF3E0010242900A2F30700B70037005F
:1089000040C0B3000E1D070070C08000411B07006F
:1089100080C08000E10F500004003A0070C0800069
:108920004A0107007EFCB70013003700202429000D
:108930007EF3070080C08000361B070050C0B300E4
:10894000FF1C07000000EB00E0E388000600370092
:1089500070C080003D0107007EFCB700E0E38000AE
:108960000000E800E0E3880081C08000E0E38000D0
:10897000808F5000F6FF3E001024290081F307008D
:1089800096003700DB0107007EFCB700D0C0B300C3
:10899000EB1C07007EDCBF005DF3070010242900FC
:1089A00078F307008D003700E0C0B300E41C070037
:1089B000DA0107007EFCB7007EDCBF0054F307003D
:1089C000102429006FF307008400370080C0800066
:1089D000101B070000C1B300D91C070080C0800035
:1089E000FA0107007D00370010C1B300D41C070056
:1089F000030207007900370020C1B300D01C070034
:108A00001B0207007500370030C1B300CC1C070003
:108A1000C90107007100370040C1B300C81C07003E
:108A2000E30107006D00370071C08000010F78007E
:108A30001E017800E10F51000D0032009E01780008
:108A4000E18F5100070039001E007800E20F50004E
:108A50000C0032009E007800E38F5000530032007B
:108A6000590037006024290030F307005B0037000D
:108A7000A50007003029290042F30700590007002C
:108A800056003700102A29003EF307009E00070019
:108A9000302929003BF30700A70107005100070018
:108AA00020C0B300A100070000C0EB00C701070011
:108AB00000C0EB00C50107004A00070030C0B3004A
:108AC0009A0007000000EB00E0E388000700370091
:108AD000E0E380000000E800E0E38800E1E38000DC
:108AE000900F2000808F500003003E00810107009E
:108AF0000004E000F6FF32003A00070082000700A1
:108B0000302929001FF307003600070030C0B300EA
:108B100086000700E0E38000BE1A0700102B290042
:108B200018F307000040EB007EFCB7001800370088
:108B30007EDCBF000040E800B61A0700A02C290028
:108B4000FAF2070027010700B21A070000C2B300BB
:108B50008BF4070023010700AE1A070000C2B30020
:108B600087F407001F010700AA1A070000C2B3001C
:108B700083F407001B010700A61A07001024290030
:108B800000F307007EDCBF000040E8007EFCB70079
:108B90007EDCBF008080FB00E0E38000808F50001F
:108BA000E3FF39000F0007000C003700E02C29001C
:108BB000F4F2070010312900F2F2070060342900B6
:108BC000F0F207000500370070C1B3005C1C07001D
:108BD0000200370080C1B300591C07000080FA0072
:108BE000000006000200FA0010372900CFF207004B
:108BF00078DCBF000080FB00000F78001E007800CA
:108C0000E10F50000E0032001E007800E10F50000E
:108C100004003C001E0078000000E0000B00320061
:108C2000350037001E007800E20F50000F003200C0
:108C30001E007800E30F5000240032002E003700A1
:108C4000A0372900CFF207002D003700AD01070043
:108C500010C0B3005D01070010C0B30078FCB7007E
:108C600070382900C7F207002500370079DCBF0003
:108C7000E14F50000A003A007ADCBF00E14F50009B
:108C800002003A002C0107000100370048010700EC
:108C90000040EB0079FCB70030392900A3F207004F
:108CA0007A01070020C0B3004801070095010700C2
:108CB00010C0B3004501070010C0B30078FCB70036
:108CC000803A2900AFF207000D0037006F0107005E
:108CD00020C0B3003D0107008A01070010C0B300A7
:108CE0003A01070010C0B30078FCB700103B290020
:108CF000A4F2070002003700A03B2900A1F2070000
:108D00000080FA00000006000000FA005F01070082
:108D1000A0C0B3002D0107007A0107000040EB005E
:108D200078FCB7000080FA00000006000400FA009A
:108D3000004F780078DCBF00E14F500002003200A5
:108D4000803C29008FF207001037290077F20700D6
:108D50001E80FB00100798001E009000E10F5000DD
:108D60000E0032001E009000E10F500004003C0095
:108D70001E0090000000E0000B00320024003700CD
:108D80001E009000E20F5000160032001E009000FE
:108D9000E30F5000080032001D003700A037290003
:108DA00078F207001C003700D7FF0700403E29007B
:108DB00074F20700180037003401070010C0B30038
:108DC000020107004F01070020C0B300FF000700A9
:108DD00030C0B30078FCB700A03E290069F207005C
:108DE0000D0037002901070020C0B300F70007007D
:108DF0004401070020C0B300F400070020C0B30006
:108E000078FCB700E03F29005EF20700020037005F
:108E1000304329005BF207000080FA0000000600E2
:108E20000000FA00C8E2A800C902A900C922A900EE
:108E3000C8C2A900CAE2A900CB02A900CB22A9009E
:108E4000CAC2A9000080FA00000006000800FA006B
:108E5000404798000601070079DCBF00E14F500051
:108E600006003A007ADCBF00910007000040EB00EA
:108E700079FCB700D044290042F207000BD8BF00AC
:108E8000684060000004E0000300320010C0B3003E
:108E9000004F78000200370000C8B300004F780090
:108EA0000040EB0030479800450037004E409000EE
:108EB0001E4060000004E00002003A00BC00070011
:108EC000010037009C000700CD000700CAC2BF00A8
:108ED0000080FB004700DE00204798000BD8BF0051
:108EE000684060000004E000100032004E40900036
:108EF0000080FB000000D100404798001E40900019
:108F00000080FB000000D100104798002E40900028
:108F1000E14F500011003A001E40900001C8B3001C
:108F200001404000104798000C0037004E40900070
:108F300000404000404798001E4090000040400024
:108F4000104798002E409000E14F500003003A0077
:108F50001E4090000040E80010479800C400070041
:108F600078DCBF00E24F500012003A003E40900013
:108F7000E64F50000F003A0010C0B30079FCB70074
:108F80004E4090001E4060000004E00003003A00E4
:108F90000040EB007AFCB7000200370010C0B300BD
:108FA0007AFCB7001E4090000080FB00300798005C
:108FB000090037003E4090000040E800304798002C
:108FC0003E409000E74F5000B8FF36001E40900032
:108FD0000080FB00300798003E0090000080FA00FF
:108FE000000006000400FA00A100070079DCBF00C1
:108FF000E14F500006003A007ADCBF002C00070069
:109000000040EB0079FCB700D0442900DDF10700F7
:109010000040EB00204798001F0037007800070051
:10902000CAC2BF000080FB004700DE001047980066
:109030000BD8BF00684060000004E00008003A0060
:109040001E40780000404000004F78001E40900015
:109050000004E0000C0032001E4FE8000A00370058
:109060001E80FB000000D100004F78001E409000E1
:109070000004E000040032001E40780001C8B30084
:1090800001404000004F7800790007002E4090001A
:109090000040E800204798002E409000E74F500025
:1090A000DEFF36001E80FB000080FA000000060094
:1090B0000400FA00204798002E4090000004E000D1
:1090C00002003A003A000700010037001A000700CA
:1090D0004B000700CAC2BF000080FB004700DE0053
:1090E000004F7800620007001E80FB000080FA003D
:1090F000000006000200FA0041000700CAC2BF00DB
:109100000080FB004700DE00004F78005800070099
:109110001E80FB000080FA00000006000000FA003C
:10912000CAC2BF000080FB004700DE000080FB00D9
:109130000080FA00000006000000FA0080DCBF009A
:109140006140600000417800024078000080EA0041
:109150008180EA00614060006140600000414000A1
:10916000912C200091407800D0CFB30000C0600067
:1091700002407000C9E2B70080DCBF0061406000BF
:109180006140600000414000B12C20009140780017
:10919000D0CFB30000C0600002407000CBE2B70047
:1091A00040C1B300521907000080FA000000060019
:1091B0000000FA00CB22A900C922A90040C1B300D7
:1091C0004B1907000080FA00000006000400FA00B6
:1091D000204798000040EB00004F78000300370064
:1091E00007000700220007001E4FE8002E409000F5
:1091F0009E4F1000FAFF39000080FA0000000600C0
:109200000000FA0080DCBF0061406000004178008F
:10921000024078000080EA008180EA00614060003E
:1092200061416000912C200091407800E0CFB300B4
:1092300000C0600002407000C9E2B70080DCBF00DF
:109240006140600061416000B12C200091407800D5
:10925000E0CFB30000C0600002407000CBE2B70076
:1092600040C6B300221907000080FA000000060083
:109270000000FA00CB02A900C902A90040C6B30051
:109280001B1907000080FA00000006000000FA0029
:1092900080DCBF006140600000417800024078003F
:1092A0000080EA008180EA00614060006140600067
:1092B0004601DD00812C200091407800F0CBB30006
:1092C00000C0600002407000C8E2B70080DCBF0050
:1092D00061406000614060004601DD00A12C20007B
:1092E00091407800F0CBB30000C0600002407000F5
:1092F000CAE2B70040C1B300FD1807000080FA00C1
:10930000000006000000FA00CAC2A900C8C2A900F5
:1093100040C1B300F61807000080FA000000060004
:109320000800FA00004F780000C6B3009E4F1000FE
:1093300007003600A0C7B3009E4F100004003E0097
:109340001E40780001CEB30001404000004F78007D
:109350001E80FB006101B900D0FD2F00F1FF2F003E
:1093600002014000838148002207980033079800DB
:10937000B0052000010020002E019000BE019000E9
:10938000800F5100818F5900A6003E002E009000F2
:10939000BE00900000600100820037008D003700A1
:1093A000A00037009F0037009E0037009D00370067
:1093B0009C0037009B00370082003700990037007F
:1093C0009800370097003700960037009500370067
:1093D0009400370093003700920037009100370067
:1093E000900037008F0037008E0037008D00370067
:1093F0008C0037008B0037008A0037008900370067
:1094000072003700870037005000370085003700B2
:1094100084003700610037005800370081003700B2
:10942000800037004B0037004C0037007D003700CC
:109430004C0037007B0037007A00370041003700CE
:109440003100370077003700310037003200370035
:109450007400370073003700720037007100370066
:1094600070003700350037006E0037006D003700A0
:109470006C0037006B0037006A0037006900370066
:109480006800370067003700660037006500370066
:109490006400370063003700620037006100370066
:1094A000600037005F0037005E0037005D00370066
:1094B0005C0037005B0037005A0037005900370066
:1094C0005800370057003700560037005500370066
:1094D0005400370053003700520037005100370066
:1094E000500037004F0037004E0037004D00370066
:1094F0004C0037004B0037004A0037004900370066
:10950000480037003D0037001E01070048003700C3
:1095100046010700460037000BD8BF0070406000CE
:109520000004E00003003A0080C1B300041A070001
:109530003F0037004A0107003D0037006E01070079
:109540003B0037008A01070039003700061A070080
:1095500037003700F6120700350037005C120700AD
:10956000330037004D00070020C080000000E000FD
:109570002F003200870007002D00370020C0800038
:109580000000E00003003A0080C1B300EC190700BE
:10959000270037009901070025003700B2010700B6
:1095A00023003700A0A4290076F0070023C2BF00E3
:1095B000614060000004E000FCFF32000000FE009B
:1095C0001B003700C6010700190037001D00070007
:1095D0001700370000A529006AF00700A717070049
:1095E00023C2BF00614060000004E000FCFF3200C5
:1095F00081BF2A00014001000D00370020C080001B
:109600000000E00004003A0011C0B30010C0B30035
:10961000C214070006003700B0A5290059F0070062
:10962000030037008000EB001107980002003700AC
:1096300012002000120798001E0090000080FA001F
:10964000000006000200FA0070A7290037F00700AA
:1096500012002000F10F2000A000200094EE07006F
:10966000004F78001E80FB0021F1070000A82900B0
:1096700044F007001E407800ECF0070000A8290025
:1096800040F007001E40780058F0070000A82900AD
:109690003CF007000080FA00000006000400FA0019
:1096A00010A8290037F00700F0A829001FF00700D4
:1096B000D0A929001DF00700A1BF2A000000EB007F
:1096C00036F20700000F78001E0078004800DE0028
:1096D000D6F00700E0C2B300A9F107001E00780031
:1096E000D2F0070000A8290026F00700B0AA290040
:1096F0000EF0070030C0800029F1070020AB2900E0
:109700000AF0070040C0800025F10700A0AB290047
:1097100006F0070040C080001007980020042300D6
:109720009E009000808F50000C0032003004230017
:109730009E009000808F50000B003200300023000C
:109740009E009000808F5000010032000900370019
:10975000D0AB2900F5EF07000800370000AC290066
:10976000F2EF07000500370030AC2900EFEF0700EB
:109770000200370060AC2900ECEF0700A0AC290024
:1097800000F00700C0AC2900FEEF07000080FA00DF
:10979000000006000000FA00B0AE2900F9EF070053
:1097A00080AF2900F7EF0700C0B02900DFEF070006
:1097B000002020005900070000102000570007007B
:1097C0000008200055000700000420005300070097
:1097D000004020005100070000A82900E9EF070021
:1097E00010B12900D1EF0700002020005800070029
:1097F0000010200056000700000820005400070059
:109800000004200052000700004020005000070024
:1098100000A82900DBEF07000BD8BF0001C8B30088
:10982000014060000004E0000300320050C1B300BA
:10983000431907000200370060C1B3004019070058
:10984000AD0007000BD8BF00614060000004E000DD
:1098500003003200B0C2B30039190700020037001C
:10986000A0C2B300361907000BD8BF000044B200F5
:109870000004E0000300320020C3B30030190700E9
:109880000200370030C3B3002D1907000BD8BF000A
:10989000704060000004E0000A0032000BD8BF00F6
:1098A0000042B2000004E0000300320040C2B300F6
:1098B000231907000500370030C2B3002019070044
:1098C0000200370040C3B3001D1907000BD8BF00CA
:1098D000644060000004E0000A0032000BD8BF00C2
:1098E000684060000004E0000300320080C2B30062
:1098F000131907000500370070C2B30010190700E4
:109900000200370050C3B3000D190700B0AE2900A4
:109910009CEF07000080FA00000006000200FA0039
:10992000000F7800401680001E0060000000E0007C
:109930000300320060B129007CEF0700020037000D
:10994000A0B1290079EF07000080FA0000000600AE
:109950000200FA00000F7800501680001E00600020
:109960000000E00003003200E0B129006FEF0700C3
:109970000200370020B229006CEF07000080FA00D7
:10998000000006000200FA00B0C1B3000CF8B700F6
:1099900058180700B916070092180700004F780002
:1099A0000040EB00104798000C0037001E4090006C
:1099B0000040E8001DF0070060B229005BEF0700DF
:1099C0001E4090009418070000A829006DEF0700C2
:1099D0001E4090000040E800104798001E40900094
:1099E0009E4F5000F1FF39009E80FB0012002000C6
:1099F00020002000AEED07000000E90020C0880034
:109A0000F0C1B300CE18070090C1B3000CF8B70046
:109A100038180700C222A800A0C1B3000CF8B70094
:109A2000341807000080FA00000006000000FA0069
:109A300000C2B300C218070012002000410020003D
:109A4000100020009AED07000000E90010C0880017
:109A500010C2B300BA1807000080FA000000060028
:109A60000000FA000BD8BF000044B2000004E00080
:109A700002003A00C0C1B300B118070020C2B30011
:109A8000AF18070012002000210020001000200065
:109A900087ED07000040E900614060006140600020
:109AA0004501DD00B180210091407800F0CDB30088
:109AB00000C06000024070000BF8B7000BD8BF0078
:109AC0000042B2000004E00005003A00CB62A900A9
:109AD000C962A90030C2B30099180700040037001A
:109AE000C962A800CB62A90040C2B3009418070065
:109AF0000080FA00000006000200FA0021E3A8003E
:109B000050C2B3008E18070090C0B3007B16070048
:109B1000000F780090B2290004EF07001E007800C3
:109B200044F00700A0C0B30074160700000F7800CF
:109B3000E0B22900FDEE07001E0078003DF00700AE
:109B4000B0C0B3006D160700000F780080B3290085
:109B5000F6EE07001E00780036F0070050B429002A
:109B600008EF070021E3A9000080FA0000000600CA
:109B70000000FA000BD8BF00644060000004E00061
:109B800003003A0080C1B3006D18070019003700C8
:109B900060C2B3006A1807001200200021002000F4
:109BA0001000200042ED07000040E9006140600025
:109BB000614060004301DD00B180210091407800E8
:109BC00070CFB30000C06000024070000BF8B70017
:109BD0000BD8BF00684060000004E00003003A00BA
:109BE00070C2B300561807000200370080C2B300ED
:109BF000531807000080FA00000006000000FA0079
:109C000090C2B3004E18070012002000210020006F
:109C10001000200026ED07000040E90061406000D0
:109C200061416000B180210091407800E0CFB30035
:109C300000C06000024070000BF8B7000BD8BF00F6
:109C4000614060000004E00003003A00A0C2B300DD
:109C50003B18070002003700B0C2B30038180700F5
:109C60000080FA00000006000200FA00D0C2B30033
:109C700033180700920020009100200010002000FF
:109C80000BED07000040E90000F8B700C0C2B300C8
:109C90002B18070023C2BF00614060000004E000F1
:109CA000FCFF3200491607000000370022C2BF0047
:109CB000614060000004E000FCFF320030118000D1
:109CC000004F78008560A90000C2B3009E4F1000CD
:109CD00001003200F5FF37000080FA0000000600A6
:109CE0000000FA0080B4290090EE0700C1BF2A00EE
:109CF0000000EB00A9F00700A9EF0700E0B429007D
:109D00008AEE0700E1BF2A000000EB00A3F0070085
:109D1000A3EF070000A829009AEE07004081210068
:109D200082EE070000A8290096EE07000080FA00E6
:109D3000000006000000FA00E0062A007BEE0700A3
:109D40000080FA00000006000200FA00C222A8000B
:109D5000C4000700F7FF070000003700B800070045
:109D6000BEFCB700BEDCBF000004E000B000350060
:109D7000BEDCBF000004E00002003A00EDFF070077
:109D8000F6FF3700BEDCBF00E14F500005003A008F
:109D9000B4000700EBF20700B2000700E5FF070080
:109DA000EEFF3700BEDCBF00E24F500005003A0076
:109DB000AC0007008BF60700AA000700DDFF0700D4
:109DC000E6FF3700BEDCBF00E34F500005003A005D
:109DD000A4000700C6F80700A2000700D5FF07008F
:109DE000DEFF3700BEDCBF00E44F500005003A0044
:109DF0009C00070012EC07009A000700CDFF070047
:109E0000D6FF3700BEDCBF00E54F500005003A002A
:109E1000940007009311070092000700C5FF070098
:109E2000CEFF3700BEDCBF00E64F500005003A0011
:109E30008C0007001B0607008A000700BDFF070013
:109E4000C6FF3700BEDCBF00EF4F500009003A00EC
:109E500010C0B300CAEF0700C222A90023C2BF008E
:109E6000614060000004E000FCFF32000000FE00E2
:109E7000BAFF3700BEDCBF00F04F500003003A00CD
:109E80000040EB00B2010700B4FF3700BEDCBF00AA
:109E9000F14F500003003A0010C0B300AC010700BE
:109EA000AEFF3700BEDCBF00F24F500034003A0076
:109EB0000000EB00800888000000EB00F00888003C
:109EC0000000EB00E00C8800A16C200091407800BD
:109ED00000CEB30000C060006041B300CAE6B70026
:109EE000570007000080FB00000F78001E0078007C
:109EF0000000D100610060000004E00001003200B9
:109F000010A1A8009E007800618060000004E000BD
:109F1000010032001081A800490007000080FB000A
:109F20004800DD00000F7800450007000080FB00BE
:109F30001E0F70001E007800D00C88009E00780074
:109F4000C10C880060002000E00C88003C00070085
:109F50000080FB004800DD00000F7800380007009B
:109F60000080FB001E0F70001E0078006008880053
:109F700011E1A80010C0B30081EF070077FF3700A0
:109F8000BEDCBF00F34F50000C003A000000EB00B5
:109F9000800888000000EB00E00C8800A16C200025
:109FA0009140780000CEB30000C06000CAE6B70060
:109FB00010C0B30072EF070068FF3700BEDCBF00BF
:109FC000F44F50000B003A0021E3A800C0C0B300DA
:109FD0004A150700000F780021E3A9001E00780051
:109FE0004800DE0066EF07001E00780064EF0700FF
:109FF0005AFF3700BEDCBF000080FB004500DE00DA
:10A000000080FB000000D100610060000004E0005F
:10A0100004003200BEDCBF001900070058EF070043
:10A020004EFF37000040EB0055EF07004BFF3700B5
:10A03000BEDCBF00A100070051EF070047FF37005B
:10A040000000FA0022C2BF00614060000004E0008E
:10A05000FCFF3200301180000080FB000080FA001D
:10A06000000006000000FA0000C0EB00040007003A
:10A070000040EB00910007000080FA00000006009D
:10A080000400FA00204798000040EB00004F7800E1
:10A090002E4090000080FB004400DE006100600064
:10A0A0000004E0000200320010C0B300004F78004E
:10A0B0009E40780061C06000614060004201DD00A8
:10A0C000912C200091407800B0CFB30000C0600018
:10A0D00002407000C9E2B7000040EB00004F78007A
:10A0E0002E4090000080FB004300DE006100600015
:10A0F0000004E0000200320010C0B300004F7800FE
:10A100009E40780061C060006140600000414000F6
:10A11000912C200091407800D0CFB30000C06000A7
:10A1200002407000C9E2B7000040EB00004F780029
:10A130002E4090000080FB004200DE0061006000C5
:10A140000004E0000200320010C0B300004F7800AD
:10A150009E40780061C0600061416000912C200049
:10A1600091407800E0CFB30000C060000240700072
:10A17000C9E2B7000040EB00004F78002E4090008D
:10A180000080FB000000D100610060000004E000DE
:10A190000200320010C0B300004F78009E407800EB
:10A1A00061C06000C700DD00C8C2BF000074A1002C
:10A1B00001407000C8E2B7000040EB00004F78009B
:10A1C0002E4090000080FB00610060000004E00071
:10A1D0000200320010C0B300004F78009E407800AB
:10A1E00061C06000614060004601DD00812C2000FC
:10A1F00091407800F0CBB30000C0600002407000D6
:10A20000C8E2B70050C0B30039150700AE40900057
:10A2100000CEB30000C0600020479800CBC2BF0052
:10A22000644060000004E000030032002E40900013
:10A230000044A00020479800CBC2BF0062406000ED
:10A240000004E000030032002E4090000034A00023
:10A2500020479800CBC2BF00614060000004E000CE
:10A26000030032002E4090000024A00020479800F8
:10A27000CAC2BF0001C8B300014060000004E00092
:10A28000030032002E4090000014A00020479800E8
:10A29000CAC2BF000044B2000004E0000300320064
:10A2A0002E4090000004A000204798002E4090000F
:10A2B0000080FB000080FA00000006000400FA00A5
:10A2C000204798002E4090000080FB004600DE00F2
:10A2D000610060000004E00003003200C002A90039
:10A2E000C202A80002003700C002A900C202A900F1
:10A2F0002E4090000080FB004500DE006100600001
:10A300000004E00003003200C962A800CB62A9008B
:10A3100002003700CB62A900C962A9000040EB002F
:10A32000004F78002E4090000080FB004400DE00CB
:10A33000610060000004E0000200320010C0B300C1
:10A34000004F78009E40780061C06000614060006E
:10A350004201DD00B12C200091407800B0CFB30065
:10A3600000C0600002407000CBE2B7000040EB008C
:10A37000004F78002E4090000080FB004300DE007C
:10A38000610060000004E0000200320010C0B30071
:10A39000004F78009E40780061C06000614060001E
:10A3A00000414000B12C200091407800D0CFB30094
:10A3B00000C0600002407000CBE2B7000040EB003C
:10A3C000004F78002E4090000080FB004200DE002D
:10A3D000610060000004E0000200320010C0B30021
:10A3E000004F78009E40780061C0600061416000CD
:10A3F000B12C200091407800E0CFB30000C0600095
:10A4000002407000CBE2B7000040EB00004F780044
:10A410002E4090000080FB000000D1006100600031
:10A420000004E0000200320010C0B300004F7800CA
:10A430009E40780061C06000C700DD00CAC2BF0056
:10A440000074A10001407000CAE2B7000040EB00B8
:10A45000004F78002E4090000080FB0061006000FB
:10A460000004E0000200320010C0B300004F78008A
:10A470009E40780061C06000614060004601DD00E0
:10A48000A12C200091407800F0CBB30000C0600008
:10A4900002407000CAE2B70050C0B3009414070035
:10A4A000AE40900000CEB30000C06000204798008E
:10A4B000CBC2BF00644060000004E0000300320033
:10A4C0002E4090000044A00020479800CBC2BF005F
:10A4D000624060000004E000030032002E40900063
:10A4E0000034A00020479800CBC2BF00614060004C
:10A4F0000004E000030032002E4090000024A00081
:10A5000020479800CAC2BF0001C8B30001406000E4
:10A510000004E000030032002E4090000014A00070
:10A5200020479800CAC2BF000044B2000004E00007
:10A53000030032002E4090000004A0002047980045
:10A540002E4090000080FB000080FA000000060012
:10A550000400FA0020479800AE4090000040EB0055
:10A56000EE100700104798001E4090000004E00025
:10A5700001003200C222A8001E40900000EE070039
:10A5800000003700EFED07000004E0000C0032008F
:10A59000F2ED0700004F780000C0EB009E4F100066
:10A5A000040032001E4090001E404000F4ED070001
:10A5B0000300370010C0B300F1ED07001A003700A8
:10A5C0001E4090000004E000EEFF3A0000E680002C
:10A5D0000000E00010003A000080EB0000E6880078
:10A5E000C2C2BF000080FB000000D10061406000DB
:10A5F0000004A20061406000614060000041400032
:10A60000212C200091407800D0CFB30000C0600022
:10A6100002407000C2E2B70000E680000000E900DE
:10A6200000E68800D7FF37000080FA00000006002F
:10A630000600FA000CD8BF000080FB006101B900E1
:10A640001207980023079800D00120000100200085
:10A650001E019000AE019000800F5100818F5900C3
:10A6600011013E001E009000AE009000006001004D
:10A670001D003700290037005A0037005900370005
:10A680005C0037007500370007013700060137000E
:10A6900005013700040137000301370002013700CC
:10A6A0000101370000013700FF003700FE003700CE
:10A6B000FD003700FC003700FB003700FA003700D0
:10A6C000F9003700F8003700F7003700F6003700D0
:10A6D000F50037004B0037004F003700F40037001B
:10A6E000F1003700F200370010C0B30094150700E6
:10A6F000B0DCBF000080FB000000D10061406000C2
:10A700005F010700AEFCB700AEDCBF00C11307005D
:10A71000A06429001BEC0700E5003700B0DCBF0097
:10A72000624060000004E00003003A00B0642900C9
:10A73000FEEB07000200370000652900FBEB070075
:10A7400040C0B3007E15070070C08000B113070041
:10A7500080C08000E10F500008003A0070C0800007
:10A7600080407800B0DCBF000080FB000000D1001A
:10A770006140600033010700170037005065290071
:10A78000EAEB070080C08000A213070050C0B300AE
:10A790006B1507000000EB0060E588000A00370039
:10A7A00070C0800080407800B0DCBF000080FB00FB
:10A7B0000000D100614060002201070060E58000D8
:10A7C0000000E80060E5880081C0800060E580004E
:10A7D000808F5000F2FF3E00A0642900E9EB0700E3
:10A7E000B3003700B03CA90090652900E5EB0700F5
:10A7F000AF003700B03CA800E0662900E1EB07009D
:10A80000AB0037000B58A9000B98A8000BD8A80084
:10A81000B03CA800A600370010682900D9EB07005B
:10A8200012002000110020001000200020EA070084
:10A83000AEFCB700C922A800C902A800CB02A9003B
:10A84000CB22A90011C0B30020C0B30091050700BE
:10A85000C0C0B3003A1507009500370071C08000F2
:10A86000010F78001E017800E30F51003300320021
:10A870009E017800E38F510004003E001E00780026
:10A880000000E00012003200140037009E00780043
:10A89000E68F50003A0032001E017800E60F5100AA
:10A8A00004003E009E017800E48F51002B0032002E
:10A8B0007A0037001E007800E70F50005000320089
:10A8C0009E007800E88F500070003200730037005F
:10A8D000406B2900ABEB070075003700807829003A
:10A8E000A8EB0700A500070070C08000E10F500032
:10A8F0006F003200E0782900A2EB07002200200060
:10A900002100200010002000E9E90700AEFCB7009C
:10A91000AEDCBF00E14F500003003A000040EB0006
:10A920007C0007000200370080C0B30079000700F8
:10A93000307B290093EB07005D00370011C0B300A6
:10A940000040EB00BF000700F0C0B3004F1307004A
:10A95000807B29008BEB07005500370080C080000A
:10A960008040780000C8B30080C070000040EB0059
:10A97000B4000700007C290082EB07004C00370080
:10A9800011C0B3000040EB00AE000700F0C0B30000
:10A990003E13070000C3B300AEFCB7000000EB009D
:10A9A00060E5880011003700E1CA2100914078007D
:10A9B00090C3B30080CF50000200360000C3B30044
:10A9C000AEFCB700E1CA21009140780010C0B3008E
:10A9D0009C000700AEDCBF000040E800AEFCB70002
:10A9E00060E580000000E80060E5880081C080002C
:10A9F00060E58000808F5000EBFF3E002C003700A8
:10AA000011C0B3000040EB008E000700F0C0B3009F
:10AA10001E13070010C2B300AEFCB70080C0800058
:10AA20000000E00002003A000005200080C088001D
:10AA30000000EB0060E588000F003700AEDCBF00CF
:10AA40000004E00002003D0010C2B300AEFCB700FD
:10AA5000E1CA21009140780010C0B30079000700DE
:10AA6000AEDCBF000040E800AEFCB70060E580004F
:10AA70000000E80060E5880081C0800060E580009B
:10AA8000808F5000EDFF3E0009003700B07C2900A8
:10AA90003CEB0700080007000500370070C1B30059
:10AAA000A71407000200370080C1B300A4140700F8
:10AAB0000080FA00000006001C00FA000000EB0015
:10AAC00010079800640147000E80E8008101200013
:10AAD000B0E907000000E000FAFF32000000EB00E0
:10AAE000000F7800060037001E007800E4004700E1
:10AAF000E0C0780010C0B300520007001E0FE8004D
:10AB00001E0090009E0F1000F7FF39000080FA0031
:10AB1000000006000200FA00004F78001E40780096
:10AB20000042B000804078000040EB004500070084
:10AB3000F0C0B300D512070081C0B3000040EB00A5
:10AB400040000700F0C0B300D012070011C0B300EE
:10AB50000040EB003B000700F0C0B300CB12070041
:10AB6000E1C0B3000040EB0036000700F0C0B300C6
:10AB7000C61207000080FA00000006000000FA007C
:10AB80000040EB00A2000700F0C0B300BF120700B6
:10AB900031C0B3000040EB004500070050C0B300D7
:10ABA000BA12070031C0B3000040EB0040000700BC
:10ABB00000CAB300CE12070031C0B3000040EB0062
:10ABC0003B00070000CAB300C912070021C0B30050
:10ABD0000040EB003600070000CAB300C4120700B3
:10ABE0000080FA00000006000600FA001007980036
:10ABF000030037009E40780010C0B300110007002A
:10AC00001E009000104F78001E40780040479800CA
:10AC10004E4090000004E0000200320010C0B3007B
:10AC2000404798004E4090009E0090008100E80050
:10AC3000110798000004E000EEFF3A000080FA00DF
:10AC4000000006000200FA00004F7800114798004B
:10AC50001E4090000080FB004400DE008040780031
:10AC60001E407800120007001E409000EF40600078
:10AC70001E4078000E0007000080FA000000060069
:10AC80000400FA00204798002E40900022000700A0
:10AC90004400DD00004F78002E4090001E000700A9
:10ACA0001E4F70001E80FB000080FA0000000600AE
:10ACB0000200FA00004F78001147980010C0B3005E
:10ACC0009E4F100004003A001E40900001C8B300DF
:10ACD00001407000104798001E4090004C00070093
:10ACE0009E40900000C2B30000C070001047980062
:10ACF0001E409000460007009E409000F0CDB3003B
:10AD000000C06000104798001E40900040000700FF
:10AD10000080FA00000006000400FA0020479800B6
:10AD20000040EB00104798000040EB00004F780017
:10AD30009E40900000C4B30000C07000104798000F
:10AD40002E409000E14F500004003A001E40900059
:10AD500001C8B30001407000104798001E409000E9
:10AD6000F040B300104798001E40900028000700F4
:10AD70009E40900000C2B30000C0700010479800D1
:10AD80001E409000220007000C000700004F7800D2
:10AD9000F0C0B3001E4F60009E409000F0CDB300A5
:10ADA00000C06000104798001E4090001800070087
:10ADB0001E80FB000080FA00000006000400FA007C
:10ADC0006F04070010C4B300D8040700380507005B
:10ADD000E14F500004003A00210007000000EB00A2
:10ADE000100798000700370001050700004F7800A2
:10ADF00010C0B3003F050700740407001E80FB006D
:10AE0000100798001E0090000080FA000000060065
:10AE10000200FA00004F78005904070000C4B30094
:10AE2000C204070022050700E14F500002003A006B
:10AE30000B000700080037001E407800BB04070025
:10AE40001B050700E14F500002003A000400070014
:10AE5000010037005D0407000080FA0000000600D2
:10AE60000000FA00807D290046EA07000080FA0011
:10AE7000000006000400FA000CD8BF000080FB00B0
:10AE8000100798001E009000F90F500017003200C4
:10AE90001E009000F90F50000A003C001E009000B8
:10AEA000E10F5000360032001E009000E50F500008
:10AEB0004B0032001E0090000000E0001100320044
:10AEC000680037001E009000FB0F50006700320042
:10AED0001E009000FB0F5000060035001E00900081
:10AEE000FD0F5000610032005E0037000BD8A80053
:10AEF0005E003700970007000040EB00901307004A
:10AF00005A00370080C08000E10F500005003A0071
:10AF100010C0B3008A13070029010700550007007D
:10AF20001400370020C0B3008513070080C08000E4
:10AF3000B811070030C0B300811307000000EB0018
:10AF4000B0E48800070037001D0107004900070032
:10AF500000C2B3008AEB0700B0E480000000E80004
:10AF6000B0E4880081C08000B0E48000808F500091
:10AF7000F5FF3E00C0F1290002EA07003B00370060
:10AF800040C0B3006E13070070C08000A11107001D
:10AF900070C080004801070098FCB70098DCBF0033
:10AFA0000004E00003003A0060C0B300641307002F
:10AFB0000800370098DCBF00E14F500003003A0062
:10AFC00070C0B3005E13070002003700D0F1290003
:10AFD000D6E90700C0F12900EAE90700230037009D
:10AFE00070C08000000F78001E0078000000E000B4
:10AFF000040032001E007800E10F5000040032000F
:10B0000015003700A0F22900DEE90700170037001D
:10B0100010F52900DBE90700E90007000004E00063
:10B0200004003A009BDCBF007A11070000C2B300A5
:10B0300053EB070022C2BF00614060000004E00043
:10B04000F5FF32003011800098FCB700C0F12900F4
:10B05000CCE907000500370070C1B30038130700C2
:10B060000200370080C1B300351307000080FA00EA
:10B07000000006000400FA00004F78001E80FB006C
:10B08000100798009E009000E28F50001D003200D3
:10B090001E009000E20F500007003C009E00900050
:10B0A0000100E0000F0032001E009000E10F500090
:10B0B00011003200230037009E009000E48F500002
:10B0C0001A0032001E009000E40F500012003500FC
:10B0D000F00F20009E009000808F5000160032007C
:10B0E000180037009BDCBF004A11070000C2B30004
:10B0F00023EB070015003700E0F629008BE9070075
:10B10000120037009BDCBF0042110700F0F7290056
:10B1100086E907000D0037009BDCBF003D110700EA
:10B12000E0F8290081E9070008003700D0F1290084
:10B130007EE9070005003700E0F929007BE90700F8
:10B140000200370040FA290078E907000080FA0081
:10B15000000006000000FA00C922A800C902A900E8
:10B16000CB02A900CB22A9000080FA000000060053
:10B170000400FA000040EB002F0107000004E0008B
:10B180000300320020002000100798000E00370056
:10B19000CBC2BF000080FB000000D1006140600016
:10B1A000004F780010C0B300230107000004E00046
:10B1B0000300320020002000100798000200370032
:10B1C0001E80FB00100798001E0090000080FA000F
:10B1D000000006000600FA000040EB00204798003F
:10B1E0000040EB0010479800CBC2BF000080FB007E
:10B1F0000000D1006140600061416000A1C92100F0
:10B2000091407800E0CFB30000C0600002407000C1
:10B210009AFCB7009ADCBF00614060000004E000C7
:10B220000300320010002000200798006100370062
:10B2300010C0B300000107000004E000030032006A
:10B2400041002000210798005A0037000040EB0021
:10B2500030479800190037001E4090000080FB0026
:10B260000000D10010479800C1FF0700004F780090
:10B2700020C0B3009E4F100003003A0041002000A0
:10B28000210798004B00370010C0B3009E4F1000FC
:10B2900007003A009E40900000C8B30000C0400084
:10B2A000104798002E4090000004A200204798000C
:10B2B0003E4090000040E800304798003E4090003B
:10B2C000E74F5000E4FF36001E4090009BFCB700A3
:10B2D000A7FF0700004F780021C0B3009ECF1000E9
:10B2E00003003A004000200020079800310037009A
:10B2F0009E40780061C0600061416000C1C92100CA
:10B3000091407800E0CFB30000C0600002407000C0
:10B310009CFCB7009CDCBF00614060008080FB00AB
:10B320002E4090000080FB00808F500004003A0007
:10B330009C5CA80020002000200798001D0037001A
:10B340009C5CA9008AFF0700004F780021C0B30071
:10B350009ECF100003003A00400020002007980014
:10B36000140037009E40780061C0600061406000BA
:10B3700000414000C1C9210091407800D0CFB30006
:10B3800000C06000024070009CFCB700C902A90028
:10B390009CDCBF00624060000004E00003003A0053
:10B3A0003000200020079800020037008000EB00EA
:10B3B000210798002E0090000080FA00000006008F
:10B3C0000200FA0000C0EB00004F7800C922A8007C
:10B3D000C902A8000040EB00104798001000370099
:10B3E000CBC2BF00614060000004E00007003A00EB
:10B3F00078FF0700004F78001E04E0000B003200C9
:10B4000040C0B3009E4F10000800320050C0B3008F
:10B41000B71007001E4090000040E8001047980059
:10B420001E409000E14F4000EDFF3A00C902A90024
:10B430001E80FB000080FA00000006000400FA00F5
:10B44000004F780010C0B3007B0007000004E0004C
:10B45000030032002000200010079800130037007E
:10B460009E40780061C06000614060000041400083
:10B47000912C200091407800D0CFB30000C0600034
:10B4800002407000C9E2B7000040EB006A0007000C
:10B490000004E000030032002000200010079800A4
:10B4A000020037008000EB00110798001E0090009A
:10B4B0000080FA00000006000800FA0040479800EB
:10B4C0000040EB0020479800C902A900CB02A90068
:10B4D000C0C3B30086100700CB22A900C922A9006F
:10B4E000C902A80010C0B300811007000040EB00A3
:10B4F000510007000004E00003003200400020007B
:10B5000030079800490037000000EB00000F78007A
:10B510001C0037004E4090000080FB00610060007E
:10B520000004E0000B00320010C0B300C3FF0700AE
:10B530000004E000030032004000200030079800C3
:10B540003A0037002E4090000004A20020479800E7
:10B55000070037000040EB00B8FF07000004E000E0
:10B560000300320040002000300798002F00370011
:10B570004E4090000080FB000000D1004047980042
:10B580001E0FE800700020009E0F1000E1FF360043
:10B590002E4090000004A200204798002E4090000A
:10B5A000A6FF07000004E000030032004000200076
:10B5B000300798001D003700C922A800CB22A9003F
:10B5C00010C0B3001C0007000004E00003003200BC
:10B5D000400020003007980014003700E4FE070008
:10B5E000E24F500003003A0040002000300798006E
:10B5F0000E003700DEFE07000080FB00000F780021
:10B60000200020009E0F100003003A0040002000A0
:10B610003007980005003700C902A900CB02A90035
:10B620001E0078000080FB00300798003E0090006C
:10B630000080FA00000006000600FA00204798008B
:10B640000080EB00000F7800CBC2BF0061406000BB
:10B650008080FB002E4090000080FB00808F500017
:10B6600003003A000000EB002007980005003700B7
:10B670001E0FE9001E00E000F3FF3A00100020005A
:10B68000200798002E0090000080FA0000000600BD
:10B690000000FA0000082A0024E807000080FA00F1
:10B6A000000006000A00FA00008020003007980021
:10B6B0001000200050E68800F5FF0700000037006A
:10B6C000A6E90700104798001E4090000080FB008C
:10B6D000400798004E009000E30F50002000320019
:10B6E000CE009000E38F50000A003C004E00900016
:10B6F000E10F500057003200CE009000E18F500063
:10B7000059003C004E0090000000E000CD003200E7
:10B71000C1003700CE009000E68F50000E003200CE
:10B720004E009000E60F500004003C00CE00900058
:10B73000E58F500086003200B70037004E009000C1
:10B74000E70F50005B003200CE009000E88F500001
:10B750004D003200B0003700CDFF0700D8FF3700A2
:10B76000BE00900030C0B300804878003E009000DA
:10B770008000E80080C0B3008048780021E3A80082
:10B78000C0C0B3005D0F0700200798003E00900086
:10B790008080E8002E0090004800DE00804878009D
:10B7A0003E009000E30040002E00900080487800AA
:10B7B000B0C0B300510F0700200798003E00900072
:10B7C000E40040002E0090004800DE008048780031
:10B7D0003E009000E50040002E0090008048780078
:10B7E000A0C0B300450F0700200798003E0090005E
:10B7F000E60040002E0090004800DE0080487800FF
:10B800003E009000E70040002E0090008048780045
:10B8100090C0B300390F0700200798003E00900049
:10B82000E80040002E0090004800DE0080487800CC
:10B830003E009000E90040002E0090008048780013
:10B8400021E3A900A10020003E009000A90007000C
:10B850009BFF370041E90700104798001E40900009
:10B860007A00070096FF37003CE907001047980070
:10B870003AE90700004F78009E4078001E40900093
:10B88000AD0007008EFF370034E90700104798002D
:10B8900032E90700004F78001E4090000080FB0056
:10B8A000C800DD001E80FB000080700050E68800AC
:10B8B00083FF370029E90700104798001E409000D9
:10B8C0000080FB00200798001E409000E14F5000D0
:10B8D00003003A0030C0B30033E90700020037002C
:10B8E00020C2B30030E907001CE9070010479800A8
:10B8F0001AE90700004F78009E409000A0CAB300EC
:10B9000080CF500003003A0050C5B3009E4F100096
:10B91000040032000000EB002007980020C2B300B2
:10B9200021E90700BE00900070C0B3008048780095
:10B930003E0090008000E8002E00900080487800D3
:10B94000210020003E0090006A0007005CFF3700E5
:10B9500002E907001047980000E90700004F78004F
:10B960008560A9001E4090000080FB00C800DD003B
:10B970001E80FB0000807000100798001E009000E1
:10B98000670040004300DE0020079800BE009000E2
:10B9900050C0B300804878003E0090000000E800EE
:10B9A0009E409000014878003E0090000080E80032
:10B9B0001E487800310020003E0090004D00070036
:10B9C0000080200000E088002E0090000000400071
:10B9D00010E088000000EB0020E088004003210018
:10B9E00030E088000000EB0040E088000000EB0041
:10B9F00050E088009560A80050E6800031E08000AB
:10BA000004E08000800178001E01900004007800AE
:10BA1000960007002AFF3700BE0090000040EB00B0
:10BA2000804878003E0090008000E8000040EB0075
:10BA300080487800110020003E0090002D00070093
:10BA40001FFF37000080FA00000006000200FA0025
:10BA5000004F7800CAC2A900CB22A900CB02A900DE
:10BA6000CB42A900CA02A90020C0B3009E4F10001B
:10BA700006003A00CAC2A800CB02A800CB22A80048
:10BA8000CB42A800CA02A80005003700CAC2A9001C
:10BA9000CB02A900CB22A900CB42A900CA02A9006F
:10BAA00010C0B3009E4F10000300320020C0B3004E
:10BAB0009E4F100007003A00C8C2A900C922A90081
:10BAC000C902A900C942A900C802A900C8E2A80089
:10BAD00006003700C8C2A800C922A800C902A800F1
:10BAE000C942A800C802A800C8E2A8000080FA0065
:10BAF000000006000600FA001007980021079800D1
:10BB00000000EB00000F7800060037009E00780070
:10BB10001E009000008040001040780098E8070068
:10BB20001E0FE8002E0090009E0F1000F7FF390056
:10BB30000080FA00000006000400FA00004F7800C0
:10BB4000114798001E80FB00100798001E0090000F
:10BB5000E40F50002F0032001E009000E40F500050
:10BB600007003C001E009000E10F50000B00320067
:10BB70001E009000E20F5000140032003900370020
:10BB80001E009000E80F50002C0032001E009000B4
:10BB9000F00F50001600320032003700C022A9001A
:10BBA0001E40900061406000614060000041400024
:10BBB000212C200091407800D0CFB30000C060005D
:10BBC00002407000C2E2B700260037001E4090001D
:10BBD0000004E00003003200C002A900C202A80075
:10BBE00020003700C002A900C202A9001D003700D2
:10BBF0001E4090000004E00003003200C962A8006B
:10BC0000CB62A90017003700CB62A900C962A90066
:10BC1000140037001E4090006140600061416000E8
:10BC2000A12C200091407800E0CFB30000C060005C
:10BC300002407000CAE2B7000A0037001E409000C0
:10BC400061406000614060004201DD00B12C2000D5
:10BC500091407800B0CFB30000C060000240700097
:10BC6000CBE2B7000080FA00000006001200FA00E4
:10BC7000500798006107980072079800030F98001A
:10BC80000040EB00004F98000000EB0030079800E8
:10BC9000730037003E0090004300DE00200798004C
:10BCA0003E00900067406000204798002E00900002
:10BCB000000040008000E80020E08000808F5000FD
:10BCC000FAFF31002E009000000040008000780054
:10BCD0005E00900000804000104078008080FB00F3
:10BCE0002E4090000080FB000088DE0061006000B4
:10BCF0000004E00002003200CB22A800010037005F
:10BD0000CB22A9002E0090000000400080007800A7
:10BD10005E009000008040000000E80010407800C5
:10BD20008080FB002E4090000080FB000088DE0039
:10BD3000610060000004E00002003200CAC2A800F6
:10BD400001003700CAC2A900CB02A9000000EB0025
:10BD5000000F7800010037001E0FE8000E08900069
:10BD60009E0F1000FCFF3900CB02A800CAC2BF0022
:10BD70000080FB004700DE008080FB005016800042
:10BD8000008060000000E0000F003200AE00900074
:10BD90006E00900080814000AE0090006E00900028
:10BDA0000080400010407800004178002E40900054
:10BDB0008080FB00100020000100DD0000407100C9
:10BDC0008049780012003700AE0090006E009000AD
:10BDD00000824000AE0090006E00900000804000A5
:10BDE00010407800804178002E4090008080FB0059
:10BDF000100020000100DD000041780002407800C2
:10BE00000080EA008180EA0000C06100004A7800FA
:10BE100010C0B300004F98002E409000E74F500034
:10BE20000C003A000040EB00004F980050E080000A
:10BE30000000E80050E0880051E0800040E0800011
:10BE40008080500000042000808F500001003600E8
:10BE5000DBE707003E0090000000E8003007980094
:10BE6000BE0090007E009000808F500089FF390056
:10BE70000E489000E14F500003003A0050E080006F
:10BE80000000E80050E08800CDE707000080FA00DD
:10BE9000000006000400FA00004F780011479800E7
:10BEA0001E4078008CFCB70030C0B3009E4F1000DD
:10BEB00005003A000020200070E4880000082000FF
:10BEC00080E48800040037000020200070E488002F
:10BED0000020200080E488001E4090000080FB00CD
:10BEE000100798001E009000E10F50000E00320075
:10BEF0001E009000E20F5000120032001E00900061
:10BF00000000E000010032001500370040C1B3001E
:10BF100092FCB70040C6B30093FCB70020C3B30047
:10BF200094FCB7001400370020C0B30092FCB700A7
:10BF3000A0C0B30093FCB70050C0B30094FCB7009E
:10BF40000D00370010C0B30092FCB70050C0B30022
:10BF500093FCB70020C0B30094FCB7000600370084
:10BF60000040EB0092FCB7000040EB0093FCB700F0
:10BF70000040EB0094FCB7000080FA0000000600CF
:10BF80000000FA0031C92100914078000030200003
:10BF90001D01070031C921009140780000202000D8
:10BFA0003201070031C921009140780000102000C3
:10BFB0002E01070031C921009140780000202000A7
:10BFC000110107000080FA00000006000000FA00DE
:10BFD00031C9210091407800003020002301070082
:10BFE00031C92100914078000010200006010700AF
:10BFF00031C9210091407800002020000201070093
:10C000000080FA00000006000800FA00604798006F
:10C010000040EB00004F78000BD8BF006840600084
:10C020000004E00003003A0000C8B3003047980065
:10C030000200370010C0B300304798006E409000F7
:10C04000204798000040EB0040479800310037003F
:10C0500022C9210012417800AE4090003E4090007D
:10C0600000C06000012020001501070031C9210037
:10C070009140780000102000E30007000008200035
:10C080003C0107001047980031C921009140780019
:10C0900000102000F50007000BD8BF0068406000CA
:10C0A0000004E0000B003A002E40900000404000E9
:10C0B000204798001E40780000404000004F780064
:10C0C0001E4090000004E0000F0032001E4FE80008
:10C0D0000D0037002E40900000404000204798009F
:10C0E0001E80FB000000D100004F78001E40900031
:10C0F0000004E000040032001E40780001C8B300D4
:10C1000001404000004F78004E4090000040E800A1
:10C11000404798004E409000E74F5000CCFF36005B
:10C120001E80FB000080FA00000006000600FA00F6
:10C13000404798000BD8BF00684060000004E00052
:10C1400003003A0000C8B30010479800020037000F
:10C1500010C0B300104798004E409000004F780088
:10C160000040EB00204798001C00370022C9210046
:10C17000124178001E4090001E4060000120200007
:10C18000CF00070031C92100914078000010200045
:10C190009D00070031C92100914078000010200067
:10C1A000B20007000BD8BF00684060000004E00048
:10C1B00004003A001E40780000404000004F780024
:10C1C000030037001E80FB000000D100004F780004
:10C1D0002E4090000040E800204798002E4090003C
:10C1E000E74F5000E1FF36000080FA000000060033
:10C1F0000400FA000040EB00004F7800002020000F
:10C20000DC0007000040EB002047980022003700C8
:10C2100031C9210091407800001020007A00070009
:10C2200000202000D30007001047980031C92100EA
:10C2300091407800001020008C0007000BD8BF0050
:10C24000684060000004E00008003A001E407800EA
:10C2500000404000004F78001E4090000004E000C5
:10C260000A0032001E4FE800080037001E80FB0065
:10C270000000D100004F78001E4090000004E00054
:10C280000200320000C8B3001E4F70002E40900024
:10C290000040E800204798002E409000E74F5000F3
:10C2A000DBFF36001E80FB000080FA000000060065
:10C2B0000200FA0080E48000AE00070031C92100CE
:10C2C00091407800001020004F00070080E48000BB
:10C2D000A8000700004F780031C921009140780084
:10C2E00000102000610007001E80FB000080FA00A3
:10C2F000000006000200FA00004F780022C9210069
:10C300001241780071E480001E4078006C00070044
:10C3100031C9210091407800001020003A00070048
:10C3200031C9210091407800001020004F00070023
:10C330000080FA00000006000400FA002047980080
:10C340000040EB00004F78000900370031C92100A0
:10C3500091407800001020002B00070031C9210017
:10C360009140780000102000400007001E4FE800B8
:10C370002E4090009E4F1000F4FF39000080FA001C
:10C38000000006000200FA00004F780022C92100D8
:10C390001241780071E480001E40780048000700D8
:10C3A0000080FA00000006000200FA00004F78004A
:10C3B00022C9210012417800011020001E4078009F
:10C3C0003F0007000080FA00000006000200FA00AB
:10C3D000004F780022C9210012417800010420009A
:10C3E0001E407800360007000080FA0000000600BA
:10C3F0000000FA0080E480005E0007000080FB007F
:10C400000080FA00000006000400FA00000F780027
:10C41000214798000BD8BF000044B2000004E000A0
:10C420000B003A00601680001E0070006016880045
:10C430001E0078000080EA008180EA008000780019
:10C44000401680000080600040168800030037001E
:10C45000401680001E007000401688002E4090009C
:10C46000A30C07000080FA00000006000400FA0098
:10C47000000F7800214798001E0078000080EA0035
:10C480008180EA00800078006016800000806000F3
:10C49000601688001E0078000080EA008180EA00B3
:10C4A0008000780040168000008060004016880000
:10C4B0002E4090008E0C07000080FA00000006005D
:10C4C0000600FA00004F78001107980042479800D4
:10C4D0001E04E0000F003A001E0090000080EA00F9
:10C4E0008180EA0080007800601680000080600093
:10C4F000601688001E0090000080EA008180EA003B
:10C50000800078004016800000806000401688009F
:10C51000140037000BD8BF000044B2000004E00054
:10C520000C003A00611680001E0090000080700030
:10C53000601688001E0090000080EA008180EA00FA
:10C54000800078004016800000806000401688005F
:10C5500004003700401680009E009000010070002B
:10C56000401688004E409000610C07000080FA00E1
:10C57000000006000400FA00000F7800401680005A
:10C580001E0070004016880000000000000000003F
:10C5900000000000501680001E0060000000E00057
:10C5A000030032001000200010079800020037003E
:10C5B0000000EB00100798001E0090000080FA00B9
:10C5C000000006000600FA00000F7800110798002E
:10C5D00020C080000000E00003003A00B0C1B300BA
:10C5E000D70D0700A20037000000EB0020E588000F
:10C5F0009900370020E58000800078001E00900040
:10C600000080400010407800C30007009FFCB70086
:10C610009FDCBF00E14F5000030032009FDCBF00F1
:10C62000E54F500014003A009FDCBF00E54F50007A
:10C630000C003A0020E580000000E80020E58800BA
:10C6400020E580009E0F500006003A009EDCBF00EF
:10C650000040E8009EFCB70020E580000000E900F3
:10C6600020E588001E01900041CA21001E007800CC
:10C670001CE3070010E588001E01900041CA21005C
:10C680001E0078007C00070000E588009FDCBF00EA
:10C69000E54F500014003A0020E580000000E8005B
:10C6A00020E5880020E580009E0F50000800320041
:10C6B00020E58000800078001E009000008040008F
:10C6C0009040780090C2B30080CF50000600320046
:10C6D00020E580000000E90020E588009EDCBF0026
:10C6E0000040E8009EFCB7009EDCBF000004E000B4
:10C6F0000500320090C1B300910D07000040EB002F
:10C700009EFCB7005A0037009FDCBF000080FB0092
:10C71000200798002E009000F30F500030003200E8
:10C720002E009000F30F500011003C002E009000EE
:10C73000F00F50001D0032002E009000F00F50004E
:10C7400004003C002E009000EF0F50001500320056
:10C75000370037002E009000F10F50001500320016
:10C760002E009000F20F500014003200300037000D
:10C770002E009000F50F5000250032002E00900092
:10C78000F50F50001C0035002E009000F60F5000F1
:10C79000250032002E009000F80F50002B003200D0
:10C7A00023003700F006070028003700FC060700CA
:10C7B00026003700080707002400370020032A005E
:10C7C000DAE3070000E58000920B070090032A00DF
:10C7D000ECE3070000E58000C50B07001B003700F5
:10C7E000C002A900C202A80050C1B300540D070046
:10C7F0000BF8A80015003700C002A900C202A9006A
:10C8000060C1B3004E0D07000BF8A9000F00370000
:10C81000C0032A00C5E30700450B0700C0042A0037
:10C82000D8E3070009003700490B0700070037006D
:10C830009FDCBF000CF8B70010E5800070C08800D6
:10C8400000E5800080C08800AA0C070020E5800079
:10C850000000E80020E5880020E580009E0F5000E1
:10C8600064FF3900D0C1B3000CF8B700A10C070079
:10C870000080FA00000006000A00FA001007980085
:10C8800021079800320798000000EB00000F7800A5
:10C890002E009000100078008000E8001E0090003C
:10C8A000808F5000170031002E009000100078009B
:10C8B000800078003E009000008040000000E8000A
:10C8C00090407800A0C3B30080CF50000D003A0024
:10C8D0002E009000100078008080E8002E0090006C
:10C8E000010878003E019000AE0090001E0090000C
:10C8F0007CE20700000F78001E00780040079800D7
:10C900000200370010002000400798004E00900001
:10C910000080FA00000006000800FA00004F7800CE
:10C92000F0C2B3009E4F10000600360090C3B30063
:10C930009E4F100003003E001000200010079800DA
:10C94000D00037001E80FB006101B90060FF2F009E
:10C95000F1FF2F0002014000838148002207980068
:10C960003307980030072000010020002E019000BE
:10C97000BE019000800F5100818F5900BF003E0022
:10C980002E009000BE00900000600100A90037005A
:10C99000BA003700B9003700A9003700B7003700E8
:10C9A000B6003700B5003700B4003700B3003700D9
:10C9B000B2003700B1003700B0003700AF003700D9
:10C9C000AE003700AD003700AC003700AB003700D9
:10C9D000AA003700A9003700A8003700A7003700D9
:10C9E000A60037008D00370077003700A30037001E
:10C9F000A2003700A1003700A00037006000370018
:10CA00009E003700610037009C0037009B00370014
:10CA10009A003700840037007D0037006D00370032
:10CA20006F003700950037009400370093003700FF
:10CA30009200370091003700900037008F003700D8
:10CA40008E0037008D0037008C0037008B003700D8
:10CA50008A003700890037008800370087003700D8
:10CA600086003700430037003C0037008300370062
:10CA7000820037007B003700800037007F003700DE
:10CA80007E0037007D0037007C0037007B003700D8
:10CA90007A003700790037007800370077003700D8
:10CAA0007600370075003700740037004300370008
:10CAB0007200370071003700700037006F003700D8
:10CAC000620037006D0037006C0037006B003700E4
:10CAD0003400370045003700350037004600370086
:10CAE00048003700650037001F003700630037003B
:10CAF000620037005E003700600037005F003700DB
:10CB00005E0037005D0037005C0037005B003700D7
:10CB10005A003700590037005800370057003700D7
:10CB20005600370055003700540037002300370007
:10CB30005200370051003700500037004F003700D7
:10CB4000450037004D0037004C0037004B003700E0
:10CB5000110037004900370015003700F1002000B0
:10CB600011079800470037000201200012079800C3
:10CB700044003700130120001307980041003700DC
:10CB800020012000100798003E00370051002000CF
:10CB9000110798003B003700320020001207980070
:10CBA00038003700230020001307980035003700B5
:10CBB0004000200010079800320037008000EB0092
:10CBC000110798002F00370062002000120798001C
:10CBD0002C0037007300200013079800290037004D
:10CBE000900020001007980026003700A1002000C8
:10CBF00011079800230037008200200012079800D8
:10CC000020003700C3002000130798001D003700E4
:10CC1000B0002000100798001A00370081012000A2
:10CC200011079800170037008201200012079800B2
:10CC3000140037008301200013079800110037000B
:10CC400080012000100798000E00370031012000FD
:10CC5000110798000B0037004201200012079800CE
:10CC60000800370063012000130798000500370013
:10CC7000500120001007980002003700C101200079
:10CC8000110798001E0090000080FA0000000600C6
:10CC9000C61C0000020000000200000000000000AE
:10CCA000000800001410000000000000B21C00008A
:10CCB0000400000000000000A61C000006000000A8
:10CCC00000000000561C00000C00000002000000E4
:10CCD00000181C001D0018001C1D0300081018007F
:10CCE0006E1C00000A00000000000000361C00005E
:10CCF0001200000002000000143404000D8206003F
:10CD00004003A00001CF00006700440000220000A3
:10CD1000B61C000004000000020000009D250D006C
:10CD200000000000481C00000E0000000000000091
:10CD3000781C00000A00000000000000BA1C00007F
:10CD40000400000000000000581B000070000000FC
:10CD500000000000A2190000020100000200000013
:10CD6000F0005E00BCE261003FDD8300C29C7E00FB
:10CD700020A3FD001F419D00C3217F00FCA24000B5
:10CD80001E5F0100E3BD3E006082DC00237D9F004A
:10CD9000C1421C00FEA0E100BF5D030080DE3C003C
:10CDA00062BEE000025CDF0081633D007C22C000C7
:10CDB0009E1D4300A1FF460018FAA40027799B009E
:10CDC000C584DA003866E500BB590700DB856700DB
:10CDD00039BAE4000658190047A5FB007826C400BC
:10CDE0009A653B00D98704005AB8E600A7F91B00F2
:10CDF00045C698007A24F800A6441A0099C7250071
:10CE00007B3A640086D85B0005E7B9008CD230001D
:10CE10006EEDB300510F4E0010F2AC002F71930075
:10CE2000CD114F00ADF370002ECC9200D38D6F006A
:10CE300031B2EC000E50AF00F1134D00CE907200F5
:10CE40002C6D3300D18F0C0052B0EE00326C8E008E
:10CE5000D0530D00EFB1F000AE4C120091CF2D0079
:10CE600073CA94007628AB00F51749000856B40041
:10CE7000EA693700D58B570009EBB50036688A00A0
:10CE8000D495CB002977F400AA481600E9B75500DD
:10CE90000B88D600346A2B007597C9004A14F60037
:10CEA000A8742A00C89615004BA9F700B6E80A0036
:10CEB00054D789006B350000961C00000800000064
:10CEC00000000000821C00000A00000000000000BA
:10CED000221C00001400000002000000B49FB800F3
:10CEE0009FBF9F00C49FC8009FCC9F00D19FDA00C6
:10CEF0009FE39F00EF9F0000141800008E010000C8
:10CF00000200000020205F00202020005F20200081
:10CF1000202020005F2020002020200020205F0013
:10CF20005F5F5F00202020005F2020005F5F200007
:10CF300020202000205F5F0020205F005F20200075
:10CF400055205F005F5F5F005F207500200D0A00C5
:10CF5000207C27007C207C00277C550020202F008F
:10CF6000225C200020755500202F22005F5F5F00AB
:10CF70007C207C00227C2F00202F200020205500C8
:10CF80007C2720005C2F2000277C75005C7C200023
:10CF90005F5F5F00227C2F00200D0A002F7C2000A5
:10CFA0007C5F7C00207C5C005C2F20005F205C00AC
:10CFB0002F205C007C207C002075200020207C003D
:10CFC000202720002F20200020205C007C207C00D7
:10CFD0005C2F7C00207C2F00207C2000205F7C00C8
:10CFE00022202000200D0A00557C2000205F200018
:10CFF000207C75002F205F005F5F20005C202000F8
:10D000007C207C002F5F5F00552F7C00202E2000AD
:10D010005C5C7500202020007C207C0020207C00AF
:10D02000207C2000207C20007C5F5F005F202000AF
:10D03000200D0A00207C5F007C207C005F7C2F009C
:10D040005F2F200020205C005F5C2000205C5F00E0
:10D050005F5F5F007C207C005F7C5C005F5C200089
:10D06000202020007C5F7C0020207C005F7C200052
:10D07000207C5F005F5F5F005F7C2000200D0A0066
:10D08000202F2F00202020005C5C20005C5C200012
:10D09000202020003E3E20005F2F2F00205C5C00FF
:10D0A0002C2D2C003E3E20005C5C2C002D2E3C00E4
:10D0B0003C2C2D002C2C2D002E202000203C3C0050
:10D0C000202020003E3E2000200D0A00285F220084
:10D0D00029202800225F29005F5F290020202800E6
:10D0E0005F5F29005F5F2900285F5F00295C2E00D9
:10D0F0002920200020285F002F202000282E2F002C
:10D1000020205C002E292000285F5F0029202800B5
:10D110005F5F2900200000009E1C00000800000046
:10D1200000000000F01B00001C00000000000000D8
:10D13000A41A0000B400000002000000CC85D40056
:10D1400085DB8500E185EB0085F38500FA85FE002F
:10D150008503860013862200862F86003D865D00AB
:10D16000866886007C868F00869E8600A986B4002D
:10D1700086C58600D686EA0086FF8600268746009A
:10D18000876887009B87B50087DA8700ED873F00B7
:10D19000884F88007488890088AD8800C588DC00C5
:10D1A00088EF88000E892C00894B890081899A00BC
:10D1B00089B68900E98966008A9E8A00E48A180097
:10D1C0008B568B007B8B9A008BBA8B00DF8BE50034
:10D1D0008BEC8B00FA8B05008C168C002C8C440099
:10D1E0008C5D8C007E8C93008C9F8C00B28CCA006E
:10D1F0008CD68C00DE8CEB008CF28C00138D320010
:10D200008D628D007A8D86008D978D00A98DC1006D
:10D210008DD68D00EF8DFB008D238E00458E58003E
:10D220008E658E00728E8E008E9B8E00C81B000055
:10D230002800000002000000143404000D820600E3
:10D240004003A00001CF000067004400002200005E
:10D250007F00140034040D008206400003A001008A
:10D26000CF007F00006700004400220000000000A3
:10D27000621C00000C00000000000000AC1C00005C
:10D280000600000000000000C81C000002000000B2
:10D29000000000008C1C00000A00000000000000DC
:10D2A000BE1C00000400000000000000C21C0000C2
:10D2B00004000000000000000C1C0000160000002C
:10D2C00000000000CA1C0000020000000000000076
:10D2D000000000000600FA000CD8BF000080FB0030
:10D2E0006101B9001207980023079800D0012000BF
:10D2F000010020001E019000AE019000800F51003F
:10D30000818F5900D1003E001E009000AE009000B9
:10D31000006001001D0037003D0037005B00370052
:10D320005A0037005F003700B30037006300370052
:10D33000690037006F00370075003700790037004B
:10D340007D00370081003700C0003700BF00370084
:10D35000BE003700BD003700BC003700BB003700FF
:10D36000BA003700B9003700B8003700B7003700FF
:10D37000B6003700B500370079003700930037005A
:10D38000B4003700B1003700B200370080C0800021
:10D39000E10F500007003A0010C0B300680A070010
:10D3A00093FB0700B4FCB700B4DCBF00990807008A
:10D3B0001400370020C0B300610A070080C080005D
:10D3C0009408070030C0B3005D0A07000000EB00BE
:10D3D00090E588000700370085FB07008D080700EF
:10D3E00000C2B30066E2070090E580000000E8009C
:10D3F00090E5880081C0800090E58000808F50001B
:10D40000F5FF3E00E07E2900DEE0070091003700D6
:10D4100040C0B3004A0A070070C080007D080700C2
:10D4200080C08000E10F500003003A0070C080000F
:10D430003EFB070012003700F07E2900BBE007002A
:10D4400080C080007308070050C0B3003C0A07008A
:10D450000000EB0090E588000500370070C08000F8
:10D4600032FB070090E580000000E80090E58800AE
:10D4700081C0800090E58000808F5000F7FF3E0063
:10D48000E07E2900BFE0070072003700BCFA070009
:10D49000307F2900A5E0070080C0B300280A0700FC
:10D4A0006C003700C9FA0700B07F29009FE0070031
:10D4B00090C0B300220A070066003700D0C0B30056
:10D4C0001F0A07007AFB070091E00700F0C0B300D5
:10D4D0001B0A07005F003700E0C0B300180A07000E
:10D4E000C3FB07008AE00700F0C0B300140A07007E
:10D4F0005800370080C080004608070000C1B30014
:10D500000F0A070080C080008BFB07005100370026
:10D5100010C1B3000A0A070010C0B300A2FB070045
:10D520004C00370020C1B300050A07000040EB00A3
:10D530009DFB07004700370030C1B300000A070019
:10D5400010C0B3008FFB07004200370040C1B3009A
:10D55000FB0907000040EB008AFB07003D00370095
:10D560000B58A8000B98A80010C3B300F4090700DB
:10D57000120020004100200010002000CCDE070037
:10D580000040E9000AF8B700E0C1B300EC09070069
:10D59000120020002100200010002000C4DE07003F
:10D5A0000040EA0061406000614060004601DD002B
:10D5B000B180210091407800F0CBB30000C0600042
:10D5C000024070000BF8B70022003700CB02A90020
:10D5D000CB22A900C922A800C902A900A18021006C
:10D5E0009140780020C0B3002AFA07000040EB0009
:10D5F000D30907001700370071C08000010F7800C1
:10D600001E017800E10F51000A0032009E017800EF
:10D61000E18F5100040039001E007800E20F500035
:10D620000500320006003700208029003FE0070097
:10D63000080037000900070019000700050037003F
:10D6400070C1B300BE0907000200370080C1B300FB
:10D65000BB0907000080FA00000006000000FA0085
:10D66000D083290047E00700A085290045E0070096
:10D670000040EB0055FB070000C0EB001C08070052
:10D6800010C0B30051FB070010C0B3002AFB070015
:10D690000040EB004DFB07000080FA000000060090
:10D6A0000A00FA00881F7800C08729001FE00700E1
:10D6B0000000EB00000F78000D0037001E0478001A
:10D6C000CBFA0700804078006300470001747800BF
:10D6D0009E00780063004700614078000080FB00F6
:10D6E00003E1070000C2B300A5E107001E0FE80038
:10D6F000300020009E0F1000F0FF3600E07E290071
:10D7000020E00700A08A290008E007006300470026
:10D71000104078000080FB004400DE000080FB0029
:10D72000400798004E009000E90F500011003200B1
:10D730004E009000E90F500004003C004E009000A5
:10D74000E80F500008003200130037004E00900030
:10D75000EA0F50000A0032004E009000EF0F500018
:10D760000A0032000C003700508B290005E007004A
:10D770000B003700C08B290002E0070008003700CB
:10D78000308C2900FFDF070005003700A08C29003E
:10D79000FCDF070002003700E08C2900F9DF0700FA
:10D7A000608D2900E1DF0700630047001040900012
:10D7B0000080FB004700DE000004E00003003A00A8
:10D7C000208E2900EFDF070002003700908E29002D
:10D7D000ECDF0700908F2900D4DF070063004700CB
:10D7E000104090008080FB0080F72F0000806000D8
:10D7F0004380DE00204798002E4090000004E000A7
:10D8000003003A0060902900C8DF07001B003700C2
:10D810002E409000EF4F500003003A00A08C2900EA
:10D82000C2DF07001500370000042000000F780059
:10D83000E30047000040EB00804878000800370014
:10D840001E00780000004000000F780063004700D1
:10D85000104078008040E8006300470001487800ED
:10D8600063004700904078002E40900080CF500029
:10D87000F3FF39001E0078003DE00700E07E29003C
:10D88000C0DF070040912900A8DF070063004700C0
:10D890009040900070C0B30000C060002047980026
:10D8A00010002000000F7800E30047000040EB006C
:10D8B00080487800080037001E0078000000400013
:10D8C000000F780063004700104078008040E800B7
:10D8D00063004700014878006300470090407800EB
:10D8E0002E40900080CF5000F3FF39001E007800DA
:10D8F0004EE00700E07E2900A2DF07004F04780019
:10D900000080FA00000006000000FA0040168000C7
:10D91000017C200001007000401688000F00070005
:10D9200020C0B3002A00070006E107000004E00061
:10D930000400320009E10700250007000004E000B0
:10D9400004003A00220107000004E00001003A0050
:10D95000F5FF37000080FA00000006000000FA0022
:10D96000C222A9000000EB00400388000000EB0089
:10D97000500388000000EB00000388000000EB006B
:10D98000100388000000EB00F0088800D10A200096
:10D9900091407800F0C8B30000C06000ADE0B7006F
:10D9A0000000EB00E008880000642000D008880038
:10D9B0000000210000E188000040EB001EFCB700E1
:10D9C0000000EB0060E088000080FA000000060024
:10D9D0000A00FA00004F7800B0E08000400798008D
:10D9E000CE009000E18F5000410032004E019000C7
:10D9F000E10F5100040039004E009000E20F50008A
:10DA000048003200ED0037009E80FB00310798008F
:10DA10003E019000E20F5100150032003E009000E0
:10DA2000E20F500007003C00BE0090000100E00043
:10DA30000B0032003E019000E10F51000F00320058
:10DA4000220037003E009000F10F5000DB00320052
:10DA5000BE009000F38F5000D80032001B0037004A
:10DA6000BEFF07001200200022079800D5003700F3
:10DA7000A0072A002DDF0700D0003700C222A8002F
:10DA80000000EB00F00888000000EB00B008880000
:10DA90000000EB00A008880080002000F00888004B
:10DAA0008660A9009660A900D10A20009140780004
:10DAB000F0C8B30000C060000044A000ADE0B700B3
:10DAC0001000200060E08800BC0037001E40780095
:10DAD0000EFCB70040C0B30013FCB7000040EB00E1
:10DAE00014FCB70010002000B0E08800B30037003D
:10DAF00014DCBF000040E80014FCB70014DCBF00D9
:10DB00008080FB00E0C02100008040001E487800BB
:10DB100041C121009140780013DCBF0080CF50004C
:10DB2000A60039000EDCBF000080FB001007980043
:10DB3000100820009E009000808F500039003200B5
:10DB4000000C20001E019000800F510005003200E3
:10DB5000000820009E009000808F50004700320097
:10DB6000940037000FDCBF000080FB004400DE00A3
:10DB7000610060000004E000030032001003800038
:10DB80000000A000100388000FDCBF000080FB0035
:10DB90004300DE00610060000004E0000400320089
:10DBA00010038000010220000100700010038800B3
:10DBB0000FDCBF000080FB004200DE00610060005F
:10DBC0000004E00004003200100380000104200083
:10DBD00001007000100388000FDCBF000080FB0014
:10DBE0000000D100610060000004E0000400320089
:10DBF000100380000108200001007000100388005D
:10DC00000FDCBF000080FB00610060000004E0004A
:10DC10000400320010038000011020000100700099
:10DC20001003880010DCBF000080FB0000E18800CA
:10DC300000E180004800DD0000E188000FDCBF004B
:10DC40008080FB0000E180000080700000E188001F
:10DC500000E180004200DD006400400000E1880037
:10DC600001E1800000002100808F5000510036004B
:10DC70000000210000E188004E00370011DCBF00E9
:10DC80000080FB0001002000C0E08800D1E0880097
:10DC9000C0E08000D1E08000C808DD000080FD0009
:10DCA000804078000040EB00C0E08800D1E08800B0
:10DCB00010DCBF000081FB0003002000C0E08000FA
:10DCC000D1E080000000710081807100C0E0880018
:10DCD000D1E08800C0E08000D1E08000C808DD000D
:10DCE0000080FD00804078000040EB00C0E088002C
:10DCF000D1E088000FDCBF000081FB0003002000A2
:10DD0000C0E08000D1E080000000710081807100DF
:10DD1000C0E08800D1E08800C0E08000D1E0800051
:10DD20004209DD00CE00DE00810071004200DD000E
:10DD300064004000E08048009201200003002000C1
:10DD400011CB0700C0E08800D1E08800C2E080006D
:10DD5000D3E080000001200001002000800F51006E
:10DD6000818F590007003600C0E08000D1E08000BC
:10DD700070005000E0805800C0E08800D1E08800CA
:10DD8000040037001000200001002000C0E08800DF
:10DD9000D1E08800C0E08000D1E080004008DE00D3
:10DDA00001002000E0088800C0E08000D1E0800091
:10DDB000D00888000000EB00B0E088000000EB0015
:10DDC000200798002E0090000080FA000000060056
:10DDD0000200FA0060E08000E10F50000100320014
:10DDE0003600370086C0BF00684060000004E000D5
:10DDF00003003A00100380000000E0002F003A000A
:10DE00001FE1A8008780A9000000EB00E0E0880087
:10DE10000F003700E2E08000501680004600DE0070
:10DE20008040780000802000000041000148780018
:10DE300087C0BF00704060000004E000FCFF3200BB
:10DE40008780A900E0E080000000E800E0E08800B2
:10DE5000E1E0800000E18000808F5000EDFF39009C
:10DE60000000EB00100388000000EB00F0088800C1
:10DE700000E18000E0E0880009003700E0E0800079
:10DE80008000E90000802000008040001040780001
:10DE9000BBDF0700E0E080000000E900E0E0880070
:10DEA000E0E080000000E000F4FF3A00ABFE070075
:10DEB00010002000000F7800020037000000EB0087
:10DEC000000F78001E0078000080FA0000000600B5
:10DED0001400FA00881F78000000EB00800888001A
:10DEE0000000EB00F00888000000EB00E00C880068
:10DEF00010E48000E20F50000A003A00A16C2000FC
:10DF00009140780000CEB30000C06000CAE6B700C0
:10DF100000C629001BDE07000000EB0010E48800AB
:10DF200080003700D0C6290016DE0700A0C92900EE
:10DF3000FEDD07002203200001FA2000400020003F
:10DF40005BDC070030079800C0CA2900F7DD070036
:10DF50003E009000E30F500007003E0060CB290018
:10DF600008DE0700E00320002007980010A1A800A9
:10DF70001081A8001B0037003E009000FE0F5000EB
:10DF800007003E00A0CB2900FEDD0700A00F200007
:10DF90002007980010A1A8001081A90011003700E7
:10DFA000BE009000400F2000808F500007003E0010
:10DFB000D0CB2900F3DD0700007D2000200798006A
:10DFC00010A1A9001081A80006003700F0CB29009D
:10DFD000ECDD070000E823002007980010A1A9004D
:10DFE0001081A9002E0090003E0190001100090050
:10DFF0000280D8000000E9005007980010CC2900EA
:10E00000CADD07005E00900059DE070060CC2900E1
:10E01000DCDD070070CC2900C4DD070022032000EE
:10E02000310620002000200021DC070000047800D9
:10E030006140B9003AC90700000F9800110F98001D
:10E040000800E00007003D000200200003782400E3
:10E050000E0890009E0890005DC90700000F980010
:10E06000110F98000E0890009E089000008FBE00CF
:10E0700002002000832C24001E00BE00B1C907004E
:10E08000008FBE005E009000CF80DE0024C9070034
:10E0900060079800710798005E0090000000E000A3
:10E0A00007003D0002002000037824006E0090006D
:10E0B000FE00900046C907006007980071079800AD
:10E0C0001E01BE006E009000FE009000DFC9070038
:10E0D00012CA070040079800A16C20009140780008
:10E0E00000CEB30000C060006041B300CAE6B700D4
:10E0F000CE009000D10C88004E009000C00C88002B
:10E1000060002000E00C8800DE00900061088800BC
:10E1100011E1A80080CD29009ADD07002000200031
:10E1200010E488004F0478000080FA000000060028
:10E130000000FA0010E48000E20F500003003A00F3
:10E1400030CE29008FDD07007900370040D029004C
:10E1500076DD07000000EB00F00888000000EB000F
:10E1600080088800C942A8006168200091407800BA
:10E1700000CEB30000C06000A040B30086E6B70048
:10E18000A0032000800888000080EB007008880051
:10E190000080EB00600888000000EB004008880069
:10E1A0000000EB00300888000000EB00B008880099
:10E1B0000000EB00A008880080002000F008880024
:10E1C000400F2000E008880000402200D0088800AE
:10E1D0008780A9001FE1A80011E1A80087C0BF0047
:10E1E000704060000004E000FCFF320011E1A90073
:10E1F0001FE1A9003008800050E48800400880003A
:10E2000040E4880040E480000100200020E4880011
:10E2100031E4880020E4800031E48000C000DD00AB
:10E220000000200020E4880031E4880050E48000F1
:10E230006101B80020E4800031E480000200400069
:10E240008380480020E4880031E4880020E48000D6
:10E2500031E48000C808DD000080FD0080407800C7
:10E260000040EB0020E4880031E4880020E48000D6
:10E2700031E480007ADD0700B0D129002BDD0700F2
:10E2800022E4800033E48000703E20000100200082
:10E29000800F5100818F59001C00360022E480005D
:10E2A00033E48000F0232400F1002000800F5100AF
:10E2B000818F59000B003E00E0D129001BDD0700D3
:10E2C00020E4800031E48000823E20000300200032
:10E2D000ADC9070062DD070010D2290013DD070079
:10E2E0000A003700E0D1290010DD070020E480009B
:10E2F00031E4800002242400F3002000A2C90700BA
:10E3000057DD070060D2290008DD070060CC290036
:10E310001CDD070086C6BF00F041B30086E6B700EB
:10E320000000EB00F00888000000EB008008880087
:10E330000080FA00000006000000FA000BD8BF00C1
:10E34000614060000004E00002003A00C942A800F9
:10E3500001003700C8C2A800B0D2290009DD0700BB
:10E360000080FA00000006000000FA000BD8BF0091
:10E37000614060000004E00003003A00C942A900C7
:10E38000CB42A80002003700C8C2A900CAC2A80038
:10E39000A0D32900FBDC07000080FA000000060083
:10E3A0000000FA000BD8BF00614060000004E000EC
:10E3B00003003A00C942A900CB42A900020037007D
:10E3C000C8C2A900CAC2A90030D42900EDDC0700E8
:10E3D0000080FA00000006000200FA000BD8BF001F
:10E3E000614060000004E00009003A00C942A80052
:10E3F0000000000000000000CBC2BF000080FB0056
:10E400004200DE0061406000004F780008003700E5
:10E41000C8C2A8000000000000000000CAC2BF007F
:10E420000080FB004600DE0061406000004F780085
:10E43000B0D42900BDDC07001E407800B4DC070022
:10E4400060CC2900CFDC07000080FA000000060045
:10E450000000FA0040072A00B4DC07000080FA0040
:10E46000000006000600FA000BD8A8000B78A900EF
:10E4700010C0B3000AF8B70020C0B300C2FCB70058
:10E4800080C0EB0020C0B30082F60700C922A900BB
:10E49000C902A900C8E2A80010C0B300CBF707006A
:10E4A000EBFF07000000370022C2BF0061406000A0
:10E4B0000004E000FCFF320030118000C5FCB70012
:10E4C000C5DCBF000080FB004400DE00C4FCB700D8
:10E4D000C4DCBF000080FB00000F78001E00780045
:10E4E000E30F5000A60032009E007800E38F50003A
:10E4F0000A003C001E017800E10F51006E0032005E
:10E500009E017800E18F510090003C001E007800D1
:10E510000000E0000B003200FB0037009E00780096
:10E52000E68F5000C40032001E017800E80F510051
:10E53000D10032009E017800E48F5100B900320012
:10E54000F1003700C5DCBF000080FB006101B900AD
:10E550001207980023079800D00020000100200037
:10E560001E019000AE019000800F5100818F590074
:10E570004E003E001E009000AE00900000600100C2
:10E58000E40037000C0037000D00370010003700A2
:10E5900013003700170037001B0037002400370036
:10E5A00026003700280037002C00370030003700E5
:10E5B0003400370038003700A5FF0700BAFF3700E6
:10E5C0006FF6070010C0B300EDDD0700B6FF37009F
:10E5D0007EF6070010C0B300E9DD0700B2FF370088
:10E5E0000040EB0079F7070010C0B300E4DD07003E
:10E5F000ADFF370010C0B30074F7070010C0B300C0
:10E60000DFDD0700A8FF3700C2DCBF00E24F50008B
:10E6100003003A00F6F60700D9DD0700A2FF370035
:10E6200000C0EB0078F60700D5DD07009EFF37003D
:10E630001FF70700D2DD07009BFF37006CF70700CC
:10E64000CFDD070098FF370010C0B3003AF707008E
:10E6500010C0B300CADD070093FF37000040EB0095
:10E6600051F7070010C0B300C5DD07008EFF37006B
:10E6700010C0B3004CF7070010C0B300C0DD0700A6
:10E6800089FF37000040EB003EF7070010C0B300E1
:10E69000BBDD070084FF370010C0B30039F7070067
:10E6A00010C0B300B6DD07007FFF37000040EB006D
:10E6B000B3DD07007CFF370051CC2100914078008A
:10E6C000F0C0B30000C06000C5FCB700C5DCBF00EF
:10E6D0000040E800C5FCB70010C0B300A8DD07008B
:10E6E0000040EB00C3FCB7001200370022C2BF009D
:10E6F000614060000004E000FCFF3200C2DCBF00AB
:10E70000E24F500005003A003011800087F6070004
:10E7100010C0B3009ADD07000300370030118000FD
:10E7200039F6070096DD0700C3DCBF000040E800B3
:10E73000C3FCB70031CC210091407800C5DCBF009C
:10E7400080CF5000E9FF390057FF370051CC21003E
:10E7500091407800F0C0B30000C06000C5FCB70075
:10E76000C5DCBF000040E800C5FCB700C5DCBF0049
:10E77000F1F6070010C0B30081DD07004AFF370043
:10E7800051CC210091407800F0C0B30000C060007F
:10E79000C5FCB700C5DCBF000040E800C5FCB70001
:10E7A00010C0B30076DD070022C2BF0061406000E8
:10E7B0000004E000FCFF320030118000C4FCB70010
:10E7C0000040EB00C3FCB7000E003700C4DCBF0004
:10E7D0000004E00003003D0010C0B300C5F60700D0
:10E7E000020037000040EB00C2F60700C4DCBF00A7
:10E7F00000404000C4FCB700C3DCBF000040E8009C
:10E80000C3FCB70031CC210091407800C5DCBF00CB
:10E8100080CF5000EDFF390010C0B30058DD070075
:10E8200021FF3700C5DCBF000505070010C0B3009D
:10E8300053DD07001CFF370051CC210091407800C8
:10E8400030C0B30000C06000C5FCB700C5DCBF002D
:10E850000AF8B700A180210091407800C2DCBF0017
:10E860008CF5070010C0B300D8F6070010C0B30045
:10E8700043DD07000CFF37000BD8A900C5DCBF0043
:10E880000080FB004300DE000000A2006100600089
:10E890000004E000010032000BD8A80020C0B30043
:10E8A000C2FCB700C5DCBF000080FB004200DE00F8
:10E8B000610060000004E0000200320030C0B300DC
:10E8C000C2FCB7000B78A900C5DCBF000080FB00CC
:10E8D0000000D100610060000004E000010032008F
:10E8E0000B78A800A180210091407800C2DCBF0015
:10E8F00068F5070010C0B300B4F6070010C0B300FD
:10E900001FDD0700E8FE37000040EB001CDD0700BC
:10E91000E5FE37000080FA00000006000200FA0061
:10E92000004F7800114798000040EB00C9FCB70089
:10E930001E407800C8FCB700C8DCBF000004E0003F
:10E940000D0032001E4090000004E0000A0032007A
:10E9500060B52900F4000700D0B62900F2000700D6
:10E9600050B92900F0000700F6DC07000004E000C1
:10E97000FDFF3200F9DC0700A0BA2900EA00070019
:10E98000CB42A800C942A900F0BA2900EF00070055
:10E99000CBC2BF000080FB004200DE00614060008F
:10E9A00011C0B300D0000700CB42A900C942A800A3
:10E9B000C222A800C022A90030BB2900E300070042
:10E9C000C2C2BF000080FB000000D10061406000B7
:10E9D00011C0B300C4000700C222A900C962A80088
:10E9E000CB62A900C0BB2900D8000700CBC2BF0082
:10E9F0000080FB004300DE006140600011C0B300F6
:10EA0000B9000700CB62A900C962A90050BC290067
:10EA1000CE000700CBC2BF000080FB004300DE0039
:10EA2000614060008040EB00AF000700C002A90019
:10EA3000C202A80020C0B30014030700E0BC2900F4
:10EA4000C2000700C2C2BF006140600011C0B30035
:10EA5000A500070030BD2900B300070021E3A8008E
:10EA600020BE2900B900070072352000712B20005C
:10EA700090C0B3005B0007001E4090000004E0005F
:10EA80000600320050BE2900B00007007235200099
:10EA9000712B2000B0C0B3005200070090BE2900C7
:10EAA000AA00070002252000011B2000A0C0B3001F
:10EAB0004C0007001E4090000004E00006003200F9
:10EAC000E0BE2900A100070002252000011B200054
:10EAD000C0C0B3004300070021E3A90020BF290004
:10EAE0009100070041168000F0C32F0000806000F5
:10EAF0004016880061168000003C200000807000F5
:10EB00006016880040C6B300E002070010C0B300E2
:10EB100054000700B0BF2900830007006116800081
:10EB2000F0C32F0000806000601688001E40900037
:10EB30000004E00002003200C962A800CB62A90014
:10EB400040C6B300D10207000040EB0045000700BB
:10EB50001E4090000004E0000A00320060C029005E
:10EB60007100070040168000013C20000100700089
:10EB70004016880040C6B300C402070010C0B300AE
:10EB800038000700C8DCBF000004E00010003200BD
:10EB90001E4090000004E0000D003200C002A900F9
:10EBA000C202A800C222A80010C129005E0007000E
:10EBB00064DC07000004E000FDFF320067DC0700B2
:10EBC000C222A900C022A800C002A900C202A90056
:10EBD0002A020700C9DCBF000080FB000080FA00A9
:10EBE000000006000A00FA0020479800210798005C
:10EBF0003207980010C42900540007002E409000EE
:10EC00003E020700000F7800C8DCBF000004E000EF
:10EC1000020032001E00780006DC070030C4290024
:10EC20004A0007002E0090009E0F100006003600DC
:10EC30003E0090009E0F10000300310010002000E5
:10EC400040079800020037000000EB0040079800E2
:10EC50000E48900011C0B300230007000080FA00A6
:10EC6000000006000200FA00004F780050C429009E
:10EC700036000700CBC2BF000080FB000000D100BF
:10EC8000614060009E40780017000700A0C4290082
:10EC90002E000700CBC2BF00614060009E4078009C
:10ECA00011000700E0C4290028000700CAC2BF0005
:10ECB0000080FB004700DE009E4078000A0007004D
:10ECC00030C5290021000700CAC2BF000080FB0038
:10ECD0004600DE00614060009E40780002000700B0
:10ECE0000080FA00000006000200FA00004F7800E1
:10ECF000114798001E4090009E4F100003003A00FC
:10ED000060C529000800070005003700A0C52900DC
:10ED100005000700C9DCBF000040E800C9FCB700DF
:10ED20000080FA00000006000200FA00000F7800E0
:10ED3000C8DCBF000004E000020032001E007800C2
:10ED400090DA07000080FA00000006000200FA00D6
:10ED5000000F7800C8DCBF000004E00002003200B1
:10ED60001E00780071DA07000080FA00000006003B
:10ED70000400FA000CD8BF000080FB006101B9005C
:10ED8000028FBE00D0012000010020001E01BE0045
:10ED9000800F5100818F5900D1003E001E00BE003F
:10EDA000006001001D0037003D003700670037009C
:10EDB0006600370070003700C60037007400370067
:10EDC0007A00370080003700860037008A0037005D
:10EDD0008E00370092003700C1003700C0003700B6
:10EDE000BF003700BE003700BD003700BC00370051
:10EDF000BB003700BA003700B9003700B800370051
:10EE0000B7003700B60037008A003700A40037008B
:10EE1000B5003700B2003700B300370080C0800073
:10EE2000E10F500006003A0010C0B300C403070011
:10EE300000C0EB0074F40700F6010700150037006E
:10EE400020C0B300BE03070080C08000F1010700AE
:10EE500030C0B300BA0307000000EB0030E58800C3
:10EE60000800370000C0EB0067F40700E901070065
:10EE700000C2B300C2DB070030E580000000E800FC
:10EE800030E5880081C0800030E58000808F500030
:10EE9000F4FF3E0080062A003ADA070092003700AD
:10EEA00040C0B300A603070070C08000D90107006E
:10EEB00080C08000E10F50000E003A0070C080005A
:10EEC00051F40700A8FCB700AADCBF006140600055
:10EED0000004E0001A00320000C2B300A8DB070003
:10EEE00010C0B30096030700A8DCBF00C9010700EB
:10EEF0001300370090062A000CDA070080C080005B
:10EF0000C401070050C0B3008D0307000000EB00F0
:10EF100030E588000600370070C080003AF4070032
:10EF2000A8FCB70030E580000000E80030E588006C
:10EF300081C0800030E58000808F5000F6FF3E00E9
:10EF400080062A000FDA0700670037000CD8BF00E0
:10EF5000E34F500002003A00AA1CA800010037004D
:10EF6000AA1CA9000040EB0018F50700A0C0B300E0
:10EF7000730307005C003700AA1CA90010C0B3008F
:10EF800012F50700B0C0B3006D030700560037004C
:10EF9000D0C0B3006A030700C5F40700DCD907003E
:10EFA00080062A00F7D907004F003700E0C0B30001
:10EFB000630307000EF50700D5D9070080062A0075
:10EFC000F0D907004800370080C080009101070099
:10EFD00000C1B3005A03070080C08000D6F40700C8
:10EFE0004100370010C1B3005503070010C0B30043
:10EFF000EDF407003C00370020C1B30050030700C8
:10F000000040EB00E8F407003700370030C1B300E0
:10F010004B03070010C0B300DAF4070032003700DA
:10F0200040C1B300460307000040EB00D5F40700E1
:10F030002D00370010C3B300410307001200200069
:10F04000410020001000200019D807000040E9000E
:10F050000AF8B700E0C1B30039030700120020002E
:10F06000210020001000200011D807000040EA0015
:10F0700061406000614060004601DD00B180210018
:10F0800091407800F0CBB30000C0600002407000F7
:10F090000BF8B7000B58A8000B98A8001200370017
:10F0A000AA1CA900A18021009140780030C0B300C3
:10F0B00078F30700C922A900C902A900C8E2A80084
:10F0C00010C0B300C1F407000040EB001C030700B0
:10F0D0000500370070C1B3001903070002003700B4
:10F0E00080C1B300160307000080FA00000006008C
:10F0F0000200FA00F0C2B300104798000040EB0095
:10F10000004F7800C922A800CB22A900C922A9007B
:10F1100005003700A0C0B300750107001E40900035
:10F120000040E900104798001E4090000004E000F5
:10F13000F8FF3C00C922A800C0C3B3006C0107005F
:10F14000CBC2BF000080FB000000D1006140600026
:10F15000BAFCB70090C2B300104798000500370012
:10F16000A0C0B300620107001E4090000040E9000B
:10F17000104798001E4090000004E000F8FF3C009B
:10F18000CBC2BF000080FB000000D10061406000E6
:10F19000BBFCB700BBDCBF000004E00002003A008B
:10F1A00010C0B300004F7800BADCBF00E14F500040
:10F1B00003003A001E40780000C0E800004F7800CD
:10F1C000A0C0B3004A0107001E80FB000080FA00C7
:10F1D000000006000400FA002047980080C0B30039
:10F1E000004F78001D0037002E4090006140600005
:10F1F000BCFCB700CB22A900C922A90050C0B300B3
:10F200003B010700BCDCBF00614060006140600062
:10F2100000414000912C200091407800D0CFB300F5
:10F2200000C0600002407000C9E2B70020C3B30014
:10F230002F01070050C0B3002D010700C922A8000C
:10F24000A0C0B3002A0107002E4090000080FB0000
:10F250000000D100204798001E4FE9001E04E00086
:10F26000E1FF3C00A0C0B300210107000080FA00CC
:10F27000000006000200FA00004F7800CB22A9002F
:10F28000C922A90050C0B300190107009E407800B0
:10F2900061C060006140600000414000912C20008E
:10F2A00091407800D0CFB30000C0600002407000F1
:10F2B000C9E2B70020C3B3000D01070050C0B3007E
:10F2C0000B010700C922A800A0C0B3000801070075
:10F2D0000080FA00000006000200FA0080C0B300BF
:10F2E000104798000040EB00004F78001D003700E9
:10F2F000CB22A900C922A90030C0B300FC0007003E
:10F30000C922A80050C0B300F9000700CBC2BF005B
:10F310000080FB000000D10061406000BCFCB70031
:10F3200040C3B300F20007001E80FB000000D100C4
:10F33000004F7800BCDCBF00E14F500004003A00F1
:10F340001E40780001C8B30001404000004F780023
:10F35000A0C0B300E60007001E4090000040E90096
:10F36000104798001E4090000004E000E0FF3C00C1
:10F37000A0C0B300DE0007001E80FB000080FA0082
:10F38000000006000000FA00CB22A900C922A90053
:10F3900030C0B300D6000700C922A80050C0B30097
:10F3A000D3000700CBC2BF000080FB000000D100EB
:10F3B00061406000BCFCB70040C3B300CC00070054
:10F3C000A0C0B300CA000700BCDCBF000080FB0087
:10F3D0000080FA00000006000800FA0020079800EC
:10F3E000310798000040EB00004F78000000EB0070
:10F3F000100798000D0037001E0090008000780074
:10F400002E00900000804000104078001E406800F0
:10F410008080FB0020D6290000804000104F78003B
:10F420001E0090000000E800100798009E00900069
:10F430003E009000808F5000EFFF35001E80FB00E3
:10F440000080FA00000006000000FA000BD8A900B6
:10F450000040EB000AF8B7000B38A9000B18A90010
:10F460000B58A9000B78A9000B98A9000BB8A900AC
:10F470000BF8A9000080FA00000006000000FA0066
:10F48000C922A800C902A800C8E2A800C8C2A800F2
:10F49000C942A800C222A900C022A9000000EB00B6
:10F4A00020C08800E8FF0700CB62A900C962A9005C
:10F4B000C002A900C202A9002D23A9002D43A90062
:10F4C0002D63A9002D83A90001322000914078000E
:10F4D00000CEB30000C0700020E3B7000000EB00D6
:10F4E0008019880020F02100201988000000EB001E
:10F4F000101988000080FA00000006000200FA00DF
:10F50000004F78001E80FB00401988002023A800CF
:10F510002003A90020C3BF00614060000004E00098
:10F52000FCFF3200001880000080FA000000060096
:10F530000000FA0021E3A800C0C0B300EFFF0700FD
:10F54000BCD9070021E3A9000080FA0000000600F2
:10F550000200FA0040FF29008AD8070030002A0084
:10F5600088D8070090012A0070D807000000EB003F
:10F57000B0D9070090022A006CD807000B003700B2
:10F5800021E3A800C0C0B300DCFF0700000F780033
:10F5900021E3A900B0022A0064D807001E00780009
:10F5A000A4D9070090022A0060D80700E5D9070017
:10F5B0000004E000F2FF3200E8D9070010032A003F
:10F5C00070D807000080FA00000006000000FA0072
:10F5D00000D8BF000080FB008000400060C3210015
:10F5E0000080400010007800401188000000EB000F
:10F5F000001188002062A8000000EB0010118800B4
:10F6000021E2A8002342A8008560A9000080FA003A
:10F61000000006000400FA00004F780010C08000CF
:10F62000100798001E009000E10F50000D003200FE
:10F630001E009000E10F5000070039001E009000EE
:10F64000E20F50000A0032001E009000E30F50004D
:10F650000A0032000B0037001E80FB0024D907008F
:10F66000080037001E407800F0D80700050037007A
:10F670001E4078005DD80700020037001E40780069
:10F68000BFD907000080FA00000006000600FA005B
:10F69000404798000040EB00204798000E003700DC
:10F6A0000000EB00000F780005003700A0CFB3008A
:10F6B0000F0007001E0078000000E800000F78002F
:10F6C0001E007800E30F5000F8FF36002E40900037
:10F6D0000040E80020479800AE4090004E40900067
:10F6E00080CF5000EEFF39000080FA0000000600D5
:10F6F0000400FA00204798000040EB00004F78001B
:10F7000013003700000000000000000000000000AF
:10F7100000000000000000000000000000000000E9
:10F7200000000000000000000000000000000000D9
:10F7300000000000000000000000000000000000C9
:10F74000000000001E4078000040E800004F7800F4
:10F750009E4078002E40900080CF5000E9FF390095
:10F760000080FA00000006000400FA004B000700C9
:10F770000000370022C2BF00624060000004E000C9
:10F780000400320010118000D1FF2F000100600042
:10F79000101188000280200001002100208121003A
:10F7A0007CD6070010079800E00F20009E00900014
:10F7B000808F50002B003200F00F20009E00900040
:10F7C000808F50001F0032001E009000E10F50009B
:10F7D000010032002900370091C08000010F78003D
:10F7E0001E0078000000E000040032009E00780057
:10F7F000E18F5000040032000700370090C1B300D1
:10F800004F0107000700370000C8BF00C4E607002B
:10F810000004E00003003A0090C080000180200056
:10F8200068F307000000EB0090C088000040EB0088
:10F83000C7FCB700EF000700E0C3B30050D90700D2
:10F840000E003700C7DCBF000040E800C7FCB7006F
:10F85000C7DCBF00F34F5000080036003AE907004C
:10F8600006003700C7DCBF00E44F5000010036003F
:10F8700025F807000040EB00C7FCB7000BD8BF001D
:10F88000624060000004E000BAFF320070C1B300C3
:10F890000CF8B70097000700B6FF37000000FA0029
:10F8A0004507A9000080EB00601988004227A900E5
:10F8B000416A20009140780000CEB30000C0600093
:10F8C0005040B300A4E6B700416C2000914078009E
:10F8D00000CEB30000C060003040B300C4E6B70003
:10F8E00080C0B30000F8B7000000EB0010C0880033
:10F8F000E2FE070035FF07008000EB00F00F20005C
:10F90000A6D9070030C0880021002000F00F200099
:10F91000A2D9070040C0880060082A0099D70700D4
:10F920005EE70700B3000700E0C3B30014D9070087
:10F930000080FA00000006000600FA00000F7800C0
:10F940002147980032479800434798005447980051
:10F950002E40900061406000614060000041400026
:10F96000F12C200091407800D0CFB30000C060009F
:10F9700002407000CFE2B700616A20009140780039
:10F9800000CEB30000C060007040B300A6E6B70030
:10F99000916C20009140780000CEB30000C0600060
:10F9A0005040B300C9E6B7001E007800C0118800BF
:10F9B0000000EB00801188003062A8003E409000FB
:10F9C00061406000614060004401DD0001232000CF
:10F9D00091407800F0CEB30000C06000024070009B
:10F9E00030E2B7004E40900063406000634060002A
:10F9F00000414000012320009140780090CFB300E7
:10FA000000C060000240700030E2B7005E4090002D
:10FA10006140600061416000012320009140780056
:10FA2000E0CFB30000C060000240700030E2B700D9
:10FA30000000EB00901188000080FA000000060032
:10FA40000000FA0031E2A8003342A80087C0A900F4
:10FA50000080FA00000006000000FA0031E2A90070
:10FA60003342A900A6C6BF00F041B300A6E6B70026
:10FA7000616C20009140780000CEB30000C06000AF
:10FA8000C6E6B700CF22A9000080FA0000000600F9
:10FA90000200FA00004F780033C2BF0062406000ED
:10FAA0000004E000FCFF3A001E80FB00A01188006B
:10FAB0000080FA00000006000000FA0032C2BF0019
:10FAC000614060000004E000FCFF3200B0118000E3
:10FAD0000080FB000080FA00000006000000FA0031
:10FAE00032C2BF00614060000080FB000080FA006D
:10FAF000000006000200FA0020C08000000F78001D
:10FB00001E007800E50F5000290032001E0078002A
:10FB1000E50F500011003E001E007800E20F50007B
:10FB20001D0032001E007800E20F500004003E006D
:10FB30001E007800E10F500015003200260037004B
:10FB40001E007800E30F5000150032001E00780000
:10FB5000E40F5000140032001F0037001E00780030
:10FB6000E70F5000160032001E007800E70F50002B
:10FB7000110039001E007800E80F5000120032001A
:10FB80001E007800E90F500011003200120037000B
:10FB90005FD1070011003700B4DF07000F00370006
:10FBA0005FDC07000D00370009D907000B003700A4
:10FBB000CFE2070009003700C6F50700070037004D
:10FBC0006BFC070005003700AAEC070003003700B4
:10FBD00097EA070001003700C222A9000080FA005E
:10FBE000000006000000FA00A00020000080FA00DB
:10FBF000000006000000FA0020C0800080004000E5
:10FC000020C221000080400010007800C7D6070005
:10FC10000080FA00000006000200FA00004F7800A1
:10FC20001E80FB008000400020C2210000804000B8
:10FC300010007800BDD607000080FA000000060022
:10FC40000200FA00004F78001E80FB004300DE0037
:10FC5000610060000004E00003003200C002A9005F
:10FC6000C202A80002003700C002A900C202A90017
:10FC70001E80FB004200DE00610060000004E00026
:10FC800003003200C962A800CB62A900020037005D
:10FC9000CB62A900C962A9001E80FB000000D10050
:10FCA000610060000004E00003003200C942A900C6
:10FCB000CB42A80002003700C942A900CB42A900EC
:10FCC0001E80FB00610060000004E00012003200B2
:10FCD0000BD8BF000044B2000004E0000500320071
:10FCE00040168000010420000100700040168800CA
:10FCF00011003700611680000004200000807000B1
:10FD00006016880041168000F0FB2F000080600024
:10FD1000401688000800370061168000F0FB2F00B5
:10FD2000008060006016880041168000F0FB2F0004
:10FD300000806000401688000080FA000000060085
:10FD40000200FA00004F78001E80FB008000400097
:10FD500040AA2100008040001000780073D6070000
:10FD60000080FA00000006000200FA000000EB002C
:10FD7000000F7800090037001E0078008000400066
:10FD800000B12100008040001000780067D6070015
:10FD900060EA28007BD607001E0FE8003002200032
:10FDA0009E0F1000F4FF36000080FA0000000600ED
:10FDB0000000FE00FFFFFF00FFFFFF00FFFFFF004E
:10FDC000FFFFFF00FFFFFF00FFFFFF00FFFFFF003F
:10FDD000FFFFFF00FFFFFF00FFFFFF00FFFFFF002F
:10FDE000FFFFFF00FFFFFF00FFFFFF00FFFFFF001F
:10FDF000FFFFFF00FFFFFF00FFFFFF00FFFFFF000F
:020000040001F9
:00000001FF
